:100000000C942B080C944A080C944A080C944A0847
:100010000C944A080C944A080C94550A0C948B0AC8
:100020000C944A080C944A080C944A080C944A0808
:100030000C944A080C944A080C944A080C94F80D45
:100040000C944A080C944A080C944A080C944A08E8
:100050000C9406540C94284B0C944A080C944A08AF
:100060000C944A080C94FD4B0C944A080C94F14BE8
:100070000C944A080C944A080C944A080C944A08B8
:100080000C947E5F0C944A080C944A080C944A081D
:100090000C943B4C0C944A080C942F4C0C944A083A
:1000A0000C944A080C944A080C944A080C944A0888
:1000B0000C944A080C944A080C944A080C944A0878
:1000C0000C944A080C944A080C944A080C944A0868
:1000D0000C944A080C944A080C944A080C944A0858
:1000E0000C944A080C94BF530C94C9530C94B55308
:1000F0000C946F530C94FA530C94EB530C94DF5301
:100100000C94D3530C944A080C944A080C944A0853
:100110000C944A080C944A080C944A080C944A0817
:1001200007634236B79BD8A71A39685618AEBAABE0
:10013000558C1D3CB7CC5763BD6DEDFD753EF61774
:100140007231BF000000803F08000000BE922449C9
:10015000123EABAAAA2ABECDCCCC4C3E00000080F9
:10016000BEABAAAAAA3E00000000BF000000803F6C
:100170000000000000084178D3BB4387D1133D192C
:100180000E3CC3BD4282AD2B3E68EC8276BED98F59
:10019000E1A93E4C80EFFFBE01C4FF7F3F0000009D
:1001A00000000A0025303278002025362E326620E5
:1001B0004F6E2D426F61726400202573002530322E
:1001C00078002025362E3266200020257300415409
:1001D00032344D4143200048494836313330200005
:1001E000424D5030383520004144584C333435208E
:1001F00000484D433538383320004C3347343230D3
:10020000304420004E484443303231362000756E71
:100210006B6E6F776E20636D640A00256300682043
:1002200020202020202020202020202020202020CE
:10023000202020202020202020202D2068656C7088
:100240000A0D0076202020202020202020202020A1
:100250002020202020202020202020202020202D91
:100260002076657273696F6E0A0D0075202020205C
:10027000202020202020202020202020202020207E
:10028000202020202020202D20757074696D650AA3
:100290000D00616573205B6F6E7C6F66665D20206C
:1002A00020202020202020202020202020202D2041
:1002B000696E746567726574790A0D006164632004
:1002C000202020202020202020202020202020202E
:1002D00020202020202020202D2073686F7720767A
:1002E0005F696E2C2061312C20613220766F6C7436
:1002F000616765730A0D0063616C69205B5B765F03
:10030000696E7C61317C61325D20766F6C747C72C9
:10031000657365747C6E6F6E655D202D2063616C06
:100320006962726174650A0D006465205B6D6173BA
:100330006B5D202020202020202020202020202035
:1003400020202020202D2064656275670A0D00683A
:10035000756D2020202020202020202020202020FB
:1003600020202020202020202020202D2068756D96
:1003700069646974792073656E736F720A0D006821
:10038000756D70205B6F6E7C6F66665D202020202F
:1003900020202020202020202020202D2068756D66
:1003A0006964697479207065726D2073656E736F0E
:1003B00072207077720A0D006964205B7265736544
:1003C000745D20202020202020202020202020209C
:1003D000202020202D2069642068616E646C696E85
:1003E000670A0D006D63752020202020202020202A
:1003F00020202020202020202020202020202020FD
:100400002D206D637520696E666F0A0D006572722E
:1004100020202020202020202020202020202020DC
:100420002020202020202020202D206572726F7235
:1004300020696E666F0A0D006E65205B666C7573D1
:10044000685D202020202020202020202020202027
:10045000202020202D206E65696768626F722074ED
:1004600061626C650A0D006C6F67205B6175746F6B
:100470007C6F6E7C6F66665D20202020202020200F
:100480002020202D206D6F746573206461746120BD
:100490006F6E205553420A0D006F772020202020D8
:1004A000202020202020202020202020202020204C
:1004B00020202020202D206F6E652D776972652009
:1004C00073656E736F72730A0D007265205B6D61E8
:1004D000736B5D2020202020202020202020202041
:1004E0002020202020202D206D6F746520726570E3
:1004F0006F72742073657474696E670A0D00726997
:10050000205B696E745D2020202020202020202088
:10051000202020202020202020202D207265706F98
:10052000727420696E74657276616C0A0D00727364
:1005300020202020202020202020202020202020BB
:10054000202020202020202020202D20726164697E
:100550006F2073746174730A0D0073732020202060
:10056000202020202020202020202020202020208B
:100570002020202020202D2073797374656D207336
:10058000756D6D6172790A0D0074787077205B313A
:10059000352D305D202020202020202020202020EC
:1005A00020202020202D205458205077722E2048C3
:1005B000696768657374203020283364426D290AA6
:1005C0000D0070777231205B6F6E7C6F66665D2008
:1005D00020202020202020202020202020202D200E
:1005E00070696E31207077720A0D007031205B6F78
:1005F0006E7C6F66665D2020202020202020202039
:10060000202020202020202D2064697361626C65E9
:100610002070756C736520703120746F2073617663
:100620006520706F7765720A0D00726573742065BE
:100630006570726F6D202020202020202020202037
:100640002020202020202D20726573746F72652079
:10065000656570726F6D0A0D0070777273205B6450
:100660006565707C666F7263655F69646C655D204B
:1006700020202020202D206D637520736C6565700F
:10068000206D6F64650A0D00626F6F74202020205A
:10069000202020202020202020202020202020205A
:1006A000202020202D207265626F6F740A0D007566
:1006B0007067722020202020202020202020202051
:1006C00020202020202020202020202D2072656244
:1006D0006F6F742076696120626F6F746C6F6164F4
:1006E00065720A0D00776474205B6F6E7C6F6666BE
:1006F0007C746573745D2020202020202020202021
:10070000202D207761746368646F670A0D0074653B
:100710007374205B6F66667C317C327C335D202095
:10072000202020202020202020202D20746573747C
:10073000206D6F6465730A0D00557074696D6520D6
:10074000256420646179732C20253032643A253089
:1007500032643A253032640A00204E657665722D87
:100760007573656420737461636B203E202564207B
:1007700062797465730A0025352E326620002537AC
:100780002E33662025372E3366002530327800520E
:100790005F49442000525F542000525F54312000D2
:1007A000525F545F4D43552000525F565F4D435595
:1007B0002000525F50302000525F50305F542000C4
:1007C000525F50312000525F50315F542000525F21
:1007D000555054494D452000525F52482000525F09
:1007E000565F494E2000525F41312000525F413236
:1007F0002000525F502000525F50412000525F495C
:10080000443D09093078257800525F543D0909308C
:1008100078257800525F54313D09093078257800F9
:10082000525F545F4D43553D093078257800525F43
:10083000565F4D43553D093078257800525F503062
:100840003D09093078257800525F50305F543D09EA
:10085000093078257800525F50313D0909307825FC
:100860007800525F50315F543D0909307825780097
:10087000525F555054494D453D0930782578005216
:100880005F52483D09093078257800525F565F492C
:100890004E3D09093078257800525F41313D090904
:1008A0003078257800525F41323D0909307825784B
:1008B00000525F503D09093078257800525F504161
:1008C0003D0909307825780025730A004E657720A8
:1008D00064656275673D307825580A004375727209
:1008E000656E742064656275673D307825580A002E
:1008F000445F4F5045523D307825780A00445F529E
:10090000583D307825780A00445F54583D307825AA
:10091000780A00445F504B543D6E307825780A00C9
:10092000445F4F573D307825780A00445F4C45447A
:100930003D307825780A00445F504F5745523D308E
:100940007825780A00445F4556454E543D30782559
:10095000780A00445F50305F4C45443D307825783C
:100960000A00445F50315F4C45443D307825780A99
:1009700000445F4145533D307825780A00445F507C
:1009800057525F313D307825780A00445F50524518
:10099000533D307825780A00445F414343454C3D40
:1009A000307825780A00445F434F4D504153533D02
:1009B000307825780A0025630025630025630054FC
:1009C0005820506F7765723D25640A004F4B0A002E
:1009D0002563007478206C656E20202020207268CA
:1009E000206D697373202020207268207374616CFD
:1009F000652020207268206D6973630A00252D31FF
:100A0000306C7520252D31306C7520252D31306CE2
:100A10007520252D31306C75200A002563004D436B
:100A2000553D2530366C780020467573653A206553
:100A3000653D253032782068663D25303278206C5F
:100A4000663D25303278206C623D253032780020BA
:100A50004F534343414C3D256420002563002563EB
:100A6000002563002563004E6577207265706F7204
:100A7000743D3078255820005573696E6720726583
:100A8000706F72743D3078255820002563004E65E4
:100A900077207265706F727420696E74657276610A
:100AA0006C3D252D64207365630A00437572726581
:100AB0006E74207265706F727420696E74657276E0
:100AC000616C3D252D64207365630A002563002554
:100AD000630053797374656D2053756D6D61727920
:100AE0000A0049443D004932433A200054582050FE
:100AF0006F7765723D25640A004E65696768626FAD
:100B000072207461626C652073697A653D25640AA0
:100B10000052494D4520616464723D252D642E25A7
:100B20002D640A005265706F727420496E7465728C
:100B300076616C3D252D640A005265706F727420D9
:100B40004D61736B3D3078252D782000565F494EFE
:100B50003D252D352E32660A00565F4D43553D2505
:100B60002D352E32660A005553425F5057523D25AF
:100B7000730A00496E74722E20546F74616C3A20AF
:100B800050303D252D6C642050313D252D6C640A7C
:100B900000496E74722E205365633A202020503035
:100BA0003D252D372E33662050313D252D372E33F0
:100BB000660A004C6F67206D6F64653D0061757457
:100BC0006F0A0025730A0048554D5F5057525F4128
:100BD0004C574159533D25730A00496E7075742076
:100BE00050313D25730A0044656275673D307825B4
:100BF0002D780A00507772313D25730A0025630075
:100C000025630052483D252D342E31662000545F67
:100C100052483D252D342E31662000256300256C79
:100C20006420432000256C642050612020252D374E
:100C30002E3266206D002563005854414C5F54529B
:100C4000494D3D2564004572726F72203020566F09
:100C50006C74004572726F72203020566F6C740095
:100C60004E6F7420737570706F727465640A0045FE
:100C700072726F72203020566F6C740025352E32E0
:100C800066200025372E33662025372E3366002553
:100C9000730A005465737420312025730A0054656B
:100CA000737420322025730A005465737420332036
:100CB00025730A005465737420342025730A0025B7
:100CC000730A0025730A0025730A0025730A00259C
:100CD000730A004932433A2000256300256300501F
:100CE0003A20256C642050612020252D372E326655
:100CF000206D0A00532025642E256420636C6F63E9
:100D00006B20256C7520747820256C7520727820F6
:100D1000256C752072747820256C7520727278208D
:100D2000256C75207265786D697420256C7520615D
:100D3000636B747820256C75206E6F61636B7478BB
:100D400020256C752061636B727820256C7520748A
:100D5000696D65646F757420256C752062616461CE
:100D6000636B727820256C7520746F6F6C6F6E6783
:100D700020256C7520746F6F73686F727420256CFA
:100D8000752062616473796E636820256C752062DA
:100D9000616463726320256C7520636F6E74656E89
:100DA00074696F6E64726F7020256C752073656E48
:100DB00064696E6764726F7020256C75206C6C744A
:100DC0007820256C75206C6C727820256C750A0073
:100DD000452025642E256420636C6F636B20256C91
:100DE000752063707520256C75206C706D20256CE6
:100DF000752069727120256C7520676C65642025EB
:100E00006C7520796C656420256C7520726C656446
:100E100020256C7520747820256C75206C6973749E
:100E2000656E20256C752073656E736F7273202557
:100E30006C752073657269616C20256C750A000AF7
:100E40002A2A2A2A2A2A2A426F6F74696E67202565
:100E5000732A2A2A2A2A2A2A0A0052616E646F6D8E
:100E60002045554936342061646472657373206788
:100E7000656E6572617465640A004D41432061646A
:100E80006472657373200025783A000A0025732088
:100E900025732C206368616E6E656C20257520704B
:100EA0006F776572202575002C20636865636B2061
:100EB0007261746520257520487A000A004F6E6CB7
:100EC000696E650A00257325730A006C6F63616C97
:100ED000686F73740041544D454741313238726632
:100EE000613100020000FFFE000001454550524FF5
:100EF0004D20697320636F72727570742C20726557
:100F000077726974696E67207769746820646566B2
:100F100061756C74732E0A006E616E00696E6600F6
:100F200000407A10F35A00A0724E18090010A5D4A0
:100F3000E80000E87648170000E40B54020000CAFD
:100F40009A3B000000E1F505000080969800000043
:100F500040420F000000A0860100000010270000A2
:100F60000000E803000000006400000000000A0028
:100F7000000000000100000000002C76D888DC672B
:100F80004F0823DFC1DFAE59E1B1B796E5E3E45383
:100F9000C63AE651997696E8E6C28426EB898C9BA0
:100FA00062ED407C6FFCEFBC9C9F40F2BAA56FA540
:100FB000F490055A2AF75C936B6CF9676DC11BFCC2
:100FC000E0E40D47FEF520E6B500D0ED902E0300DD
:100FD000943577050080841E080000204E0A00002A
:100FE00000C80C333333330F986E12831141EF8DE9
:100FF0002114893BE65516CFFEE6DB18D1844B3829
:101000001BF77C1D901DA4BBE424203284725E2259
:101010008100C9F124ECA1E53D27494E46494E49DE
:1010200054594E414E000020410000C84200401C6F
:101030004620BCBE4CCA1B0E5AAEC59D74CDCCCC4E
:101040003D0AD7233C17B7D13877CC2B329595E69C
:10105000241FB14F0A0011241FBECFEFD1E4DEBF21
:10106000CDBF16E0A0E0B2E0EAEEF5EF00E00BBF86
:1010700002C007900D92AC3AB107D9F71DE2ACEA75
:10108000B6E001C01D92A635B107E1F70E94A66C3B
:101090000C94F37A0C940000E0917B17F0E0EF7170
:1010A000F070E053F84E808380917B178F5F8093C0
:1010B0007B17809190248860809390244FED54E0BA
:1010C000CA0161E10E94C53B80E090E008954F9223
:1010D0005F926F927F928F929F92AF92BF92CF92C8
:1010E000DF92EF92FF920F931F93CF93DF93CDB7D1
:1010F000DEB760970FB6F894DEBF0FBECDBF4B01D1
:101100008091B3069091B40681FD74980E9451427B
:101110003C0189EB96E00E94C13C0AC0C8010296DE
:10112000B4010E949C390097F1F4C8010E94673D08
:101130008C01009799F725C1C8010296B4010E945D
:101140009339D3018C918150F801808780E091E040
:10115000A0E0B0E081879287A387B48789EB96E00F
:10116000B8010E94303DC8010D9660E074E641EE82
:1011700059E098010E94523F84E00E947543D801D3
:1011800015969C938E93149783E00E9475432C01CF
:10119000F80197838683D301CC908085C81ADD241B
:1011A000EE24FF2486E0CC0CDD1CEE1CFF1C8A958F
:1011B000D1F7618572858385948520EC30E040E02D
:1011C00050E00E94F373DC01CB01892F9A2FAB2FE3
:1011D000BB27C80ED91EEA1EFB1EF801C186D286A7
:1011E000E386F486D3018C9180878091B306909139
:1011F000B40681FD08C08091FF0480FD04C081FF1A
:10120000B8C01D9BB6C0EDB7FEB772970FB6F89485
:10121000FEBF0FBEEDBFADB6BEB60894A11CB11C9B
:1012200080E092E092838183C3010196D5011396F9
:101230009C938E931297F401808114968C9314974B
:1012400015961C921597818116968C931697179672
:101250001C92D3018C91F50180871186D8011496D8
:101260008D919C9115979387828755864486BB27DD
:10127000AF2D9E2D8D2D97878687C701B60124E659
:1012800030E040E050E00E94F373672F782F892F01
:1012900099270E943974DC01CB01F501918B808B79
:1012A0000E94E47720911B058DB79EB742960FB63A
:1012B000F8949EBF0FBE8DBF2223A9F000D000D0AE
:1012C000EDB7FEB731968CED9CE0ADB7BEB7129688
:1012D0009C938E931197228313820E94F6770F902E
:1012E0000F900F900F908091191C86FF42C00E94B2
:1012F0001148C30104960E94D247EDB7FEB73C9750
:101300000FB6F894FEBF0FBEEDBF31966E01089484
:10131000C11CD11CADB7BEB71296DC92CE9211970C
:1013200080E190E0938382838CE392E095838483D1
:10133000D80114968D919C91159797838683169664
:101340008D919C91179791878087D3018C9182878B
:1013500013860E944B78EDB7FEB73C960FB6F89413
:10136000FEBF0FBEEDBF82E00E94ED47C6010E94A6
:10137000D2478091B3069091B40681FF0BC0749A56
:1013800009C08CE295E00E944E3C8C01009709F068
:10139000D3CEEFCF60960FB6F894DEBF0FBECDBFB1
:1013A000DF91CF911F910F91FF90EF90DF90CF9041
:1013B000BF90AF909F908F907F906F905F904F9075
:1013C0000895CF93DF93EC018091B3069091B4061A
:1013D00087FF2EC08DB79EB70C970FB6F8949EBFAF
:1013E0000FBE8DBFEDB7FEB731968FE492E0ADB77B
:1013F000BEB712969C938E9311978A818283138233
:101400008B81848315828885868317828C819D8158
:10141000918780878E819F81938782870E94E4775E
:101420008DB79EB70C960FB6F8949EBF0FBE8DBFBA
:1014300089EB96E0BE010E94FB3C8CE295E0BE0188
:101440000E94793CDF91CF91089587EE93E081155A
:10145000910511F00197F1F70895882369F06D98CF
:101460007598ED9A80916A00886080936A008091F7
:1014700068008160809368008091FF04909100056E
:1014800091FF10C06E988EB18F6B8EB9EE9A8091DD
:101490006A00806280936A00809168008160809316
:1014A00068000895769AEE9808951F920F920FB6ED
:1014B0000F9211248F939F93AF93BF9380916800F5
:1014C00080FF20C08091702490917124A09172249B
:1014D000B09173240196A11DB11D80937024909347
:1014E0007124A0937224B09373248091B3069091D9
:1014F000B40690FF07C0749882E090E090932905AD
:1015000080932805BF91AF919F918F910F900FBE4F
:101510000F901F9018951F920F920FB60F921124E3
:101520008F939F93AF93BF938091680080FF20C0FB
:101530008091742490917524A0917624B0917724A1
:101540000196A11DB11D8093742490937524A093DE
:101550007624B09377248091B3069091B40691FFDE
:1015600007C0739882E090E0909329058093280546
:10157000BF91AF919F918F910F900FBE0F901F90D1
:10158000189580937C0080917B00877F80937B00FF
:1015900080917C00806C80937C0085E080937A0051
:1015A00080917A00806880937A0080917B0087FF29
:1015B000FCCF80917B0085FFFCCF80917A00806416
:1015C00080937A0080917A0086FDFCCF109279009A
:1015D0001092780084E090E060E070E020917A0062
:1015E000206420937A0020917A0026FDFCCF209180
:1015F000780030917900620F731F019779F710928C
:101600007C0080917A008F7780937A007695679539
:101610007695679580E090E00E947971462F572F6C
:10162000682F792FCB01BA01089580E00E94C10A8A
:1016300020912405309125054091260550912705DC
:101640000E942B7221EE3AE744E95EE30E94A97002
:10165000462F572F682F792FCB01BA01089580E1CB
:1016600080935101809351019091510195FF03C0E6
:101670008F5F8F31B9F76BE4869FB0011124882703
:1016800077FD8095982F0E947B7120E030E64FE92E
:1016900054E40E94A970462F572F682F792FCB0151
:1016A000BA0120E030E04AE754E40E941171462F6D
:1016B000572F682F792FCB01BA0108958091030528
:1016C00083FF4DC080917B00886080937B0089EC14
:1016D00080937C0085E080937A0080917A00806816
:1016E00080937A0080917B0087FFFCCF80917B0004
:1016F00085FFFCCF80917A00806480937A0080918E
:101700007A0086FDFCCF80917A00806480937A0015
:1017100080917A0086FDFCCF60917800709179000D
:1017200080E090E00E94797127ED33EA40E95FE3C1
:101730000E942B7226E636E648E853E40E94A87021
:10174000DC01CB018093701790937117A0937217EF
:10175000B093731780917A008F7780937A00089501
:10176000CF92DF92EF92FF921F93CF93DF93CDB78B
:10177000DEB729970FB6F894DEBF0FBECDBF6C0160
:101780001092AC068FEF8983ACE8EA2EA7E1FA2E1F
:1017900010E03FC0183009F440C0CE010196BE01F0
:1017A0006E5F7F4F0E94384589818F3F11F08E3FD9
:1017B00019F48093AC0631C0CE010296C114D10455
:1017C00079F40E94514580938D24DE011296E5E85C
:1017D000F4E288E09D9191938150E1F711E01DC002
:1017E0000E945145F7018083DE01129620E030E02F
:1017F000C70108974D91FC01E20FF31F40832F5F53
:101800003F4F28303105B1F71F5F89E090E0E80EC7
:10181000F91E8981882309F0BDCF812F29960FB643
:10182000F894DEBF0FBECDBFDF91CF911F91FF9027
:10183000EF90DF90CF90089500D082EA91E0EDB76D
:10184000FEB7928381830E94F6770F900F900895E0
:101850002F923F924F925F926F927F928F929F92C0
:10186000AF92BF92CF92DF92EF92FF920F931F93AE
:10187000CF93DF9300D000D0CDB7DEB78C010097B7
:1018800041F489E290E06BE270E04AE250E027E048
:101890000AC08130910549F489E290E06BE270E082
:1018A0004AE250E026E00E940D44C8010E94B00BBD
:1018B0006DEA862E66E0962E800E911ED4018C93E2
:1018C0000115110599F02CE8A22E27E1B22E00E0B7
:1018D00010E03DEB632E31E0732E42EC442E41E0EC
:1018E000542E5AEC252E51E0352E10C185E894E295
:1018F0000E947446FC01BF01882777FD8095982FD0
:101900000E947B71F82EE92E05E814E2AA24BB247C
:1019100094EAC92E91E0D92ED8018D918D0100D085
:1019200000D0EDB7FEB73196ADB7BEB71296DC92D8
:10193000CE921197828313826B837C830E94F67709
:101940000894A11CB11C0F900F900F900F906B8109
:101950007C81B8E0AB16B104F9F600D000D000D01D
:101960000DB71EB70F5F1F4F89EA91E0EDB7FEB7C5
:10197000928381839701862F972FA32FBE2DBC01C1
:10198000CD0120E030E048EC52E40E941171DC010E
:10199000CB01F80182839383A483B5830E94F677F9
:1019A0002DB73EB72A5F3F4F0FB6F8943EBF0FBE2C
:1019B0002DBF80918D24882319F08EE792E002C01C
:1019C00087E892E000D000D029EB31E0ADB7BEB798
:1019D00012963C932E93119714969C938E93139783
:1019E0000E94F6770F900F900F900F900E941C0CA2
:1019F00094C0C801B3E0880F991FBA95E1F7800F32
:101A0000911F8C57984E0E947446FC01BF01882795
:101A100077FD8095982F0E947B716C0120E030E06B
:101A200088EFE82E8FEFF82EEA0CFB1C00D000D0D8
:101A3000ADB7BEB71196EDB7FEB772826182F701FE
:101A4000E20FF31F808112968C93129713961C92CB
:101A500029833A836B837C830E94F67729813A81BC
:101A60002F5F3F4F0F900F900F900F906B817C81F5
:101A700028303105D9F600D000D000D0EDB6FEB642
:101A80000894E11CF11CADB7BEB712965C924E9261
:101A90001197862F972FAC2DBD2DBC01CD0120E0D5
:101AA00030E048EC52E40E941171DC01CB01F701F7
:101AB00082839383A483B5830E94F6772DB73EB7C4
:101AC0002A5F3F4F0FB6F8943EBF0FBE2DBFD50122
:101AD0008C91882319F08EE792E002C087E892E0AB
:101AE00000D000D0EDB7FEB7328221829483838389
:101AF0000E94F6770F900F900F900F900E941C0C91
:101B00000F5F1F4F29E030E0A20EB31ED4018C916D
:101B100090E0081719070CF46CCF0F900F900F90FE
:101B20000F90DF91CF911F910F91FF90EF90DF9079
:101B3000CF90BF90AF909F908F907F906F905F906D
:101B40004F903F902F900895CF93DF9300D0CDB763
:101B5000DEB780918624898380918C248A83CE018C
:101B600001960E94AE390F900F90DF91CF910895AA
:101B7000CF93DF93EC01809185248F3FB1F5809165
:101B800086248F3F91F5809187248F3F71F5809156
:101B900088248F3F51F5809189248F3F31F58091C2
:101BA0008A248F3F11F580918B248F3FF1F480912F
:101BB0008C248F3FD1F489E290E06BE270E04AE23E
:101BC00050E027E00E940D4480E090E00E94B00BBE
:101BD000C355D94F888385E894E260E070E049E01E
:101BE00050E00E943C790E94A40DDF91CF910895AE
:101BF0001F920F920FB60F920BB60F9211242F93D4
:101C00003F934F935F936F937F938F939F93AF9384
:101C1000BF93EF93FF9380919024826080939024F0
:101C20008091FF0486FD2B9A87FD2B9A80912805D1
:101C3000909129051816190614F4749A739A8091D4
:101C4000B3069091B40685FF02C074987398809192
:101C50002A0590912B05019790932B0580932A05D7
:101C6000009709F068C08091B7069091B8069C0172
:101C70002F5F3F4F3093B8062093B70640911B204B
:101C800050911C2060911D2070911E204F5F5F4F6E
:101C90006F4F7F4F40931B2050931C2060931D205B
:101CA00070931E2020E130E030932B0520932A050D
:101CB0002091FF0420FD02C01D9B05C01092B106BB
:101CC0001092B00606C021E030E03093B1062093B8
:101CD000B006209101053091020521153105A1F0D2
:101CE0000296B9010E941274009771F4779880915E
:101CF000B3069091B40693FF07C0749884E090E017
:101D000090932905809328052115310581F0809154
:101D1000B7069091B806B9010E941274009739F481
:101D200087EC94E062E140E050E00E94C53B809186
:101D3000FF0486FD2B9880E595E060E040E050E0F0
:101D40000E94C53BFF91EF91BF91AF919F918F9101
:101D50007F916F915F914F913F912F910F900BBEAB
:101D60000F900FBE0F901F90189580917B17909148
:101D70002F20891B08950E94B50E882379F0E091E9
:101D80002F20F0E0EF71F070E053F84E808190E08A
:101D900020912F202F5F20932F2008958FEF9FEF0A
:101DA0000895CF93DF93EC011092B6061092B5061A
:101DB00088819981009731F022E08B3B920709F0EE
:101DC000B7C009C00E94B50E882341F48BEB92E0A6
:101DD00099838883B1C0613109F0AEC0F8947894DA
:101DE0000E94BB0E90E09093C1068093C0068D3098
:101DF00009F47CC08F3F31F38231910569F18F374F
:101E0000910521F08830910509F053C08091C206F8
:101E10009091C306181619060CF060C06091502D01
:101E20007091512D88E090E00E94B8776091502D1C
:101E30007091512D80E290E00E94B8776091502D12
:101E40007091512D88E090E00E94B8778091C20691
:101E50009091C30601973EC06091502D7091512D15
:101E60008DE090E00E94B8771092C5061092C406EB
:101E700014C0805D9F4DFC0180816091502D709158
:101E8000512D90E00E94B8778091C4069091C506CC
:101E900001969093C5068093C4068091C4069091E4
:101EA000C5062091C2063091C306821793070CF332
:101EB00015C06091502D7091512D0E94B87780917E
:101EC000C2069091C3062091C006FC01E05DFF4D63
:101ED000208301969093C3068093C2068091C20628
:101EE0009091C3068F33910509F06CCF10922F208B
:101EF00010927B178091C2069091C306FC01E05DB1
:101F0000FF4D10829093B6068093B5061092C306DB
:101F10001092C20680918E2490918F24009709F42C
:101F200051CF6091BE0640E050E00E94C53B4ACFD1
:101F30001982188283E001C081E0DF91CF9108957A
:101F400078948091B0069091B106009731F080911D
:101F5000FF049091000590FF03C083B7817F03C009
:101F600083B7817F866083BFF89483B7816083BF26
:101F70007894889583B78E7F83BF78940895CF93A4
:101F8000DF93EC0188819981009721F029E08B3F54
:101F9000920799F40E94304D0E94A00F8091640E28
:101FA0009091650E65E840E050E00E94C53B8BEFE4
:101FB00099E09983888381E003C01982188283E0C5
:101FC000DF91CF910895CF93DF930E94304D80EB46
:101FD0000E94F2468823B1F40E9458478091191C50
:101FE00090911A1C816090931A1C8093191C00D048
:101FF0008EEC91E0EDB7FEB7928381830E94F67775
:102000000F900F90CEB1D0E0C470D070729A0E9441
:10201000304D8EE40E94F2468823B1F40E94584766
:102020008091191C90911A1C826090931A1C8093C5
:10203000191C00D087ED91E0EDB7FEB79283818344
:102040000E94F6770F900F90209709F472980E94E3
:10205000304D8EEE0E94F2468823B1F40E9458471C
:102060008091191C90911A1C846090931A1C809383
:10207000191C00D080EE91E0EDB7FEB7928381830A
:102080000E94F6770F900F9086EA0E94F24688230E
:10209000B1F40E9458478091191C90911A1C8860D5
:1020A00090931A1C8093191C00D088EE91E0EDB734
:1020B000FEB7928381830E94F6770F900F900E9463
:1020C000304D8CE30E94F2468823B1F40E945847B9
:1020D0008091191C90911A1C806190931A1C809316
:1020E000191C00D081EF91E0EDB7FEB79283818398
:1020F0000E94F6770F900F900E94304D82ED0E9463
:10210000F2468823B1F40E9458478091191C90919F
:102110001A1C806290931A1C8093191C00D08AEFBD
:1021200091E0EDB7FEB7928381830E94F6770F901E
:102130000F90C7E0D0E00E94304D8CE70E94F2463D
:102140008823B9F40E9458478091191C90911A1C59
:10215000806490931A1C8093191C00D084E092E054
:10216000EDB7FEB7928381830E94F6770F900F90B0
:1021700002C0219701F70E9458470E941C0CDF9172
:10218000CF910895CF93DF9300D0CDB7DEB74A83C8
:1021900069830E942E476981862F0E9460474A8189
:1021A000842F0E9460470E9458470F900F90DF9144
:1021B000CF910895AF92BF92DF92EF92FF920F936B
:1021C0001F93CF93DF9300D00F92CDB7DEB7082FC8
:1021D000D22E4A835B8369830E942E476981862FB2
:1021E0000E946047802F81600E9455474A81042FDA
:1021F0005B81152FEE24FF24AD2CBB240894A1088D
:10220000B1080FC0EA14FB0419F40E947B4702C016
:102210000E947147F80180830894E11CF11C0F5F54
:102220001F4FED1478F30E9458470F900F900F90B6
:10223000DF91CF911F910F91FF90EF90DF90BF90B2
:10224000AF900895AF92BF92DF92EF92FF920F93FB
:102250001F93CF93DF93CDB7DEB760970FB6F89497
:10226000DEBF0FBECDBF8E010F5F1F4F80E1D801D3
:102270001D928A95E9F780EB68E9A80128E00E94A1
:10228000DA1000D088E892E0EDB7FEB79283818340
:102290000E94E47778010F900F90DD24AFE8AA2E1A
:1022A000A2E0BA2ED8018D918D0100D000D0EDB7FB
:1022B000FEB73196ADB7BEB71296BC92AE921197EB
:1022C000828313820E94E477D3940F900F900F9033
:1022D0000F90B7E0DB1631F700D000D0EDB7FEB7B6
:1022E000319685E992E0ADB7BEB712969C938E9376
:1022F00011978885828313820E94E477AE014F5F35
:102300005F4F80E1FA0111928A95E9F70F900F90E3
:102310000F900F9080EB60E828E00E94DA1000D068
:102320008BE992E0ADB7BEB712969C938E9311974E
:102330000E94E4770F900F907FE0D72E0FE812E015
:10234000F70181917F0100D000D0EDB7FEB7319643
:10235000ADB7BEB712961C930E931197828313826A
:102360000E94E477DA940F900F900F900F9041F74E
:1023700000D000D0EDB7FEB7319685E992E0ADB759
:10238000BEB712969C938E93119788858283138291
:102390000E94E4770F900F900F900F9060960FB609
:1023A000F894DEBF0FBECDBFDF91CF911F910F918B
:1023B000FF90EF90DF90BF90AF900895CF93DF93A1
:1023C00000D0CDB7DEB71A8219828EEE6AEAAE016E
:1023D0004F5F5F4F22E00E94DA10398120E08A814E
:1023E00090E0822B932B9093F1178093F0178EEE51
:1023F0006CEAAE014F5F5F4F22E00E94DA10398134
:1024000020E08A8190E0822B932B9093F3178093A6
:10241000F2178EEE6EEAAE014F5F5F4F22E00E9430
:10242000DA10398120E08A8190E0822B932B9093FF
:10243000F5178093F4178EEE60EBAE014F5F5F4FA0
:1024400022E00E94DA10398120E08A8190E0822B1C
:10245000932B90930318809302188EEE62EBAE01DB
:102460004F5F5F4F22E00E94DA10398120E08A81BD
:1024700090E0822B932B90930518809304188EEE96
:1024800064EBAE014F5F5F4F22E00E94DA103981AA
:1024900020E08A8190E0822B932B90930718809301
:1024A00006188EEE66EBAE014F5F5F4F22E00E9492
:1024B000DA10398120E08A8190E0822B932B90936F
:1024C000F7178093F6178EEE68EBAE014F5F5F4F04
:1024D00022E00E94DA10398120E08A8190E0822B8C
:1024E000932B9093F9178093F8178EEE6AEBAE0159
:1024F0004F5F5F4F22E00E94DA10398120E08A812D
:1025000090E0822B932B9093FD178093FC178EEE17
:102510006CEBAE014F5F5F4F22E00E94DA10398111
:1025200020E08A8190E0822B932B9093FF17809379
:10253000FE178EEE6EEBAE014F5F5F4F22E00E9402
:10254000DA10398120E08A8190E0822B932B9093DE
:102550000118809300180F900F90DF91CF9108958C
:102560002F923F924F925F926F927F928F929F92A3
:10257000AF92BF92CF92DF92EF92FF920F931F9391
:10258000CF93DF93CDB7DEB76C970FB6F894DEBF6D
:102590000FBECDBF882E4A8F2B8FFE01319683E070
:1025A000DF011D928A95E9F780911418882339F488
:1025B0006C8F0E94DE1181E0809314186C8D66236D
:1025C00009F478C08EEE64EF4EE20E94C21069E01A
:1025D0007AE180E090E00E94DF468EEE66EFAE0189
:1025E0004F5F5F4F22E00E94DA10898190E0A0E007
:1025F000B0E0BA2FA92F982F88274A8150E060E0D9
:1026000070E0842B952BA62BB72B209106183091C8
:102610000718A90160E070E0841B950BA60BB70BAF
:10262000209104183091051840E050E0BC01CD0124
:102630000E94F3736B017C01AFE0F594E794D794AB
:10264000C794AA95D1F76091FE177091FF1788275C
:1026500077FD8095982FBBE0660F771F881F991F25
:10266000BA95D1F72091001830910118442737FD11
:102670004095542F2C0D3D1D4E1D5F1D0E945B7417
:102680002C0D3D1D3093FB172093FA17285F3F4F09
:1026900014E0359527951A95E1F76901EE24D7FCEA
:1026A000E094FE2CC0920818D0920918E0920A1803
:1026B000F0920B18082D0295000F000F007C0C5CA7
:1026C000282D30E0398F288F63E070E0082C02C09D
:1026D000660F771F0A94E2F7882777FD8095982F79
:1026E00025E335E040E050E00E94F373DC01CB01CC
:1026F0000296A11DB11D888B998BAA8BBB8B20E5FF
:1027000033EC40E050E004C0559547953795279548
:102710008A94D2F72C8B3D8B4E8B5F8B10E01C86FE
:102720001D861E861F86E8E02E2E312C488D598D81
:10273000241A350A73C18EEE64EF402F0E94C21036
:10274000688979898A899B890E94DF468EEE66EFC7
:10275000AE014F5F5F4F23E00E94DA108091FA17BD
:102760009091FB17805A9F409C01442737FD40956C
:10277000542F2C833D834E835F83CA01B9010E948D
:10278000F3732B013C016091F4177091F5178827C2
:1027900077FD8095982F0E94F3736B017C01BDE05B
:1027A000F594E794D794C794BA95D1F76091F6174A
:1027B0007091F717882777FD8095982FA3019201D4
:1027C000ECE05595479537952795EA95D1F70E9406
:1027D000F373DC01CB01CD01BB2797FDB095AB2F87
:1027E000C80ED91EEA1EFB1E82E090E0A0E0B0E019
:1027F000C80ED91EEA1EFB1EE2E0F594E794D794BA
:10280000C794EA95D1F720E030E840E050E0C20EEE
:10281000D31EE41EF51E209102183091031840E0EB
:1028200050E0C701B6010E94F373DC01CB01FFE069
:10283000B695A79597958795FA95D1F78887998743
:10284000AA87BB8789809924AA24BB245401992490
:1028500088248A8190E0A0E0B0E0BA2FA92F982FB9
:102860008827882A992AAA2ABB2A8B8190E0A0E08F
:10287000B0E0882A992AAA2ABB2A022C04C0B5945F
:10288000A794979487940A94D2F7C090F017D090A9
:10289000F117EE24D7FCE094FE2CE2E0CC0CDD1C1A
:1028A000EE1CFF1CEA95D1F76091F8177091F917AB
:1028B000882777FD8095982FA30192010E94F373DA
:1028C0002B013C01F7E17594679457944794FA956E
:1028D000D1F76091F2177091F317882777FD8095F3
:1028E000982F2C813D814E815F810E94F373DC0122
:1028F000CB01EBE0B595A79597958795EA95D1F72C
:10290000480E591E6A1E7B1EC40CD51CE61CF71C03
:10291000088C04C0CC0CDD1CEE1CFF1C0A94D2F702
:1029200022E030E040E050E0C20ED31EE41EF51E6F
:10293000F2E0F594E794D794C794FA95D1F78C1800
:102940009D08AE08BF08C501B4012C893D894E8998
:102950005F890E94F37397FD0DC0660F771F881F74
:10296000991F288539854A855B850E9439744901FC
:102970005A010CC0288539854A855B850E943974C7
:1029800049015A01880C991CAA1CBB1C5527B7FC8D
:102990005A954B2D3A2D292DCA01B9010E94F37386
:1029A0002EED3BE040E050E00E94F3736C01FF2409
:1029B000D7FCF094EF2CC501B40123E433EE4FEFC4
:1029C0005FEF0E94F373DC01CB01CD01BB2797FDC4
:1029D000B095AB2FC80ED91EEA1EFB1E8FEC9EE0F1
:1029E000A0E0B0E0C80ED91EEA1EFB1EE4E0F5949C
:1029F000E794D794C794EA95D1F7C80CD91CEA1C80
:102A0000FB1C2C853D854E855F852C0D3D1D4E1D87
:102A10005F1D2C873D874E875F871F5F3A8D131799
:102A200009F089CE112391F0212F30E040E050E0F1
:102A30006C857D858E859F850E94397420930C1846
:102A400030930D1840930E1850930F184B8D44235C
:102A5000E9F160910C1870910D1880910E18909109
:102A60000F18611571058105910581F10E947B7137
:102A700020E836EE45EC57E40E94117121E03EED6E
:102A800042E45EE30E948E72B62FA72F382F292FC3
:102A900060E070E080E89FE3FD01A9010F2F1E2F89
:102AA000252F342FA90198010E94A8702BE43AE346
:102AB0004DEB57E30E941171DC01CB01809310189C
:102AC00090931118A0931218B09313186C960FB628
:102AD000F894DEBF0FBECDBFDF91CF911F910F9154
:102AE000FF90EF90DF90CF90BF90AF909F908F902E
:102AF0007F906F905F904F903F902F900895CF936D
:102B0000DF9300D000D000D0CDB7DEB7FE01319604
:102B100086E0DF011D928A95E9F780917A17882374
:102B200099F486EA61E340E00E94C21086EA6CE212
:102B30004AE00E94C21081E080937A176CE77EE33E
:102B400080E090E00E94DF4686EA6DE248E00E9465
:102B5000C2106CE77EE380E090E00E94DF4686EAE8
:102B600062E3AE014F5F5F4F26E00E94DA1086EA13
:102B70006DE247E00E94C2109A8180E0698170E0B6
:102B8000682B792B70937517609374179C8180E084
:102B90004B8150E0482B592B509377174093761771
:102BA0003E8120E08D8190E0822B932B90937917CA
:102BB000809378172DB73EB7285030400FB6F89461
:102BC0003EBF0FBE2DBFEDB7FEB731962FE932E005
:102BD000ADB7BEB712963C932E9311977383628361
:102BE00055834483978386830E94E4772DB73EB74D
:102BF000285F3F4F0FB6F8943EBF0FBE2DBF2696FD
:102C00000FB6F894DEBF0FBECDBFDF91CF91089510
:102C10000F931F93CF93DF9300D000D000D0CDB798
:102C2000DEB78E010F5F1F4F86E0D8011D928A9597
:102C3000E9F78CE362E041E00E94C2108CE360E0BF
:102C400048E50E94C21062E174E380E090E00E94D7
:102C5000DF468CE363E0A80126E00E94DA108CE3F3
:102C600062E043E00E94C210998180E06A8170E0D6
:102C7000682B792B70935B1760935A179B8180E0C8
:102C80004C8150E0482B592B50935D1740935C17B3
:102C90003D8120E08E8190E0822B932B90935F17F3
:102CA00080935E17EDB7FEB738970FB6F894FEBF66
:102CB0000FBEEDBF31962DEA32E0ADB7BEB712962A
:102CC0003C932E9311977383628355834483978338
:102CD00086830E94E477EDB7FEB738960FB6F89476
:102CE000FEBF0FBEEDBF26960FB6F894DEBF0FBE37
:102CF000CDBFDF91CF911F910F910895CF93DF93B7
:102D0000EC0188819981009731F029E0843E920797
:102D100009F071C00BC08AED96E060E870E00E9497
:102D2000593E84EE99E09983888369C08AED96E0E4
:102D30000E94843E009709F462C08091B30690918E
:102D4000B40694FF3FC08091191C82FF3BC083E012
:102D500061E048E021E00E94B0128DB79EB70A976B
:102D60000FB6F8949EBF0FBE8DBFEDB7FEB731967C
:102D70008FED9CE0ADB7BEB712969C938E931197E2
:102D800080910C1890910D18A0910E18B0910F1809
:102D900082839383A483B583809110189091111836
:102DA000A0911218B091131886839783A087B187DA
:102DB0000E94F6778DB79EB70A960FB6F8949EBF1D
:102DC0000FBE8DBF8091B3069091B40695FF06C0EB
:102DD0008091191C83FF02C00E947F158091B30669
:102DE0009091B40696FF97CF8091191C84FF93CFE2
:102DF0000E94081690CF1982188283E001C081E0FA
:102E0000DF91CF910895FF920F931F93CF93DF939C
:102E1000729A8091FF0483FD06C0C0E5D0E00E9455
:102E2000250A2197E1F78EE40E94F246882309F0F3
:102E30008BC0C0E5D0E00E94250A2197E1F78FE41E
:102E40000E94F2460E947147C82F8295869586950A
:102E500083708130A9F44091232050912420609107
:102E60002520709126204F5F5F4F6F4F7F4F40931B
:102E7000232050932420609325207093262016C091
:102E80008230A0F040912720509128206091292085
:102E900070912A204F5F5F4F6F4F7F4F40932720E5
:102EA000509328206093292070932A200E94714714
:102EB0001C2F1F7300E0080F111D0E947147F82E90
:102EC0000E947B47DF2D90E0C92FC80FD11DD695FA
:102ED000C795D695C7950E9458478091FF0483FFF8
:102EE0007298B80180E090E00E94797120E134E0AE
:102EF00048EC5BE30E942B72DC01CB018093151838
:102F000090931618A0931718B0931818BE0180E07C
:102F100090E00E94797124EA3CEF44E25CE30E9475
:102F20002B7220E030E040E252E40E94A870DC0105
:102F3000CB018093912490939224A0939324B093F7
:102F4000942480E090E015C080911F209091202073
:102F5000A0912120B09122200196A11DB11D809346
:102F60001F2090932020A0932120B093222081E065
:102F700090E0DF91CF911F910F91FF90089572988B
:102F8000729A8EE40E94F24680EA0E94604780E0D6
:102F90000E94604780E00E9460478FE40E94F246F2
:102FA0000E94714782958695869583708130A9F439
:102FB000409123205091242060912520709126205B
:102FC0004F5F5F4F6F4F7F4F4093232050932420DC
:102FD000609325207093262016C08230A0F0409187
:102FE0002720509128206091292070912A204F5F3E
:102FF0005F4F6F4F7F4F409327205093282060935F
:10300000292070932A2000D000D0EDB7FEB731966A
:103010002BEB32E0ADB7BEB712963C932E931197CF
:10302000828313820E94E4770F900F900F900F908D
:103030008EE40E94F24680E80E94604780E00E9491
:10304000604780E00E9460470E94584780E090E01F
:10305000089500D08EE092E0ADB7BEB712969C9373
:103060008E9311970E94F67720911B050F900F9079
:103070002223A9F000D000D0EDB7FEB731968BE146
:1030800092E0ADB7BEB712969C938E9311972283B0
:1030900013820E94F6770F900F900F900F90089573
:1030A00000D08EE192E0EDB7FEB7928381830E945B
:1030B000F67783E492E0EDB7FEB7928381830E94B6
:1030C000F6778BE692E0EDB7FEB7928381830E949C
:1030D000F67782E992E0EDB7FEB7928381830E9492
:1030E000F6778CEB92E0EDB7FEB7928381830E9476
:1030F000F67787EF92E0EDB7FEB7928381830E9467
:10310000F67789E293E0EDB7FEB7928381830E9460
:10311000F6778FE493E0EDB7FEB7928381830E9448
:10312000F6778FE793E0EDB7FEB7928381830E9435
:10313000F67788EB93E0EDB7FEB7928381830E9428
:10314000F67784EE93E0EDB7FEB7928381830E9419
:10315000F6778DE094E0EDB7FEB7928381830E940D
:10316000F67788E394E0EDB7FEB7928381830E94FF
:10317000F67787E694E0EDB7FEB7928381830E94ED
:10318000F67789E994E0EDB7FEB7928381830E94D8
:10319000F6778AEC94E0EDB7FEB7928381830E94C4
:1031A000F6778EEF94E0EDB7FEB7928381830E94AD
:1031B000F6778EE295E0EDB7FEB7928381830E94A9
:1031C000F6778AE595E0EDB7FEB7928381830E949A
:1031D000F67789E895E0EDB7FEB7928381830E9488
:1031E000F67782EC95E0EDB7FEB7928381830E947B
:1031F000F6778BEE95E0EDB7FEB7928381830E9460
:10320000F6778AE296E0EDB7FEB7928381830E945B
:10321000F67789E596E0EDB7FEB7928381830E9449
:10322000F67788E896E0EDB7FEB7928381830E9437
:10323000F6778FEA96E0EDB7FEB7928381830E941E
:10324000F67785EE96E0EDB7FEB7928381830E9414
:10325000F6778EE097E0EDB7FEB7928381830E9408
:10326000F6770F900F9008958BEC92E00E941D78F6
:1032700008954F925F926F927F928F929F92AF923A
:10328000BF92CF92DF92EF92FF920F931F93CF9353
:10329000DF9300D000D0CDB7DEB760911B207091D6
:1032A0001C2080911D2090911E2080901B209090CA
:1032B0001C20A0901D20B0901E2040901B205090FC
:1032C0001C2060901D2070901E2020911B203091AA
:1032D0001C2040911D2050911E2029833A834B834E
:1032E0005C834DB75EB74A5050400FB6F8945EBF4E
:1032F0000FBE4DBF0DB71EB70F5F1F4F29E337E05D
:10330000EDB7FEB732832183A0E8CA2EA1E5DA2EFD
:10331000A1E0EA2EF12CA70196010E943974F80170
:1033200033832283C501B401A70196010E94397439
:10333000B0E1CB2EBEE0DB2EE12CF12CA7019601F3
:103340000E943974332727FD3095F8013583248393
:10335000C301B201A70196010E9439742CE3C22E69
:10336000D12CE12CF12CA70196010E94397433274E
:1033700027FD3095F8013783268369817A818B8117
:103380009C81A70196010E943974772767FD70958B
:10339000F801718760870E94F6772DB73EB7265FE8
:1033A0003F4F0FB6F8943EBF0FBE2DBF0F900F904A
:1033B0000F900F90DF91CF911F910F91FF90EF90A1
:1033C000DF90CF90BF90AF909F908F907F906F9045
:1033D0005F904F900895E6E5FDE28081918122E4BF
:1033E00082349207B9F000D000D089E597E0ADB7FC
:1033F000BEB712969C938E931197E655FD42149694
:10340000FC93EE9313970E94F6770F900F900F9016
:103410000F9008953A96B1E4E53FFB07F0F2089566
:10342000EF92FF920F931F93CF93DF930E94150BA0
:10343000DC01CB0100D000D000D027E737E0EDB7AA
:10344000FEB73283218383839483A583B6830E944E
:10345000F6778DB79EB706960FB6F8949EBF0FBE4F
:103460008DBF81E00E94C10A209120053091210585
:1034700040912205509123050E942B728B01D82F79
:10348000C92F82E00E94C10AAB01BC01EDB7FEB7B3
:103490003A970FB6F894FEBF0FBEEDBFEDB6FEB67D
:1034A0000894E11CF11C2EE737E0328321839E0152
:1034B000802F912FA32FB22FF70182839383A483B0
:1034C000B583CB01BA0120911C0530911D054091B7
:1034D0001E0550911F050E942B72DC01CB01F701E4
:1034E00086839783A087B1870E94F6778DB79EB7B2
:1034F0000A960FB6F8949EBF0FBE8DBF0E941C0C9B
:10350000DF91CF911F910F91FF90EF900895EF926F
:10351000FF920F931F93CF93DF93882389F085E861
:1035200094E26FEF70E049E050E00E946E7785E82A
:1035300094E260E070E049E050E00E943C7922C0F3
:1035400005E814E2C0E0D0E03AE8E32E37E0F32EDD
:10355000D8018D918D0100D000D0EDB7FEB7319626
:10356000ADB7BEB71296FC92EE921197828313828A
:103570000E94F67721960F900F900F900F90C83011
:10358000D10531F70E941C0CDF91CF911F910F9153
:10359000FF90EF900895CF92DF92EF92FF926091AB
:1035A000190570911A0580E090E00E9460776CEE3A
:1035B00072E00E947577009709F085C083E19AE078
:1035C000909304058093030583E095E06EE070E03E
:1035D00042E050E00E943C798CE390E09093020539
:1035E0008093010581E095E06CE070E042E050E0FE
:1035F0000E943C798AE090E0909300058093FF045C
:103600008FEF94E06AE070E042E050E00E943C7985
:103610001092B4061092B30683EB96E06CE170E072
:1036200042E050E00E943C790F2EF2E2CF2EFFEFF5
:10363000DF2EFCECEF2EFBE3FF2EF02DC0922005D9
:10364000D0922105E0922205F092230580E295E0D8
:1036500064E170E044E050E00E943C79C0921C05B7
:10366000D0921D05E0921E05F0921F058CE195E0B9
:1036700060E170E044E050E00E943C798DEE97E418
:10368000AAE8BCE38093240590932505A093260522
:10369000B093270584E295E068E170E044E050E0F3
:1036A0000E943C791092AF068FEA96E069E070E0E4
:1036B00041E050E00E943C7981E00E94871A80E05E
:1036C00090E00E94B80DFF90EF90DF90CF900895AA
:1036D000882309F401C18091030580FF0BC000D04D
:1036E0008FE897E0EDB7FEB7928381830E94F6776B
:1036F0000F900F908091030581FF0BC000D085E9EA
:1037000097E0EDB7FEB7928381830E94F6770F9022
:103710000F908091030582FF0BC000D08AE997E0EB
:10372000EDB7FEB7928381830E94F6770F900F90DA
:103730008091030583FF0BC000D080EA97E0EDB7CE
:10374000FEB7928381830E94F6770F900F9080914D
:10375000030584FF0BC000D089EA97E0EDB7FEB700
:10376000928381830E94F6770F900F9080910305DA
:1037700085FF0BC000D082EB97E0EDB7FEB79283D8
:1037800081830E94F6770F900F908091030586FF4A
:103790000BC000D088EB97E0EDB7FEB79283818332
:1037A0000E94F6770F900F908091030587FF0BC062
:1037B00000D080EC97E0EDB7FEB7928381830E9442
:1037C000F6770F900F90809103059091040590FF7C
:1037D0000BC000D086EC97E0EDB7FEB792838183F3
:1037E0000E94F6770F900F90809103059091040549
:1037F00091FF0BC000D08EEC97E0EDB7FEB792833F
:1038000081830E94F6770F900F908091030590912D
:10381000040592FF0BC000D088ED97E0EDB7FEB72E
:10382000928381830E94F6770F900F908091030519
:103830009091040593FF0BC000D08EED97E0EDB79B
:10384000FEB7928381830E94F6770F900F9080914C
:1038500003059091040594FF0BC000D086EE97E01D
:10386000EDB7FEB7928381830E94F6770F900F9099
:10387000809103059091040595FF0BC000D08CEE5C
:1038800097E0EDB7FEB7928381830E94F6770F90A1
:103890000F90809103059091040596FF0BC000D016
:1038A00082EF97E0EDB7FEB7928381830E94F677AF
:1038B0000F900F90809103059091040597FF4AC1E6
:1038C00000D087EF97E0EDB7FEB7928381830E9427
:1038D000F6770F900F903EC100D000D08DEF97E0AB
:1038E000EDB7FEB79283818381E090E09483838378
:1038F0000E94F6770F900F900F900F900E941C0C73
:1039000000D000D089E098E0EDB7FEB792838183C4
:1039100082E090E0948383830E94F6770F900F906B
:103920000F900F900E941C0C00D000D084E198E012
:10393000EDB7FEB79283818384E090E09483838324
:103940000E94F6770F900F900F900F900E941C0C22
:1039500000D000D080E298E0EDB7FEB7928381837B
:1039600088E090E0948383830E94F6770F900F9015
:103970000F900F900E941C0C00D000D08EE298E0B7
:10398000EDB7FEB79283818380E190E094838383D7
:103990000E94F6770F900F900F900F900E941C0CD2
:1039A00000D000D08CE398E0EDB7FEB7928381831E
:1039B00080E290E0948383830E94F6770F900F90CB
:1039C0000F900F900E941C0C00D000D088E498E06B
:1039D000EDB7FEB79283818380E490E09483838384
:1039E0000E94F6770F900F900F900F900E941C0C82
:1039F00000D000D086E598E0EDB7FEB792838183D2
:103A000080E890E0948383830E94F6770F900F9074
:103A10000F900F900E941C0C00D000D082E698E01E
:103A2000EDB7FEB79283818380E091E09483838336
:103A30000E94F6770F900F900F900F900E941C0C31
:103A400000D000D080E798E0EDB7FEB79283818385
:103A500080E092E0948383830E94F6770F900F902A
:103A60000F900F900E941C0C00D000D08FE798E0C0
:103A7000EDB7FEB79283818380E094E094838383E3
:103A80000E94F6770F900F900F900F900E941C0CE1
:103A900000D000D08BE898E0EDB7FEB79283818329
:103AA00080E098E0948383830E94F6770F900F90D4
:103AB0000F900F900E941C0C00D000D089E998E074
:103AC000EDB7FEB79283818380E090E19483838396
:103AD0000E94F6770F900F900F900F900E941C0C91
:103AE00000D000D085EA98E0EDB7FEB792838183DD
:103AF00080E090E2948383830E94F6770F900F908A
:103B00000F900F900E941C0C00D000D081EB98E029
:103B1000EDB7FEB79283818380E090E49483838342
:103B20000E94F6770F900F900F900F900E941C0C40
:103B300000D000D08CEB98E0EDB7FEB79283818384
:103B400080E090E8948383830E94F6770F900F9033
:103B50000F900F900E941C0C08952F923F924F924D
:103B60005F926F927F928F929F92AF92BF92CF920D
:103B7000DF92EF92FF920F931F93CF93DF9300D0CA
:103B8000CDB7DEB79A838983DC018D919C91119723
:103B9000009711F00C9441306091190570911A054D
:103BA00080E390E20E94607780E390E260E470E05E
:103BB0000E947E77009759F46091502D7091512D9D
:103BC0008AE090E00E94B87781E00C944630813022
:103BD000910549F420903020332444245524662450
:103BE00077244301BEC18230910599F43091302091
:103BF00020913120932F80E0820F911D1C01892F8D
:103C0000880F880B482E582E682E782E882E982ED6
:103C1000A8C18330910509F09CC02091302080908C
:103C20003120B090322030E040E050E060E070E0C1
:103C300080E090E000E10E94E96B922EA32E142F09
:103C4000F52EE62EC72E282ED92E282D30E040E066
:103C500050E060E070E080E090E008E00E94E96BF6
:103C6000290DB1E0291508F0B0E03A0DE1E03A1570
:103C700008F0E0E0B30FF1E0B31708F0F0E0EF2B4D
:103C8000410F31E0411708F030E0E40FF1E0E417B4
:103C900008F0F0E03F2B5F0D41E05F1508F040E0D9
:103CA000A32FA50F31E0A51708F030E0432B6E0DD0
:103CB00031E06E1508F030E0F42FF60F41E0F61712
:103CC00008F040E0342B7C0D41E07C1508F040E02A
:103CD000532F570F31E0571708F030E0432B820D78
:103CE00031E0821508F030E0480F61E0481708F035
:103CF00060E0362BD90ED30EB20E81E0B21608F07A
:103D000080E0182F1B0F71E01B1708F070E07E0F8A
:103D100061E07E1708F060E06A0F31E06A1708F092
:103D200030E03F0F21E03F1708F020E0250F91E041
:103D3000251708F090E0940F81E0941708F080E0D8
:103D40002B2C312E472E562E632E722E892E982E16
:103D5000FDC08430910509F0FBC020913020809097
:103D60003120A0903220B090332030E040E050E08D
:103D700060E070E080E090E008E10E94E96B722E64
:103D8000932E142FF52EE62EC72E282ED92E282D51
:103D900030E040E050E060E070E080E090E000E182
:103DA0000E94E96B270DF1E0271508F0F0E0390DCE
:103DB000E1E0391508F0E0E0F30FA1E0F31708F0B7
:103DC000A0E0EA2B410F31E0411708F030E0E40FAA
:103DD000A1E0E41708F0A0E03A2B5F0D41E05F1589
:103DE00008F040E0B32FB50F31E0B51708F030E030
:103DF000432B6E0D31E06E1508F030E0A42FA60FB6
:103E000041E0A61708F040E0342B7C0D41E07C1522
:103E100008F040E0532F570F31E0571708F030E01B
:103E2000432B820D31E0821508F030E0480F61E04D
:103E3000481708F060E0362BD90ED30E222E2B0C3B
:103E400081E0221608F080E0B82EBF0E81E0BF1698
:103E500008F080E0982E9E0E81E09E1608F080E02B
:103E6000C82ECB0E11E0CB1608F010E01A0F81E03F
:103E70001A1708F080E0F82EF50E81E0F51608F02C
:103E800080E0E82EE40E81E0E41608F080E0D80E31
:103E90002A2D30E040E050E060E070E080E090E00B
:103EA00008E00E94E96B220DE1E0221508F0E0E055
:103EB0003B0DF1E03B1508F0F0E0E30FA1E0E31764
:103EC00008F0A0E0FA2B490D31E0491508F030E088
:103ED000F40FA1E0F41708F0A0E03A2B5C0D41E0EC
:103EE0005C1508F040E0A32FA50F31E0A51708F0FE
:103EF00030E0432B610F31E0611708F030E0542FC0
:103F0000560F41E0561708F040E0342B7F0D41E09A
:103F10007F1508F040E0632F670F31E0671708F066
:103F200030E0432B8E0D31E08E1508F030E0480F65
:103F300071E0481708F070E0372BD90E222E3E2E84
:103F40004F2E5A2E652E762E842E932E9D0C09C050
:103F5000FAE02F2E33244424552466247724882421
:103F600099240E941C0CBDE62B1691F4E5E73E1641
:103F700079F4F8E64F1661F4552051F4662041F4C7
:103F8000772031F4882021F4992011F40C94F42E38
:103F90009101A201B301C4011DE6A12E05E7B02ED7
:103FA000E8E6CE2EDD24EE24FF2400E010E00E949F
:103FB000636C823008F072C283E3281689F491E7BB
:103FC000391671F4442061F4552051F4662041F40F
:103FD000772031F4882021F4992011F40C94E52EF7
:103FE0009101A201B301C401A3E3AA2EB1E7BB2E44
:103FF000CC24DD24EE24FF2400E010E00E94636C5A
:10400000823008F022C1A5E62A1681F4B4E63B16F8
:1040100069F4442059F4552049F4662039F4772096
:1040200029F4882019F4992009F4B5C69101A20158
:10403000B301C401E5E6AE2EF4E6BF2ECC24DD24A8
:10404000EE24FF2400E010E00E94636C823008F050
:104050007BC0E5E72E1679F4332069F4442059F447
:10406000552049F4662039F4772029F4882019F482
:10407000992009F4DFC79101A201B301C40105E74A
:10408000A02EBB24CC24DD24EE24FF2400E010E08D
:104090000E94636C823010F5F8E62F1611F00C9434
:1040A0003F30332011F00C943F30442011F00C9439
:1040B0003F30552011F00C943F30662011F00C94E5
:1040C0003F30772011F00C943F30882011F00C9491
:1040D0003F30992011F00C943F3087C786E72816AF
:1040E00079F4332069F4442059F4552049F46620CA
:1040F00039F4772029F4882019F4992009F4B2C7FB
:1041000094E6291611F00C943F30A1E63A1611F00E
:104110000C943F30442011F00C943F30552011F0A6
:104120000C943F30662011F00C943F30772011F052
:104130000C943F30882011F00C943F30992011F0FE
:104140000C943F300C94E52EB5E62B1689F4EEE680
:104150003E1671F4442061F4552051F4662041F478
:10416000772031F4882021F4992011F40C94102B3D
:104170009101A201B301C401B5E6AB2E1EE6B12E3A
:10418000CC24DD24EE24FF2400E010E00E94636CC8
:10419000823018F5F4E62F1611F00C943F3089E6C2
:1041A000381611F00C943F30442011F00C943F303D
:1041B000552011F00C943F30662011F00C943F30E4
:1041C000772011F00C943F30882011F00C943F3090
:1041D000992011F00C943F300CC797E7291689F409
:1041E000AFE63A1671F4442061F4552051F466208C
:1041F00041F4772031F4882021F4992011F40C94B3
:10420000BA2AB1E32B1611F00C943F30E0E73E16CA
:1042100011F00C943F30442011F00C943F305520A5
:1042200011F00C943F30662011F00C943F30772051
:1042300011F00C943F30882011F00C943F309920FD
:1042400011F00C943F300C949A2BF3E62F1691F456
:1042500084E6381679F491E6491661F4552051F454
:10426000662041F4772031F4882021F4992011F45C
:104270000C94E52E9101A201B301C401E3E6AE2E38
:10428000F4E6BF2EA1E6CA2EDD24EE24FF2400E0D2
:1042900010E00E94636C823008F06BC0A9E62A1619
:1042A00089F4B2E73B1671F4442061F4552051F4CF
:1042B000662041F4772031F4882021F4992011F40C
:1042C0000C94872C9101A201B301C40119E6A12E1F
:1042D00002E7B02ECC24DD24EE24FF2400E010E021
:1042E0000E94636C823070F4E5E62E1611F00C9497
:1042F0003F303B1411F00C943F30442011F00C94EB
:104300003F30EAC1F3E72F1689F482E7381671F4DB
:10431000442061F4552051F4662041F4772031F4B3
:10432000882021F4992011F40C94E02C93E72916AD
:1043300011F00C943F30391611F00C943F304420AA
:1043400011F00C943F30552011F00C943F30662052
:1043500011F00C943F30772011F00C943F308820FE
:1043600011F00C943F30992011F00C943F300C94D4
:10437000EF2CA2E62A1689F4B5E63B1671F4E4E6C2
:104380004E1659F4552049F4662039F4772029F463
:10439000882019F4992009F4FEC49101A201B30107
:1043A000C401F2E6AF2EA5E6BA2EB4E6CB2EDD248C
:1043B000EE24FF2400E010E00E94636C8230B8F528
:1043C000F8E72F1681F43C1471F481E6481659F48D
:1043D000552049F4662039F4772029F4882019F40F
:1043E000992009F414C393E7291611F00C943F3077
:1043F000A5E63A1611F00C943F30B1E64B1611F0D9
:104400000C943F30552011F00C943F30662011F091
:104410000C943F30772011F00C943F30882011F03D
:104420000C943F30992011F00C943F302BC6E2E7FA
:104430002E1681F43E1671F4F5E64F1659F4552008
:1044400049F4662039F4772029F4882019F499205A
:1044500009F4AEC783E6281611F00C943F309DE6B0
:10446000391611F00C943F30A8E64A1611F00C945E
:104470003F30552011F00C943F30662011F00C9421
:104480003F30772011F00C943F30882011F00C94CD
:104490003F30992011F00C943F30C1C2B0E72B1689
:1044A00091F4ECE63E1679F4F5E64F1661F488E6F1
:1044B000581649F4662039F4772029F4882019F435
:1044C000992009F492C59101A201B301C401B0E79A
:1044D000AB2E1CE6B12E05E6C02EE8E6DE2EEE245D
:1044E000FF2400E010E00E94636C823008F043C1BA
:1044F00090E3291689F4A1E33A1671F4B1E74B165B
:1045000059F4552049F4662039F4772029F488209D
:1045100019F4992009F44CC79101A201B301C40117
:10452000E0E3AE2EF1E3BF2EA1E7CA2EDD24EE2498
:10453000FF2400E010E00E94636C823008F082C02B
:10454000E4E62E1689F4F3E63F1671F48CE648167D
:1045500059F4552049F4662039F4772029F488204D
:1045600019F4992009F4CEC69101A201B301C40146
:10457000B4E6AB2E13E6B12E0CE6C02EDD24EE24FD
:10458000FF2400E010E00E94636C823018F52B14C9
:1045900011F00C943F3092E3391611F00C943F3037
:1045A000A9E64A1611F00C943F30552011F00C94F6
:1045B0003F30662011F00C943F30772011F00C94BE
:1045C0003F30882011F00C943F30992011F00C946A
:1045D0003F3021C2B7E62B1689F4EFE63E1671F4A0
:1045E000FCE64F1659F4552049F4662039F477203B
:1045F00029F4882019F4992009F487C685E728163C
:1046000011F00C943F3093E6391611F00C943F30C2
:10461000ADE64A1611F00C943F30552011F00C9481
:104620003F30662011F00C943F30772011F00C944D
:104630003F30882011F00C943F30992011F00C94F9
:104640003F3019C7B4E72B1691F4E4E63E1679F42F
:10465000F7E74F1661F4552051F4662041F47720B6
:1046600031F4882021F4992011F40C94D52F910174
:10467000A201B301C401E4E7AE2EF4E6BF2EA7E722
:10468000CA2EDD24EE24FF2400E010E00E94636CBB
:104690008230C0F581E3281681F4381671F491E771
:1046A000491659F4552049F4662039F4772029F445
:1046B000882019F4992009F4DEC6A0E72A1611F023
:1046C0000C943F30B5E63B1611F00C943F30E2E716
:1046D0004E1611F00C943F30552011F00C943F30E1
:1046E000662011F00C943F30772011F00C943F308D
:1046F000882011F00C943F30992011F00C943F3039
:104700000C94212CF4E72F1689F48FE6381671F4F7
:10471000481661F492E6591649F4662039F4772078
:1047200029F4882019F4992009F40BC5A9E62A1662
:1047300011F00C943F30BCE63B1611F00C943F3066
:10474000E1E64E1611F00C943F30F3E65F1611F0DF
:104750000C943F30662011F00C943F30772011F01C
:104760000C943F30882011F00C943F30992011F0C8
:104770000C943F3080C183E7281699F492E73916EC
:1047800081F4A7E74A1669F4B0E75B1651F4662096
:1047900041F4772031F4882021F4992011F40C940D
:1047A000E52B9101A201B301C401A3E7AA2EB2E750
:1047B000BB2E17E7C12E00E7D02EEE24FF2400E029
:1047C00010E00E94636C823008F085C02D1491F4D3
:1047D000EDE63E1679F4F5E74F1661F488E65816D3
:1047E00049F4662039F4772029F4882019F49920B7
:1047F00009F4E6C69101A201B301C40110E7A12E9C
:104800000DE6B02EE5E7CE2EF8E6DF2EEE24FF24EF
:1048100000E010E00E94636C823010F591E62916EA
:1048200011F00C943F303B1411F00C943F304C14B9
:1048300011F00C943F305D1411F00C943F30662061
:1048400011F00C943F30772011F00C943F30882009
:1048500011F00C943F30992011F00C943F309FC61A
:10486000A3E72A1699F4B5E63B1681F4E2E74E1663
:1048700069F4F0E75F1651F4662041F4772031F4D3
:10488000882021F4992011F40C943E2F81E32816FE
:1048900011F00C943F3092E7391611F00C943F3030
:1048A000A7E74A1611F00C943F30B0E75B1611F001
:1048B0000C943F30662011F00C943F30772011F0BB
:1048C0000C943F30882011F00C943F30992011F067
:1048D0000C943F30A8C0E7E72E1691F4F0E73F169E
:1048E00079F488E7481661F494E7591649F466208C
:1048F00039F4772029F4882019F4992009F4F8C3B1
:104900009101A201B301C401E7E7AE2EF0E7BF2E8B
:10491000A8E7CA2EB4E7DB2EEE24FF2400E010E067
:104920000E94636C8230C0F52D1491F4A3E73A160F
:1049300079F4B5E64B1661F4E2E75E1649F46620B9
:1049400039F4772029F4882019F4992009F4EFC666
:10495000F4E72F1611F00C943F3083E7381611F06E
:104960000C943F3095E6491611F00C943F305F16D9
:1049700011F00C943F30662011F00C943F307720FA
:1049800011F00C943F30882011F00C943F309920A6
:1049900011F00C943F30D8C3A2E72A1691F4B7E681
:1049A0003B1679F4E0E74E1661F4F5E75F1649F43B
:1049B000662039F4772029F4882019F4992009F425
:1049C00072C48CE6281611F00C943F3091E639162B
:1049D00011F00C943F30A4E74A1611F00C943F30CC
:1049E000B8E75B1611F00C943F30662011F00C9480
:1049F0003F30772011F00C943F30882011F00C9458
:104A00003F30992011F00C943F300C94992F0E9464
:104A10007F150C9441300E94E30F0C9441300E94AA
:104A200008160C9441306091190570911A0580E0C8
:104A300090E00E9460778C0163EF72E00E947577CE
:104A4000009719F477980C944130C80166EF72E032
:104A50000E947577009719F4779A0C9441307799F2
:104A600003C083EF92E002C086EF92E000D000D056
:104A700028EC38E036C36091190570911A0580E082
:104A800090E00E9460778C016DE073E00E94757782
:104A9000009709F04DC06091190570911A0580E0EA
:104AA00090E00E9460778C01009711F40C944130E3
:104AB00060E173E00E947577009729F482E29FEF2E
:104AC000ACECBBE324C0C80166E173E00E947577DB
:104AD000009729F482E29FEFACECBAE318C0C8015A
:104AE0000E9453766B017C0120E030E040E050E012
:104AF0000E940D718823C1F081E00E94C10A9B01D0
:104B0000AC01C701B6010E941171DC01CB01809399
:104B1000200590932105A0932205B093230580E200
:104B200095E064E170E0B6C000D086E49CE07FC010
:104B3000C8016BE173E00E947577009709F04DC0E2
:104B40006091190570911A0580E090E00E946077ED
:104B50008C01009711F40C94413060E173E00E94E5
:104B60007577009729F482E29FEFACECBBE324C099
:104B7000C80166E173E00E947577009729F482E22C
:104B80009FEFACECBAE318C0C8010E9453766B01EA
:104B90007C0120E030E040E050E00E940D7188236D
:104BA000C1F082E00E94C10A9B01AC01C701B601BD
:104BB0000E941171DC01CB0180931C0590931D05AF
:104BC000A0931E05B0931F058CE195E060E170E0B5
:104BD00061C000D083E59CE064C0C8016EE173E071
:104BE0000E947577009709F066C060911905709171
:104BF0001A0580E090E00E9460778C01009711F424
:104C00000C94413060E173E00E947577009729F4BD
:104C10008DEE97E4AAE8BCE331C0C80166E173E019
:104C20000E947577009751F400D080E69CE0ADB704
:104C3000BEB712969C938E93119737C0C8010E94FD
:104C400053766B017C0120E030E040E050E00E94B0
:104C50000D71882319F180E00E94C10A4B015C01AB
:104C6000C701B60121EE3AE744E95EE30E94A8706D
:104C7000A50194010E941171DC01CB0180932405F0
:104C800090932505A0932605B093270584E295E02F
:104C900068E170E044E050E00C94183000D08FE6FA
:104CA0009CE0EDB7FEB7928381830E94F6770F9068
:104CB0000F900C9441300E94150BAB01BC0100D049
:104CC00000D000D08CE79CE0ADB7BEB712969C93A5
:104CD0008E931197EDB7FEB7438354836583768334
:104CE0000E94F6778DB79EB706960FB6F8949EBFD2
:104CF0000FBE8DBF81E00E94C10A20912005309136
:104D0000210540912205509123050E942B726B01D1
:104D1000182F092F82E00E94C10AAB01BC01ADB778
:104D2000BEB71A970FB6F894BEBF0FBEADBFEDB6B3
:104D3000FEB60894E11CF11C83E89CE012969C935B
:104D40008E93119798018C2D9D2DA32FB22FF701D3
:104D500082839383A483B583CB01BA0120911C0580
:104D600030911D0540911E0550911F050E942B7228
:104D7000DC01CB01F70186839783A087B1870E946E
:104D8000F6778DB79EB70A960FB6F8949EBF0FBE02
:104D90008DBF0C94D22F6091190570911A0580E097
:104DA00090E00E946077009771F160E070E040E170
:104DB00050E00E941275AB01BC018091B306909146
:104DC000B4068417950799F15093B4064093B3063F
:104DD00083EB96E06CE170E042E050E00E943C79A9
:104DE0008091B3069091B40600D000D02CEC38E04E
:104DF000ADB7BEB712963C932E93119714969C9321
:104E00008E9313970EC08091B3069091B40600D094
:104E100000D02CED38E0EDB7FEB7328321839483C8
:104E200083830E94F6770F900F900F900F900E944F
:104E30001C0C00D000D080EF98E0ADB7BEB7129642
:104E40009C938E93119781E090E014969C938E939F
:104E500013970E94F6778DEF98E0EDB7FEB7928337
:104E6000818382E090E0948383830E94F67788E0D8
:104E700099E0ADB7BEB712969C938E93119784E0DC
:104E800090E014969C938E9313970E94F67783E19B
:104E900099E0EDB7FEB79283818388E090E0948338
:104EA00083830E94F67780E299E0ADB7BEB7129691
:104EB0009C938E93119780E190E014969C938E932F
:104EC00013970E94F6778BE299E0EDB7FEB79283D5
:104ED000818380E290E0948383830E94F67787E366
:104EE00099E0ADB7BEB712969C938E93119780E46C
:104EF00090E014969C938E9313970E94F67785E426
:104F000099E0EDB7FEB79283818380E890E09483C7
:104F100083830E94F67783E599E0ADB7BEB712961A
:104F20009C938E93119780E091E014969C938E93BE
:104F300013970E94F67782E699E0EDB7FEB7928369
:104F4000818380E092E0948383830E94F67781E7F7
:104F500099E0ADB7BEB712969C938E93119780E0FF
:104F600094E014969C938E9313970E94F6778DE7A6
:104F700099E0EDB7FEB79283818380E098E0948357
:104F800083830E94F6778BE899E0ADB7BEB712969F
:104F90009C938E93119780E090E114969C938E934E
:104FA00013970E94F67788E999E0EDB7FEB79283F0
:104FB000818380E090E2948383830E94F67786EA7F
:104FC00099E0ADB7BEB712969C938E93119780E08F
:104FD00090E414969C938E9313970E94F6770F900B
:104FE0000F900F900F900C9441300E9450180C9429
:104FF00041306091190570911A0580E090E00E949F
:10500000607760E173E00E947577009711F481E0AA
:1050100001C080E00E94871A20911B05222311F411
:105020000C94413000D000D0EDB7FEB7319686EB3E
:1050300099E00FC00E94391920911B05222311F419
:105040000C94413000D000D0EDB7FEB7319689EB1B
:1050500099E0ADB7BEB712969C938E9311972283B9
:105060001382BBCF0E94341920911B05222311F417
:105070000C94413000D000D0EDB7FEB731968CEBE8
:1050800099E0E7CF6091190570911A0580E090E0F2
:105090000E9460778C0163EF72E00E947577009741
:1050A00031F48091FF04909100058460B7C7C80176
:1050B00066EF72E00E9475779C018091FF049091E9
:1050C00000052115310511F48B7FA8C782FF03C0AD
:1050D00083EF92E002C086EF92E000D000D02FE88C
:1050E0003CE0EDB7FEB7328321839483838375CF91
:1050F0006091190570911A0580E090E00E94607738
:105100000E945776803160F48093AF0690E00E9451
:105110008A518FEA96E069E070E041E050E088C78C
:1051200000D000D0EDB7FEB731968FEB99E0ADB768
:10513000BEB712969C938E9311978091AF0682838F
:105140008FCF0C9400009DC76091190570911A05CE
:1051500080E090E00E9460778C0163E273E00E943F
:105160007577009739F4219A8091FF04909100059A
:10517000806154C7C80165E273E00E9475770097AB
:1051800039F4229A8091FF0490910005806246C70D
:10519000C80167E273E00E947577009739F4239A9B
:1051A0008091FF0490910005806438C7C80169E2CE
:1051B00073E00E947577009739F4239A8091FF0479
:1051C0009091000580682AC7C80166EF72E00E94CE
:1051D00075779C018091FF049091000521153105A0
:1051E00039F48F70909300058093FF042B9A1AC7AF
:1051F00084FF03C083EF92E002C086EF92E000D00C
:1052000000D023E93CE0EDB7FEB7328321839483DD
:1052100083830E94F6778091FF040F900F900F9088
:105220000F9085FF03C083EF92E002C086EF92E00B
:1052300000D000D02EE93CE0ADB7BEB712963C934B
:105240002E93119714969C938E9313970E94F67742
:105250008091FF040F900F900F900F9086FF03C076
:1052600083EF92E002C086EF92E000D000D029EAFE
:105270003CE0EDB7FEB732832183948383830E94A1
:10528000F6778091FF040F900F900F900F9087FF9B
:1052900003C083EF92E002C086EF92E000D000D01E
:1052A00024EB3CE0E4C600D08CEC99E0EDB7FEB70F
:1052B000928381830E94F67720911B050F900F90B7
:1052C0002223A9F000D000D0EDB7FEB7319680EDD3
:1052D00099E0ADB7BEB712969C938E931197228337
:1052E00013820E94F6770F900F900F900F9088E135
:1052F0000FB6F89480936000109260000FBE0C947B
:10530000007CBFC60E947548BCC6609119057091AB
:105310001A0580E090E00E9460777C0163EF72E004
:105320000E947577009749F40E94384E8091FF04DF
:105330009091000581608D7F71C6C70166EF72E0B4
:105340000E947577009741F40E94294F8091FF04D5
:10535000909100058C7F62C60BE213E0C701B80193
:105360000E947577009749F40E94294F8091FF04AD
:10537000909100058E7F826051C68091FF0481FF6D
:105380000BC000D000D08FEB9CE0EDB7FEB792834E
:1053900081831483038321CE80FF03C083EF92E0D7
:1053A00002C086EF92E000D000D023EC3CE05FC664
:1053B00000D083ED99E0EDB7FEB7928381830E9420
:1053C000F6778DB79EB740970FB6F8949EBF0FBE85
:1053D0008DBFEDB7FEB731968DEF99E0ADB7BEB793
:1053E00012969C938E93119780912B2090912C2054
:1053F000A0912D20B0912E2082839383A483B58326
:1054000080911F2090912020A0912120B0912220F6
:1054100086839783A087B187809123209091242051
:10542000A0912520B091262082879387A487B587F5
:105430008091272090912820A0912920B0912A20A6
:1054400086879787A08BB18B0E94F67720911B05EA
:10545000EDB7FEB772960FB6F894FEBF0FBEEDBF64
:10546000222309F40EC600D000D0EDB7FEB7319666
:105470008BE19AE0EECDF89409E081E090E0FC0148
:1054800000935700C895F02C20E030E0F90100931C
:105490005700C895E02C7894F89423E030E0F901A7
:1054A00000935700C895102D82E090E0FC01009316
:1054B0005700C895002D789400D000D000D02EE180
:1054C0003AE0EDB7FEB7328321838091CC179091FB
:1054D000CD17A091CE17B091CF1783839483A58366
:1054E000B6830E94F67700D000D0EDB7FEB73196B4
:1054F00088E29AE0ADB7BEB712969C938E9311974F
:105500000283138214831582E6821782F086118645
:105510000E94F677EDB7FEB73A960FB6F894FEBF45
:105520000FBEEDBF0E94EB192091660000D000D0A5
:10553000EDB7FEB731968FE49AE0ADB7BEB71296DD
:105540009C938E931197228313820E94F6770F907B
:105550000F900F900F900E941C0C20911B0522238E
:1055600009F48FC500D000D0EDB7FEB731968BE5BA
:105570009AE06FCD80E090E00E94280C81E090E0FE
:105580000E94280C20911B05222309F47AC500D023
:1055900000D0EDB7FEB731968EE59AE05ACD0E9465
:1055A000BF170E941C0C20911B05222309F469C51A
:1055B00000D000D0EDB7FEB7319681E69AE049CD34
:1055C0006091190570911A0580E090E00E94607763
:1055D0008C0163EF72E00E947577009731F480913F
:1055E000FF0490910005886019C5C80166EF72E05C
:1055F0000E9475779C018091FF0490910005211510
:10560000310511F4877F0AC583FF03C083EF92E061
:1056100002C086EF92E000D000D027EC3CE061CDE4
:105620006091190570911A0580E090E00E94607702
:1056300060E373E00E947577009731F5F89489EB89
:1056400096E00E94C13C0CC0C8010D960E94D93F53
:105650008CE295E0B8010E94793CC8010E94673D48
:105660008C01009789F704C089EB96E00E94EE3C1C
:1056700089EB96E00E94493D0097B1F789EB96E0EF
:105680000E94BD3C789446C089EB96E00E94C13CE4
:105690007C0106E313E03BC08DB79EB70C970FB6B5
:1056A000F8949EBF0FBE8DBFEDB7FEB73196ADB774
:1056B000BEB712961C930E931197D70112968C9138
:1056C00012978283138213968C9113978483158289
:1056D00018968C9118978683178214968D919C91B9
:1056E00015979187808716968D919C911797938730
:1056F00082870E94E477EDB7FEB73C960FB6F89428
:10570000FEBF0FBEEDBFC7010E94673D7C01E114E3
:10571000F10411F620911B05222309F4B2C400D034
:1057200000D0EDB7FEB7319684E69AE092CC0E94A5
:10573000CB1AA7C46091190570911A0580E090E01A
:105740000E9460778C0163EF72E00E94757700978A
:1057500031F48091FF049091000592600EC0C80161
:1057600066EF72E00E9475779C018091FF04909132
:1057700000052115310571F49D7F909300058093FC
:10578000FF048FEF94E06AE070E042E050E00E9496
:105790003C7917C091FF03C083EF92E002C086EF0F
:1057A00092E000D000D02BEC3CE0EDB7FEB73283A6
:1057B0002183948383830E94F6770F900F900F903C
:1057C0000F9081E00E942D0A5CC4609119057091D0
:1057D0001A0580E090E00E9460778C0165E073E03C
:1057E0000E947577009731F48091FF049091000535
:1057F0009E7F14C4C8016AEF72E00E9475779C0115
:105800008091FF04909100052115310511F49160FC
:1058100005C490FF03C08AEF92E002C085E093E0E8
:1058200000D000D02DE533E0ADB7BEB712963C9363
:105830002E93119714969C938E9313970E94E4775E
:10584000CECB6091190570911A0580E090E00E941E
:105850006077009769F160E070E040E150E00E94FD
:105860001275DC01CB01909304058093030500D0F1
:1058700000D04DB75EB74F5F5F4F27E63AE0EDB718
:10588000FEB732832183FA01938382830E94F677E5
:105890000F900F900F900F9083E095E06EE070E016
:1058A00042E050E00E943C7981E00E94681BE9C31D
:1058B00080E00E94681B0E941C0C00D000D088E78A
:1058C0009AE0ADB7BEB712969C938E9311978091D4
:1058D00003059091040514969C938E9313970E9450
:1058E000F6770F900F900F900F9081E00E94681B49
:1058F0000E941C0C20911B05222309F4C2C300D076
:1059000000D0EDB7FEB731968BE89AE0A2CB60915C
:10591000190570911A0580E090E00E946077009769
:1059200051F160E070E04AE050E00E941275DC0145
:10593000CB01909302058093010500D000D04DB7B4
:105940005EB74F5F5F4F2EE83AE0EDB7FEB73283A8
:105950002183FA01938382830E94F6770F900F9040
:105960000F900F9081E095E06CE070E042E050E035
:105970000E943C7918C000D000D08BEA9AE0ADB705
:10598000BEB712969C938E931197809101059091CA
:10599000020514969C938E9313970E94F6770F90AE
:1059A0000F900F900F9020911B05222309F469C3DB
:1059B00000D000D0EDB7FEB731968CEC9AE049CB21
:1059C0000E94124020911B05222309F45AC300D0E3
:1059D00000D0EDB7FEB731968FEC9AE03ACB00D00D
:1059E00082ED9AE0EDB7FEB7928381830E94F6774D
:1059F0000F900F900E94341900D082EE9AE0ADB75C
:105A0000BEB712969C938E9311970E94F6770F90D3
:105A10000F9080E00E94871A00D086EE9AE0EDB7E2
:105A2000FEB7928381830E94F6770F900F900E94B9
:105A3000E30F8091191C80FF02C00E9422110E9476
:105A4000391900D000D0EDB7FEB731968CEE9AE050
:105A5000ADB7BEB712969C938E9311978091AF0607
:105A6000828313820E94F67789EF9AE0EDB7FEB742
:105A70009283818380E490E0948383830E94F6770D
:105A800000D0EDB7FEB7319681E19BE0ADB7BEB770
:105A900012969C938E931197809195248283138202
:105AA00080919624848315820E94F6770F900F9040
:105AB00084E29BE0EDB7FEB792838183809101057C
:105AC00090910205948383830E94F67789E39BE09B
:105AD000ADB7BEB712969C938E9311978091030534
:105AE0009091040514969C938E9313970E94F677D9
:105AF0000F900F900F900F9081E00E94681B0E9402
:105B0000150BAB01BC0100D000D000D08CE49BE0B1
:105B1000EDB7FEB792838183438354836583768395
:105B20000E94F677EDB7FEB736960FB6F894FEBF33
:105B30000FBEEDBF0E945E0B0E942F0BAB01BC019C
:105B400000D000D000D089E59BE0ADB7BEB712967B
:105B50009C938E931197EDB7FEB74383548365836F
:105B600076830E94F6778DB79EB706960FB6F894A7
:105B70009EBF0FBE8DBF1D9B03C08AE093E002C095
:105B800086EF92E000D000D027E63BE0ADB7BEB78D
:105B900012963C932E93119714969C938E93139781
:105BA0000E94F6778091702490917124A0917224C4
:105BB000B09173244091742450917524609176249F
:105BC0007091772400D000D000D00DB71EB70F5FC2
:105BD0001F4F23E73BE0EDB7FEB732832183F80187
:105BE00082839383A483B5834683578360877187B9
:105BF0000E94F677EDB7FEB7319681E99BE0ADB72D
:105C0000BEB712969C938E93119780917D249091AC
:105C10007E24A0917F24B091802482839383A483E7
:105C2000B5838091812490918224A0918324B091A6
:105C3000842486839783A087B1870E94F677EDB787
:105C4000FEB738960FB6F894FEBF0FBEEDBF83EBDC
:105C50009BE0928381830E94F6778091FF040F90EE
:105C60000F9081FF0EC000D08DEB9BE0ADB7BEB7AB
:105C700012969C938E9311970E94F6770F900F9037
:105C800017C080FF03C083EF92E002C086EF92E06E
:105C900000D000D023EC3BE0EDB7FEB73283218388
:105CA000948383830E94F6770F900F900F900F904C
:105CB0008091FF0483FF03C083EF92E002C086EF70
:105CC00092E000D000D027EC3BE0ADB7BEB7129613
:105CD0003C932E93119714969C938E9313970E9446
:105CE000F6778091FF04909100050F900F900F9030
:105CF0000F9091FF03C083EF92E002C086EF92E025
:105D000000D000D02AED3BE0EDB7FEB7328321830F
:105D1000948383830E94F6778091B3069091B406B2
:105D200027EE3BE0ADB7BEB712963C932E9311978A
:105D300014969C938E9313970E94F6770F900F9072
:105D40000F900F90779903C083EF92E002C086EF27
:105D500092E000D000D024EF3BE0EDB7FEB73283F5
:105D60002183948383830E94F6778091FF0490912E
:105D700000050F900F900F900F9090FF03C08AEFD7
:105D800092E002C085E093E000D000D02DE533E042
:105D9000ADB7BEB712963C932E93119714969C9371
:105DA0008E9313970E94E47720911B050F900F901C
:105DB0000F900F90222309F464C100D000D0EDB7FA
:105DC000FEB731968DEF9BE044C90E94101A2091D6
:105DD0001B05222309F455C100D000D0EDB7FEB752
:105DE000319680E09CE035C90E9403170097B9F511
:105DF00000D000D000D083E09CE0EDB7FEB79283E6
:105E000081838091151890911618A0911718B09160
:105E1000181883839483A583B6830E94F6778EE057
:105E20009CE0ADB7BEB712969C938E93119780916C
:105E3000912490919224A0919324B0919424EDB751
:105E4000FEB783839483A583B6830E94F6778DB7CC
:105E50009EB706960FB6F8949EBF0FBE8DBF0E94E8
:105E60001C0C20911B05222309F40BC100D000D08B
:105E7000EDB7FEB731968BE19CE0EBC883E061E0C3
:105E800048E021E00E94B01200D000D000D08EE1A6
:105E90009CE0EDB7FEB792838183809108189091C2
:105EA0000918A0910A18B0910B1883839483A583D5
:105EB000B6830E94F67700D000D0EDB7FEB73196DA
:105EC00085E29CE0ADB7BEB712969C938E93119776
:105ED00080910C1890910D18A0910E18B0910F1888
:105EE00082839383A483B5838091101890911118B5
:105EF000A0911218B091131886839783A087B18759
:105F00000E94F677EDB7FEB73A960FB6F894FEBF4B
:105F10000FBEEDBF0E941C0C20911B05222309F42B
:105F2000B0C000D000D0EDB7FEB7319686E39CE05C
:105F300090C86091190570911A0580E090E00E9468
:105F4000607766E673E00E9475770097B1F4609120
:105F5000190570911A0580E090E00E946077009723
:105F600009F48FC00E945776803108F08AC0909162
:105F70005201982B9093520184C08091520100D01D
:105F800000D029E33CE0EDB7FEB73283218390E0F7
:105F90008F709070948383830E94F6770F900F9098
:105FA0000F900F900E941C0C6CC0609119057091AD
:105FB0001A0580E090E00E9460778C0163EF72E048
:105FC0000E947577009741F40E94244D8091FF0450
:105FD00090910005946022C0C80166EF72E00E94B3
:105FE0007577009741F5F8940E94324D88E10FB61D
:105FF000F89480936000109260000FBE84B7877F92
:1060000084BF80916000886180936000109260007E
:1060100078948091FF04909100059B7F90930005F8
:106020008093FF048FEF94E06AE070E042E050E07C
:106030000E943C7926C0C8016BE673E00E94757728
:106040009C018091FF04909100052115310521F4F8
:1060500092FF17C0F894FFCF92FF03C083EF92E046
:1060600002C086EF92E000D000D02FEC3CE0ADB74C
:10607000BEB712963C932E9311970C94E9270E9479
:106080002918E981FA811182108283E00F900F9024
:10609000DF91CF911F910F91FF90EF90DF90CF9004
:1060A000BF90AF909F908F907F906F905F904F9038
:1060B0003F902F900895F89491E2E0E0F0E0909303
:1060C00057008491E2E0F0E0909357004491E4E0BF
:1060D000F0E090935700E49190E0A0E0B0E0DC01A4
:1060E0009927882750E060E070E0762F652F542FC5
:1060F0004427840F951FA61FB71F8E0F911DA11D4A
:10610000B11D8093CC179093CD17A093CE17B09369
:10611000CF1778940895CF93DF93CDB7DEB7279745
:106120000FB6F894DEBF0FBECDBFCE0102966EE073
:1061300070E042E050E00E941E798A819B812FEF3F
:106140008F3F920749F483E095E06EE070E042E013
:1061500050E00E943C7904C09093040580930305AD
:10616000CE0102966CE070E042E050E00E941E79A1
:106170008A819B812FEF8F3F920779F48CE390E027
:10618000909302058093010581E095E06CE070E05A
:1061900042E050E00E943C7904C090930205809355
:1061A0000105CE0102966AE070E042E050E00E94F4
:1061B0001E798A819B812FEF8F3F920779F48AE0C5
:1061C00090E0909300058093FF048FEF94E06AE0E5
:1061D00070E042E050E00E943C7904C090930005DA
:1061E0008093FF04CE0102966CE170E042E050E043
:1061F0000E941E798A819B812FEF8F3F920769F45D
:106200001092B4061092B30683EB96E06CE170E056
:1062100042E050E00E943C7904C09093B406809321
:10622000B30685E894E260E070E049E050E00E9447
:106230001E790E94A40DCE01049664E170E044E052
:1062400050E00E941E798C819D81AE81BF818F3F7D
:106250002FEF92072FEFA2072FEFB20749F480E24A
:1062600095E064E170E044E050E00E943C7908C0B1
:1062700080E295E064E170E044E050E00E941E7925
:10628000CE01049660E170E044E050E00E941E7987
:106290008C819D81AE81BF818F3F2FEF92072FEFC1
:1062A000A2072FEFB20749F48CE195E060E170E0BE
:1062B00044E050E00E943C7908C08CE195E060E148
:1062C00070E044E050E00E941E79CE01049668E13F
:1062D00070E044E050E00E941E798C819D81AE8187
:1062E000BF818F3F2FEF92072FEFA2072FEFB2074B
:1062F00049F484E295E068E170E044E050E00E94F7
:106300003C7908C084E295E068E170E044E050E048
:106310000E941E79CE01019669E070E041E050E0F4
:106320000E941E7989818F3F49F48FEA96E069E0E7
:1063300070E041E050E00E943C7908C08FEA96E0AE
:1063400069E070E041E050E00E941E7927960FB6A8
:10635000F894DEBF0FBECDBFDF91CF9108950E94AC
:10636000184D6C9A6B9A6A9A6F9A729A749A739A89
:10637000779A809880B3897F80BB87E080937E0086
:10638000549A0E945B300E948B3081E00E942D0A5B
:1063900080E090E00E94B80D0E94EC468091FF04DE
:1063A00086FD239A0895CF93DF93EC01888199812C
:1063B000009731F029E0853D920709F08CC082C03A
:1063C0000E94AF318091FF0480FD06C081FF02C0B2
:1063D0001D9902C00E94294F809170008C7F80938C
:1063E00070008091B60080628093B6001092B20077
:1063F00082E08093B1008091B60090E08770907049
:106400000097C9F78091700081608093700080E0F0
:1064100090E06CE478E00E94FB4C0E94341980E02C
:106420000E94871A00D083ED9CE0ADB7BEB71296EC
:106430009C938E9311970E94F6770F900F900E9475
:10644000E30F8091191C86FF02C00E94204880E063
:1064500090E00E948A510E94EB4F8093BB0600D0CF
:1064600000D000D0EDB7FEB7319620E733E0ADB7EE
:10647000BEB712963C932E9311978283138280911C
:10648000AF06848315820E94E4771092BD061092B5
:10649000BC06EDB7FEB736960FB6F894FEBF0FBE3A
:1064A000EDBF85EF94E090938F2480938E2483E258
:1064B00090E09093BF068093BE0685ED99E09983A6
:1064C00088830DC0633259F48CEB96E060E070E095
:1064D0000E94AD1DE6CF1982188283E001C081E0E1
:1064E000DF91CF9108958536910564F12091B3062F
:1064F0003091B40620FF10C000D000D022E833E075
:10650000EDB7FEB732832183948383830E94E477BF
:106510000F900F900F900F9080912B2090912C2036
:10652000A0912D20B0912E200196A11DB11D809328
:106530002B2090932C20A0932D20B0932E2081E02F
:1065400090E0089580E090E008954F925F926F92FE
:106550007F928F929F92AF92BF92CF92DF92EF92F3
:10656000FF920F931F93CF93DF93CDB7DEB7CB5737
:10657000D0400FB6F894DEBF0FBECDBF2C016338FC
:1065800051F486EC96E0EC966FAFEC970E94FF39E1
:10659000EC966FADEC97D2018D919C911197B8E07C
:1065A000823C9B07E9F0E8E0833C9E0718F40097E3
:1065B00061F09AC6F9E08C399F0709F46EC629E0AC
:1065C000833A920709F090C681C686EC96E061E8AE
:1065D00070E044E355E00E94E43982EC98E071C633
:1065E000623109F086C60E945E0B8091030590918E
:1065F000040592FF02C00E94031780910305909149
:10660000040593FF0CC00E94150BDC01CB018093A5
:10661000782490937924A0937A24B0937B2480915A
:10662000030580FF60C000D000D000D0EDB7FEB7FA
:10663000319672E0C72ED12CCC0EDD1EADB7BEB7A1
:106640001296DC92CE92119788E790E09383828332
:1066500086E993E0958384830E944B788C0185E8DA
:10666000A82E84E2B82EEDB7FEB736960FB6F89492
:10667000FEBF0FBEEDBFEE24FF2498E7892E912CBC
:106680002AE9622E23E0722ED5012D915D01EDB72E
:10669000FEB738970FB6F894FEBF0FBEEDBF319628
:1066A000C601800F911FADB7BEB712969C938E9313
:1066B00011979382828275826482268317820E9458
:1066C0004B78080F191F0894E11CF11CEDB7FEB7B9
:1066D00038960FB6F894FEBF0FBEEDBFF8E0EF1688
:1066E000F10491F602C000E010E080910305909162
:1066F0000405009781F12DB73EB7285030400FB602
:10670000F8943EBF0FBE2DBFEDB7FEB73196CE0158
:106710000296800F911FADB7BEB712969C938E93D1
:10672000119788E790E0938382838FE993E09583C4
:1067300084838091B0069091B106978386830E94EE
:106740004B78080F191FEDB7FEB738960FB6F894BF
:10675000FEBF0FBEEDBF8091030581FF51C089E2EE
:1067600090E06BE270E04AE250E027E00E940D44C6
:1067700085E894E20E9474462DB73EB72A50304017
:106780000FB6F8943EBF0FBE2DBFEDB6FEB608940F
:10679000E11CF11C9E012E5F3F4F200F311FADB752
:1067A000BEB712963C932E93119728E730E0F7017D
:1067B0003383228326EA33E0358324839C01B901A5
:1067C000882777FD8095982F0E947B7120E030E02C
:1067D00048EC52E40E941171DC01CB01F701868381
:1067E0009783A087B1870E944B78080F191F2DB798
:1067F0003EB7265F3F4F0FB6F8943EBF0FBE2DBF8A
:106800008091030582FF57C089E290E06BE270E05F
:106810004AE250E026E00E940D4481E090E00E94B0
:10682000B00B8093AE0684E897E10E9474464DB7A2
:106830005EB74A5050400FB6F8945EBF0FBE4DBFD2
:10684000EDB6FEB60894E11CF11C9E012E5F3F4F91
:10685000200F311FADB7BEB712963C932E93119700
:1068600028E730E0F7013383228320EB33E03583E0
:1068700024839C01B901882777FD8095982F0E9479
:106880007B7120E030E048EC52E40E941171DC01A1
:10689000CB01F70186839783A087B1870E944B784D
:1068A000080F191F2DB73EB7265F3F4F0FB6F8945C
:1068B0003EBF0FBE2DBF8091030583FF36C04DB78D
:1068C0005EB74A5050400FB6F8945EBF0FBE4DBF42
:1068D000EDB7FEB73196CE010296800F911FADB78E
:1068E000BEB712969C938E93119788E790E093839E
:1068F00082838BEB93E095838483809170179091D2
:106900007117A0917217B091731786839783A08730
:10691000B1870E944B78080F191FEDB7FEB73A9662
:106920000FB6F894FEBF0FBEEDBF8091030584FF44
:1069300032C00E942F0BAB01BC012DB73EB72A50CD
:1069400030400FB6F8943EBF0FBE2DBFEDB7FEB777
:106950003196CE010296800F911FADB7BEB7129649
:106960009C938E93119788E790E09383828389ECC0
:1069700093E09583848346835783608771870E9461
:106980004B78080F191FEDB7FEB73A960FB6F8947B
:10699000FEBF0FBEEDBF8091030585FF38C0F894A0
:1069A00040917024509171246091722470917324ED
:1069B00078942DB73EB72A5030400FB6F8943EBFBA
:1069C0000FBE2DBFEDB7FEB73196CE010296800FF8
:1069D000911FADB7BEB712969C938E93119788E71F
:1069E00090E09383828387ED93E09583848346834D
:1069F0005783608771870E944B78080F191FEDB786
:106A0000FEB73A960FB6F894FEBF0FBEEDBF809169
:106A1000030586FF8DC080910105909102050097C6
:106A200009F486C0F8948090702490907124A0900E
:106A30007224B0907324789480917C1790917D1784
:106A4000A0917E17B0917F17A5019401281B390BE7
:106A50004A0B5B0BCA01B9010E947971E62EC72E61
:106A6000F82ED92E609101057091020580E090E02A
:106A70000E9479719B01AC018E2D9C2DAF2DBD2DF7
:106A8000BC01CD010E941171E82EC92E4DB75EB731
:106A90004A5050400FB6F8945EBF0FBE4DBFEDB7E1
:106AA000FEB73196CE010296800F911FADB7BEB7EB
:106AB00012969C938E93119788E790E0938382833C
:106AC00080EE93E095838483862F972FAE2DBC2D87
:106AD00086839783A087B187EC966FAFEC97EB9690
:106AE0007FAFEB970E944B78080F191FEC966FADA4
:106AF000EC97EB967FADEB97862F972FAE2DBC2DA5
:106B000080937D2490937E24A0937F24B09380244F
:106B100080927C1790927D17A0927E17B0927F177B
:106B2000EDB7FEB73A960FB6F894FEBF0FBEEDBFB5
:106B30008091030587FF3EC0F894409174245091E2
:106B40007524609176247091772478942DB73EB7A0
:106B50002A5030400FB6F8943EBF0FBE2DBFEDB7A0
:106B6000FEB73196CE010296800F911FADB7BEB72A
:106B700012969C938E93119788E790E0938382837B
:106B80008DEE93E095838483468357836087718776
:106B90000E944B78080F191FEDB7FEB73A960FB653
:106BA000F894FEBF0FBEEDBFC8010E94733200977C
:106BB00009F013CD809103059091040590FF8DC0DD
:106BC0008091010590910205009709F486C0F89420
:106BD0008090742490907524A0907624B0907724AF
:106BE00078948091801790918117A0918217B0912D
:106BF0008317A5019401281B390B4A0B5B0BCA01B3
:106C0000B9010E947971E62EC72EF82ED92E609117
:106C100001057091020580E090E00E9479719B016E
:106C2000AC018E2D9C2DAF2DBD2DBC01CD010E9440
:106C30001171E82EC92E4DB75EB74A5050400FB6BD
:106C4000F8945EBF0FBE4DBFEDB7FEB73196CE01D3
:106C50000296800F911FADB7BEB712969C938E938C
:106C6000119788E790E09383828386EF93E0958382
:106C70008483862F972FAE2DBC2D86839783A08784
:106C8000B187EC966FAFEC97EB967FAFEB970E94D6
:106C90004B78080F191FEC966FADEC97EB967FAD14
:106CA000EB97862F972FAE2DBC2D80938124909348
:106CB0008224A0938324B09384248092801790929E
:106CC0008117A0928217B0928317EDB7FEB73A965C
:106CD0000FB6F894FEBF0FBEEDBF809103059091F3
:106CE000040591FF3CC040911B2050911C206091F5
:106CF0001D2070911E202DB73EB72A5030400FB690
:106D0000F8943EBF0FBE2DBFEDB7FEB73196CE0152
:106D10000296800F911FADB7BEB712969C938E93CB
:106D2000119788E790E09383828383E094E09583D2
:106D3000848346835783608771870E944B78080F4E
:106D4000191FEDB7FEB73A960FB6F894FEBF0FBE07
:106D5000EDBFC8010E947332009709F03ECC8091CC
:106D600003059091040592FF3CC02DB73EB72A5011
:106D700030400FB6F8943EBF0FBE2DBFEDB7FEB743
:106D80003196CE010296800F911FADB7BEB7129615
:106D90009C938E93119788E790E0938382838CE095
:106DA00094E0958384838091151890911618A09192
:106DB0001718B091181886839783A087B1870E940F
:106DC0004B78080F191FEDB7FEB73A960FB6F89437
:106DD000FEBF0FBEEDBFC8010E947332009709F0DD
:106DE000FCCB809103059091040593FF3CC02DB727
:106DF0003EB72A5030400FB6F8943EBF0FBE2DBFAD
:106E0000EDB7FEB73196CE010296800F911FADB758
:106E1000BEB712969C938E93119788E790E0938368
:106E2000828387E194E09583848380917824909194
:106E30007924A0917A24B0917B2486839783A087BC
:106E4000B1870E944B78080F191FEDB7FEB73A962D
:106E50000FB6F894FEBF0FBEEDBFC8010E9473329B
:106E6000009709F0BACB809103059091040594FF37
:106E70004CC081E00E94C10AAB01BC012DB73EB7F6
:106E80002A5030400FB6F8943EBF0FBE2DBFEDB66E
:106E9000FEB60894E11CF11CCE010296800F911FF2
:106EA000ADB7BEB712969C938E93119788E790E08A
:106EB000F7019383828384E294E095838483CB01FA
:106EC000BA01209120053091210540912205509171
:106ED00023050E942B72DC01CB01F7018683978387
:106EE000A087B1870E944B78080F191F2DB73EB7B6
:106EF000265F3F4F0FB6F8943EBF0FBE2DBFC801AF
:106F00000E947332009709F068CB8091030590913D
:106F1000040595FF4BC082E00E94C10AAB01BC0191
:106F20008DB79EB70A970FB6F8949EBF0FBE8DBF60
:106F3000EDB6FEB60894E11CF11CCE010296800F5E
:106F4000911FADB7BEB712969C938E93119788E7A9
:106F500090E0F7019383828381E394E095838483B7
:106F6000CB01BA0120911C0530911D0540911E05F1
:106F700050911F050E942B72DC01CB01F701868323
:106F80009783A087B1870E944B78080F191F2DB7F0
:106F90003EB7265F3F4F0FB6F8943EBF0FBE2DBFE2
:106FA000C8010E947332009709F017CB8091030546
:106FB0009091040596FF06C083E061E046E020E082
:106FC0000E94B012809103059091040597FF06C0BE
:106FD00083E061E046E021E00E94B0128091030569
:106FE0009091040596FF3CC04DB75EB74A505040A3
:106FF0000FB6F8945EBF0FBE4DBFEDB7FEB731962A
:10700000CE010296800F911FADB7BEB712969C932A
:107010008E93119788E790E0938382838EE394E0C8
:107020009583848380910C1890910D18A0910E186F
:10703000B0910F1886839783A087B1870E944B7801
:10704000080F191FEDB7FEB73A960FB6F894FEBFBA
:107050000FBEEDBFC8010E947332009709F0BDCA90
:10706000809103059091040597FF3CC02DB73EB772
:107070002A5030400FB6F8943EBF0FBE2DBFEDB77B
:10708000FEB73196CE010296800F911FADB7BEB705
:1070900012969C938E93119788E790E09383828356
:1070A00086E494E095838483809110189091111860
:1070B000A0911218B091131886839783A087B18787
:1070C0000E944B78080F191FEDB7FEB73A960FB61E
:1070D000F894FEBF0FBEEDBFC8010E947332009747
:1070E00009F07BCA779A8091B3069091B40693FD1C
:1070F000749A8091B3069091B40682FD08C0809185
:10710000FF0480FD04C081FF31C01D9B2FC000D053
:1071100000D081E594E0ADB7BEB712969C938E93F4
:107120001197CE01029614969C938E9313970E940A
:10713000E47720911B050F900F900F900F90222362
:10714000A9F000D000D0EDB7FEB7319689ED9CE0F4
:10715000ADB7BEB712969C938E931197228313827C
:107160000E94F6770F900F900F900F908091D106AC
:107170008983FE01E00FF11F12828091B306909186
:10718000B40680FF12C000D000D088E594E0EDB7CF
:10719000FEB792838183C8010296948383830E9401
:1071A000E4770F900F900F900F9062E0C62ED12CD5
:1071B000C00ED11ECE010196B6010E9419438091E6
:1071C000FF0482FF49C085E095E0BE016F5F7F4FFD
:1071D000A60120E730E20E9485478091B306909196
:1071E000B40692FF39C040E7E42E40E2F42E00E0FE
:1071F00010E059E6A52E54E0B52ED7018D917D0102
:1072000000D000D0EDB7FEB73196ADB7BEB712963D
:10721000BC92AE921197828313820E94E4770F5F33
:107220001F4F0F900F900F900F900031110529F70D
:107230008AE090E00E94167800D000D08EE694E0BC
:10724000EDB7FEB792838183D482C3820E94E47734
:107250000F900F900F900F908091B3069091B4060D
:1072600082FD73980E94384E86EC96E00E94023AA6
:107270008091B0069091B106009711F00E94294FBD
:107280008091D1068F5F8093D1068091B306909153
:10729000B40682FFA2C9739AA0C982ED96E00E944B
:1072A000843E009731F10E94384E8091FF0487FDA3
:1072B0002B9882ED96E060E470E00E94593E83EAEC
:1072C00099E0D20111969C938E9313C082ED96E0C3
:1072D0000E94843E009769F00E94294F8091FF042C
:1072E00087FF7BC92B9A79C9F2011182108283E052
:1072F00001C081E0C558DF4F0FB6F894DEBF0FBE66
:10730000CDBFDF91CF911F910F91FF90EF90DF9054
:10731000CF90BF90AF909F908F907F906F905F9035
:107320004F9008950895FC01DB018C9180831196A4
:107330008C91119781830895FC01DB0190818C91E0
:10734000981741F421E030E0918111968C911197CA
:10735000981711F020E030E0C9010895BC0185E9DB
:1073600094E20E9493390895DC011996ED91FC9105
:107370001A970280F381E02D309709F0099508955E
:107380000F931F93CF93DF9300D0CDB7DEB78C015F
:1073900088E10E948843BC01CE0101960E94933986
:1073A000D8011996ED91FC911A970190F081E02D8A
:1073B000C801BE016F5F7F4F09950F900F90DF915D
:1073C000CF911F910F910895EF92FF920F931F930A
:1073D000CF93DF93EC018B017A014AE355E00E94E1
:1073E000103AFA86E986C8016EE375E00E946E3AAB
:1073F000DF91CF911F910F91FF90EF9008950E9420
:10740000293A0895CF93DF93EC0188E165E974E2AE
:107410000E947E43CE010E942C3ADF91CF910895C5
:10742000EF92FF920F931F93CF93DF93EC018B01A9
:107430007A010E944A3AF886EF82C80162E475E058
:107440000E946E3ADF91CF911F910F91FF90EF90C4
:1074500008950E94533A08950E94A1540895DC01B2
:107460001796ED91FC9118970190F081E02D099508
:107470000895DC011796ED91FC9118970280F38135
:10748000E02D309709F00995089582E69EE00E946C
:10749000BD3C0895FC017383628382E69EE0BF01D8
:1074A0000E94303D0895BC0182E69EE00E94FB3CB4
:1074B0000895CF93DF93EC0182E69EE00E94C13CE9
:1074C00008C0FC01228133812C173D0721F00E9466
:1074D000673D0097B1F7DF91CF9108950F931F9308
:1074E000CF93DF938B010E94593AEC01009731F062
:1074F0001D830C83C8010E94E4568E83DF91CF91D7
:107500001F910F9108951F93CF93DF93EC01162FD6
:10751000888580FF1DC0EC81FD813097C9F0D09334
:10752000650EC093640E82E08887CE0106960995A9
:10753000992787FD909502978230910510F01338B6
:1075400029F4CE01BE010E94AC3A02C081E08887D6
:10755000DF91CF911F910895CF92DF92EF92FF922A
:107560000F931F93CF93DF93EC017B01C090640EC8
:10757000D090650E0091660E1091670EF80103C061
:107580000190F081E02DEC17FD0719F03097C1F75D
:1075900046C0209709F443C08885882309F11886DE
:1075A0000BC0C017D10729F0C80167E8AE010E94DF
:1075B000833AF801008111810115110591F7EC81E1
:1075C000FD81309769F0CE15DF0551F0D093650E3F
:1075D000C093640ECE01069663E840E050E0099542
:1075E000E091660EF091670ECE17DF0791F4888167
:1075F00099819093670E8093660E0DC08081918172
:107600008C179D0729F4888199819183808303C019
:10761000FC01309799F7D092650EC092640EDF910D
:10762000CF911F910F91FF90EF90DF90CF90089531
:107630001F93CF93DF931092680EC091660ED09186
:10764000670E11E00EC08985882341F018871986DE
:10765000CE0162E840E050E00E94833A0990D88170
:10766000C02D209781F7DF91CF911F9108958091D0
:10767000690E982F9F5F9093690E08956091640E34
:107680007091650E0E94AC3A08958AE88093690E65
:1076900010926A0E10926B0E1092670E1092660E88
:1076A0001092650E1092640E08958091680E8823E2
:1076B00011F00E94183B70916B0E772309F455C0AE
:1076C00020916A0E30E0F901EE0FFF1FEE0FFF1F51
:1076D000E20FF31FE459F14F608160930C0F418179
:1076E000528150930E0F40930D0F8381948190939C
:1076F000100F80930F0F2F5F3F4F2F71307020932B
:107700006A0E715070936B0E009741F58091660E72
:107710009091670E18C08091680E882311F00E9426
:10772000183B40910D0F50910E0F8091110F9091C9
:10773000120F60910C0F0E94833AE091110FF091AB
:10774000120F808191819093120F8093110F80917D
:10775000110F9091120F0097F1F607C0613819F4DC
:1077600021E0FC0120870E94833A8091680E2091DD
:107770006B0E90E0820F911D08958091680E20910C
:107780006B0E90E0820F911D08959C0170916B0E1D
:107790007032D9F080916A0E870F8F718093130F2A
:1077A00090E0FC01EE0FFF1FEE0FFF1FE80FF91F27
:1077B000E459F14F608352834183348323837F5F95
:1077C00070936B0E80E090E0089581E090E0089562
:1077D000CF93DF93C091640ED091650E0E94833ADF
:1077E000D093650EC093640EDF91CF910895FC0194
:1077F000AB019091660E8091670EA92FB82F03C040
:107800000D90BC91A02DAE17BF0791F01097C1F756
:10781000309771F090838183F093670EE093660E4A
:1078200081E0808717821682CF0161E80E94E83BE1
:107830000895FC01009741F080858150823020F44A
:1078400081E081878093680E089521E030E0FC019B
:107850008085882311F420E030E0C9010895CF939A
:10786000DF93EC014A815B818C819D8160E070E057
:107870000E946E772A813B8188819981289FA0018F
:10788000299F500D389F500D11248E819F8160E0FB
:1078900070E00E946E77DF91CF910895DC0112961F
:1078A0002D913C91139780E090E01DC01496ED91CE
:1078B000FC911597E80FF91F4081442399F421E0CA
:1078C00020832D913C911197829FA001839F500DA1
:1078D000929F500D112416968D919C911797840FAD
:1078E000951F089501968217930701F780E090E0B5
:1078F0000895FC0146815781A281B38120E030E0E8
:1079000019C04617570781F4A481B581A20FB31F90
:107910008C91181614F481508C930480F581E02D1D
:10792000E20FF31F8081089580819181480F591FD4
:107930002F5F3F4F2A173B0721F78FEF0895FC0178
:107940004681578164177507A8F0A081B1818281B3
:107950009381A89F9001A99F300DB89F300D1124ED
:10796000240F351F81E090E06217730728F080E054
:1079700090E0089580E090E00895FC01118210826B
:107980000895FC01808191810895FB01208131815E
:10799000FC01318320830895FC018081918100974F
:1079A00011F40895C901FC012081318121153105AF
:1079B000C9F70895DC01ED91FC911197309729F4F6
:1079C0000BC0DF010190F081E02D80819181009753
:1079D000C1F711961C921E92CF010895DC01ED9122
:1079E000FC911197309729F08081918111969C9399
:1079F0008E93CF010895CF93DF93EC01E881F98155
:107A00003097B9F0A0E0B0E002C0DF01FC01808156
:107A10009181E617F70759F4109719F49983888331
:107A200003C011969C938E931182108202C000971E
:107A300061F7DF91CF9108950F931F93CF93DF9359
:107A40008C01EB010E94FB3CF801808191819983BC
:107A50008883D183C083DF91CF911F910F910895C7
:107A60000F931F93CF93DF938C01EB010E94FB3C9C
:107A700019821882C8010E94CC3C009711F4F801C9
:107A800001C0FC01D183C083DF91CF911F910F9181
:107A90000895DC01ED91FC91119780E090E004C025
:107AA00001960190F081E02D3097D1F70895FB0108
:107AB000BA01309719F40E941C3D0895808191818C
:107AC000DA0111969C938E93518340830895009719
:107AD00021F0FC0180819181089580E090E008957B
:107AE0008091140F9091150F009729F41092170FA1
:107AF0001092160F08950E94A94BBC01E091140F3B
:107B0000F091150F4281538180819181480F591F57
:107B1000461B570B0CC08281938120813181820FDB
:107B2000931F861B970B8417950708F4AC010480FC
:107B3000F581E02D309779F7460F571F5093170FB7
:107B40004093160F089580E595E00E94193C089532
:107B5000EF92FF920F931F93CF93DF937C01FC0171
:107B600080819181009729F08A35910509F06DC0D7
:107B70000BC01092150F1092140F8AE590E0F701D8
:107B80009183808381E065C0673859F5A091140F17
:107B9000B091150F04C014960D90BC91A02D1097B4
:107BA00041F316968D919C9117978417950799F339
:107BB000A093140FB093150F0DC086819781841781
:107BC000950739F48481958115969C938E9314972B
:107BD000FD01DF011496ED91FC911597309769F73F
:107BE000CCCF623851F6C091140FD091150F00E040
:107BF00010E028C0CE010E94C95A0097F1F08E8192
:107C00009F8168E8AE010E94C53B0097A1F41F82E6
:107C10001E828C819D810115110521F0F80195834B
:107C2000848304C09093150F8093140F1D821C82CF
:107C30000E94703DD8CF0E94A33D9C818D818E0112
:107C4000C92FD82F2097B1F698CFF7011182108253
:107C500083E0DF91CF911F910F91FF90EF900895F6
:107C6000CF93DF93EC010E94A33D8E819F813091E1
:107C7000140F2091150F009759F0E32FF22F06C033
:107C8000EC17FD0789F00480F581E02D3097C1F7EE
:107C90008091640E9091650E9F838E833C832D832B
:107CA000D093150FC093140F0E94703DDF91CF91B8
:107CB0000895CF93DF93EC010E94A95ACE010E9450
:107CC000303EDF91CF910895CF93DF93EC010E9476
:107CD000B55ACE010E94303EDF91CF910895CF93E7
:107CE000DF93EC010E94BF5ACE010E94303EDF912B
:107CF000CF910895FC0180819181860F971F918318
:107D000080830E94703D089521E030E0FC0186816F
:107D10009781009711F020E030E0C9010895FC013F
:107D20002281338180819181280F391FC9010895F3
:107D3000FC0180819181089581E090E02091140FF1
:107D40003091150F2115310511F480E090E0089570
:107D50008091140F9091150F009729F08091160FC4
:107D60009091170F089580E090E00895CF93DF93EE
:107D7000EC01E091140FF091150F8E179F0741F45D
:107D80008C819D819093150F8093140F14C0FC017A
:107D9000309731F0848195818C179D07C1F707C01A
:107DA0001D821C821F821E82DF91CF9108958C81DB
:107DB0009D81958384830E94703DF2CFEF92FF9264
:107DC0000F931F93CF93DF937C018A01FC01808185
:107DD0009181009729F08B34910509F049C01AC0B0
:107DE00089E19FE00E94C13CEC0109C06C817D816A
:107DF000CE0102960E94593E0990D881C02D20974D
:107E0000A9F781E08093180F8BE490E0F70191834C
:107E1000808333C0683889F589E19FE00E94C13CC6
:107E2000EC0123C0CE01029608171907D9F489E1A5
:107E30009FE0BE010E94FB3C0091640E1091650E14
:107E40008A859B859093650E8093640EEC85FD85F5
:107E5000309719F08E859F8509951093650E0093D4
:107E6000640ED2CF0990D881C02D2097D9F6CCCFFF
:107E7000F7011182108283E001C081E0DF91CF9190
:107E80001F910F91FF90EF9008951092180F89E1C4
:107E90009FE00E94BD3C89E695E060E070E00E94B2
:107EA000F73B08950F931F93CF93DF93EC0100915D
:107EB000640E1091650E1B870A875D874C873F878C
:107EC0002E878091180F882379F089E695E09093AA
:107ED000650E8093640ECE0102960E94593E109367
:107EE000650E0093640E02C07D836C8389E19FE080
:107EF000BE010E94FB3C89E19FE0BE010E94303D33
:107F0000DF91CF911F910F9108950F931F93CF93FE
:107F1000DF93EC018091180F882391F00091640E9B
:107F20001091650E89E695E09093650E8093640E3E
:107F3000CE0102960E94643E1093650E0093640E7B
:107F400089E19FE0BE010E94FB3C89E19FE0BE0108
:107F50000E94303DDF91CF911F910F9108950F93B3
:107F60001F93CF93DF93EC018091180F882391F03A
:107F70000091640E1091650E89E695E09093650E70
:107F80008093640ECE0102960E946F3E1093650EA0
:107F90000093640E89E19FE0BE010E94FB3C89E1F1
:107FA0009FE0BE010E94303DDF91CF911F910F9164
:107FB0000895CF93DF93EC018091180F882329F067
:107FC000CE0102960E94B63E04C01F821E82198610
:107FD000188689E19FE0BE010E94FB3CDF91CF91B2
:107FE0000895CF93DF93EC018091180F882329F037
:107FF000CE0102960E94843E12C089E19FE00E9459
:10800000C13C06C08C179D0741F0FC018081918125
:108010000097C1F781E090E002C080E090E0DF913E
:10802000CF910895CF93DF93D0919524C09196245A
:108030000E94D54BAB01BC018DB79EB782559040D5
:108040000FB6F8949EBF0FBE8DBFEDB7FEB7319649
:1080500084EF9CE0ADB7BEB712969C938E931197B8
:10806000D2831382C48315824683578360877187C6
:108070008091882690918926A0918A26B0918B269E
:1080800082879387A487B58780918C2690918D26CF
:10809000A0918E26B0918F2686879787A08BB18B73
:1080A0008091902690919126A0919226B09193264E
:1080B000828B938BA48BB58B80919426909195267F
:1080C000A0919626B0919726868B978BA08FB18F23
:1080D0008091982690919926A0919A26B0919B26FE
:1080E000828F938FA48FB58F80919C2690919D262F
:1080F000A0919E26B0919F26868F978FA0A3B1A3B3
:108100008091A0269091A126A091A226B091A326AD
:1081100082A393A3A4A3B5A38091A4269091A5269E
:10812000A091A626B091A72686A397A3A0A7B1A742
:108130008091A8269091A926A091AA26B091AB265D
:1081400082A793A7A4A7B5A78091AC269091AD264E
:10815000A091AE26B091AF2686A797A7A0ABB1ABF2
:108160008091B0269091B126A091B226B091B3260D
:1081700082AB93ABA4ABB5AB8091B4269091B526FE
:10818000A091B626B091B72686AB97ABA0AFB1AFA2
:108190008091B8269091B926A091BA26B091BB26BD
:1081A00082AF93AFA4AFB5AFEDB7FEB7FF968091A6
:1081B000BC269091BD26A091BE26B091BF2680839B
:1081C0009183A283B383EDB7FEB7ED5BFF4F809140
:1081D000C0269091C126A091C226B091C32680836B
:1081E0009183A283B383EDB7FEB7E95BFF4F809124
:1081F000C4269091C526A091C626B091C72680833B
:108200009183A283B383EDB7FEB7E55BFF4F809107
:10821000C8269091C926A091CA26B091CB2680830A
:108220009183A283B383EDB7FEB7E15BFF4F8091EB
:10823000CC269091CD26A091CE26B091CF268083DA
:108240009183A283B3830E94F677D0919524C09145
:1082500096248DB79EB78E5A9F4F0FB6F8949EBF47
:108260000FBE8DBF0E94D54BAB01BC01ADB7BEB7F1
:10827000D2970FB6F894BEBF0FBEADBFEDB7FEB735
:10828000319680ED9DE012969C938E931197D28348
:108290001382C483158246835783608771878091D8
:1082A000D0269091D126A091D226B091D326828754
:1082B0009387A487B5878091D4269091D526A091E5
:1082C000D626B091D72686879787A08BB18B8091D1
:1082D000D8269091D926A091DA26B091DB26828B00
:1082E000938BA48BB58B8091DC269091DD26A09199
:1082F000DE26B091DF26868B978BA08FB18F809181
:10830000E0269091E126A091E226B091E326828FAB
:10831000938FA48FB58F8091E4269091E526A0914C
:10832000E626B091E726868F978FA0A3B1A3809110
:10833000E8269091E926A091EA26B091EB2682A347
:1083400093A3A4A3B5A38091EC269091ED26A091D0
:10835000EE26B091EF2686A397A3A0A7B1A78091A0
:10836000F8269091F926A091FA26B091FB2682A7D3
:1083700093A7A4A7B5A78091FC269091FD26A09174
:10838000FE26B091FF2686A797A7A0ABB1AB0E94AF
:10839000F6778DB79EB7C2960FB6F8949EBF0FBE04
:1083A0008DBFDF91CF91089580E380931F0F0895D3
:1083B000CF93DF9360911F0F70E0C0E3D0E0C61B46
:1083C000D70B6E5D704FAE010E946577CE01DF91D5
:1083D000CF910895CF92DF92EF92FF920F931F9368
:1083E000CF93DF937C01C0901D0FD0901E0F609142
:1083F0001F0F70E08601005D1F4F061B170B013831
:108400001105D8F4C0E3D0E0C61BD70B6E5D704FEA
:10841000AE010E946577C7018C0F9D1F6091200FF0
:108420007091210F20911B0F30911C0F620F731F51
:10843000A6010E946577C80102C080E090E0DF914C
:10844000CF911F910F91FF90EF90DF90CF90089503
:1084500090911F0F980F90931F0F089540911D0F3B
:1084600050911E0F9C014817590798F080911B0FDF
:1084700090911C0F820F931F90931C0F80931B0FE2
:10848000421B530B50931E0F40931D0F81E090E051
:10849000089580E090E0089590931E0F80931D0F43
:1084A000089580911B0F90911C0F8E5A904F089544
:1084B00080911F0F90E08E5D904F089581E090E0D5
:1084C0002091200F3091210F4FE02235340711F415
:1084D00080E090E008950E945E42009769F082E596
:1084E0009FE06091200F7091210F40911D0F5091DE
:1084F0001E0F0E946577089540911B0F50911C0F2D
:1085000041155105C1F080911D0F90911E0FC0962D
:10851000A2E5BFE020E330E007C0FD01E40FF51F56
:1085200060816D932F5F3F4F28173907B4F3109286
:108530001C0F10921B0F08958091200F9091210F16
:10854000089580911D0F90911E0F089590911F0F17
:1085500080E3891B089520E380911F0F281B8091E1
:108560001D0F90911E0F820F911D08951F93CF93A1
:10857000DF93EC0110911F0F812F90E08C179D0766
:108580006CF00E94AB428C0F9D1F8138910530F436
:108590001C1B10931F0F81E090E002C080E090E070
:1085A000DF91CF911F910895CF93DF93EFE9F4E22C
:1085B0001192119284E2EF3CF807D1F7C0E0D0E0CD
:1085C000CE01880F991F89569B4D68E375E00E9484
:1085D00093392196C430D10599F7DF91CF91089551
:1085E00010921C0F10921B0F10921E0F10921D0F55
:1085F00080E380931F0F82E59FE09093210F80938B
:10860000200F0E94D44208950F931F93CF93DF93BE
:10861000EC018B010E94F042D093210FC093200FF8
:1086200010931E0F00931D0FDF91CF911F910F919B
:108630000895EF92FF920F931F93CF93DF9300D093
:10864000CDB7DEB78C0169837A830E94F0426981DD
:10865000E62E7A81F72E81E8E816F10418F030E86A
:10866000E32EF12C8091200F9091210FB801A701EA
:108670000E946577F0921E0FE0921D0FC7010F90C8
:108680000F90DF91CF911F910F91FF90EF90089580
:10869000FC01AFE9B4E280E30D9001928150E1F773
:1086A000FB01A7E9B4E288E00D9001928150E1F767
:1086B0000895AFE9B4E2FC0180E301900D9281508E
:1086C000E1F7A7E9B4E2FB0188E001900D92815047
:1086D000E1F70895E82FF0E0EE0FFF1FE156FB4DA4
:1086E0007183608381E090E00895E82FF0E0EE0F61
:1086F000FF1FE156FB4D80819181089590E0880F26
:10870000991F89599B4D0E94933981E090E008950B
:1087100090E0880F991F89599B4D08958115910507
:1087200011F00197F1F70895E091D224F091D3244C
:1087300090818091D12489230895E091CF24F091F4
:10874000D02480819091D124892B8083E091D424FE
:10875000F091D52480819091D124892B8083089534
:10876000E091CF24F091D02490818091D124809504
:1087700089238083E091D424F091D5249081809145
:10878000D12480958923808308951F93CF93DF930D
:10879000E091CF24F091D02490818091D1248095D4
:1087A00089238083E091D424F091D5248081909115
:1087B000D124892B80838FEB93E00E948E431FB7D7
:1087C000F894E091D424F091D52490818091D12423
:1087D00080958923808383E890E00E948E43E09116
:1087E000D224F091D324D081C091D1241FBF78949A
:1087F0008BE393E00E948E43E091D224F091D32446
:1088000080819091D124892319F08D2F8C2301C070
:1088100081E0DF91CF911F9108955093D52440932B
:10882000D4247093D0246093CF249093D324809346
:10883000D22481E090E002C0880F991F2A95E2F7C8
:108840008093D1240E94C5430895CF93DF93C82F0E
:10885000DFB7F894E091D424F091D52480819091F1
:10886000D124892B808383E090E00E948E43CC2327
:1088700051F0E091D424F091D52490818091D124BD
:1088800080958923808387E190E00E948E43E09168
:10889000D224F091D32480819091D124892309F4AA
:1088A000C0E089E590E00E948E43E091D424F091ED
:1088B000D52490818091D124809589238083DFBF46
:1088C0008BE390E00E948E438C2FDF91CF9108952F
:1088D000CF93DF93C82FD8E08C2F81700E9425445E
:1088E000C6958111C068D150B9F78C2FDF91CF9117
:1088F00008958FEF0E9468440895DF92EF92FF92EF
:108900000F931F93CF93DF93182FEB010E94C54362
:10891000882381F580EF0E946844EE2400E498E00B
:10892000D92E81E00E942544F82E81E00E94254442
:10893000882319F0FF2069F020C0FF2051F40117AF
:1089400028F0888180FF05C0101719F0E02EFF2461
:10895000F3948F2D0E942544888186958883FF207B
:1089600011F0806888830150DA94D9F621960023AB
:10897000B1F605C0EE24EA9402C08EEFE82E8E2DEB
:10898000DF91CF911F910F91FF90EF90DF900895AD
:108990000F931F93CF93DF93182FEB010E94C543D2
:1089A000209751F085E50E94684408E089910E9473
:1089B00068440150D9F703C08CEC0E946844812FB1
:1089C0000E946844DF91CF911F910F9108950F93FA
:1089D0001F93CF93DF93E82FDB01EA01B9014C919C
:1089E00050E011969C91119780E0482B592BE03173
:1089F00081F4CA018E7F33E0880F991F3A95E1F721
:108A000016962C9116974CE050E0421B5109480FE6
:108A1000591F57FF06C081E08883509541955F4FED
:108A200001C01882E83299F414968C91149790E062
:108A30009C01207630702036310549F086FF02C057
:108A40004E7F05C085FF02C04C7F01C0487FCA0130
:108A500024E0969587952A95E1F7FB0180834F7076
:108A6000F801408380E0DF91CF911F910F9108952D
:108A70000F931F93CF93DF93EC018B018881B80193
:108A80000E947D44888381508D3F30F4F8018081BD
:108A9000883211F0803191F7DF91CF911F910F91C2
:108AA0000895CF93DF93EC010E94C54384EBBE0190
:108AB0000E94C84481E00E942544C82F0E94C543FB
:108AC00081E0CC2309F480E0DF91CF9108951F93DA
:108AD000CF93DF93182FEB010E94C5430E9494436C
:108AE000882349F084E4BE010E94C844113029F073
:108AF0000E949D4302C082E001C080E0DF91CF91DF
:108B00001F9108956F927F928F929F92BF92CF9202
:108B1000DF92EF92FF920F931F93CF93DF93CDB726
:108B2000DEB729970FB6F894DEBF0FBECDBF7C012C
:108B30004B013A0169010E94C5438EEBB7010E94C7
:108B4000C8448E010F5F1F4FE9E0BE2E0E9479449A
:108B5000F80181938F01BA94C9F7CE01019669E0BB
:108B600070E00E94635F882361F4F7018081BE0199
:108B70006F5F7F4FA401930186010E94E74480E06C
:108B800001C083E029960FB6F894DEBF0FBECDBFBB
:108B9000DF91CF911F910F91FF90EF90DF90CF90D9
:108BA000BF909F908F907F906F9008958F929F922B
:108BB000AF92BF92CF92DF92EF92FF920F931F93EB
:108BC000CF93DF93CDB7DEB729970FB6F894DEBF0A
:108BD0000FBECDBFD82E5B014A0179018EEB60E05C
:108BE00070E00E94C8448E010F5F1F4FF9E0CF2E46
:108BF0000E947944F80181938F01CA94C9F7CE018C
:108C0000019669E070E00E94635F882359F48D2D1E
:108C1000BE016F5F7F4FA501940187010E94E74469
:108C200080E001C083E029960FB6F894DEBF0FBE46
:108C3000CDBFDF91CF911F910F91FF90EF90DF900B
:108C4000CF90BF90AF909F908F900895EF92FF923A
:108C50001F93CF93DF93CDB7DEB728970FB6F89465
:108C6000DEBF0FBECDBF182F262FDE011196E3E722
:108C7000F5E088E001900D928150E1F7E42EFF24A9
:108C8000E7FCF09441E752E0E49EC001E59E900DC0
:108C9000F49E900D112464E670E00E942674CB01CE
:108CA00034E6239F90011124820F931FFE01319619
:108CB00040E0219130E0E216F30611F4019603C082
:108CC0004F5F4830B1F7112319F0909581959F4F70
:108CD00028960FB6F894DEBF0FBECDBFDF91CF91BF
:108CE0001F91FF90EF9008950F931F93CF93DF9301
:108CF000CDB7DEB72B970FB6F894DEBF0FBECDBF52
:108D0000182F092F885F612F792F0E9467458823CC
:108D100009F048C066E471E48FE090E00E94DF460D
:108D2000812F902FBE016D5F7F4FAE014E5F5F4F71
:108D30009E012F5F3F4F0E948245882399F5DE01F7
:108D40001496E3E7F5E088E001900D928150E1F799
:108D5000E9814E2F50E021E732E0429FC001439F5E
:108D6000900D529F900D112464E670E00E942674CD
:108D7000CB013A8124E6329F90011124820F931F88
:108D8000DE01149620E03D91E31711F4019603C033
:108D90002F5F2830C1F72B81222331F090958195E8
:108DA0009F4F02C084E391E22B960FB6F894DEBF8A
:108DB0000FBECDBFDF91CF911F910F910895DC01C0
:108DC000CB0181159105A105B10529F08150904095
:108DD000A040B040D9F708951092B90080E2809386
:108DE000B800089594EA9093BC0040EA56E861E028
:108DF00070E005C04150504060407040F1F09091EB
:108E0000BC0097FFF7CF1DC09031B9F48093BB0031
:108E100084E88093BC0080EA96E8A1E0B0E004C05A
:108E20000197A109B10959F02091BC0027FFF8CFA3
:108E30000EC081E0903421F40FC081E0089581E0FC
:108E400008959091B900987F9830F1F6DFCF909116
:108E5000B900987F983169F780E0089544EA34E8D2
:108E600024E94093BC009091BC0097FFFCCF909107
:108E7000B900987F983011F0903199F78093BB003A
:108E80003093BC009091BC0097FFFCCF9091B9004B
:108E9000987F903211F0983539F42093BC0090916E
:108EA000BC0094FDFCCFDDCF08950E94F2460895EA
:108EB00084E98093BC008091BC0084FDFCCF0895C0
:108EC0008093BB0084E88093BC008091BC0087FF46
:108ED000FCCF9091B900987F81E0983209F480E04E
:108EE000089584EC8093BC008091BC0087FFFCCF88
:108EF0008091BB00089584E88093BC008091BC0001
:108F000087FFFCCF8091BB000895FC0180E1919127
:108F100090933F018150D9F780913C018F7D8093E0
:108F20003C0180913C01877F80933C01FB0180E103
:108F3000919190933E018150D9F780913C018068D6
:108F400080933C0180913D0180FFFCCF4051504017
:108F500080913C01806280933C0180913C01877F3D
:108F600080933C0112C0FB0180E1919190933E01FE
:108F70008150D9F780913C01806880933C018091B9
:108F80003D0180FFFCCF40515040141615065CF3A4
:108F9000F90180E190913E0191938150D9F781E0F0
:108FA00090E008950F931F93CF93DF938C018CE78C
:108FB0000E942E478CE70E946047C0E1D0E0F80194
:108FC00081918F010E9460472197C9F70E945847FD
:108FD000DF91CF911F910F910895813039F48CE783
:108FE00090E060E070E040E050E006C08CE790E088
:108FF00060E070E040EC50E00E94C21008958130C3
:1090000039F48CE790E060E070E04EE050E006C09C
:109010008CE790E060E070E048E050E00E94C21011
:1090200008958CE790E060E070E041E050E00E943D
:10903000C2106AE67AE080E090E00E94DF46089580
:109040008CE790E060E070E048E350E00E94C210DE
:109050008CE790E060E070E049E350E00E94C210CD
:109060008CE790E060E070E044E150E00E94C210C4
:109070008CE790E060E070E048E750E00E94C210AA
:109080008CE790E060E070E04EE550E00E94C21096
:109090008CE790E060E070E04DE650E00E94C21086
:1090A0006CE17AE186E090E00E94DF468CE790E098
:1090B00060E070E04CE050E00E94C2108CE790E06D
:1090C00060E070E041E050E00E94C2108CE790E068
:1090D00060E070E046E050E00E94C2106AE67AE08C
:1090E00080E090E00E94DF460895CF93DF93CDB7F4
:1090F000DEB7A2970FB6F894DEBF0FBECDBFDE017C
:109100005296EBE7F5E081E101900D928150E1F795
:10911000DE011196ECE8F5E081E101900D928150BD
:10912000E1F70E942048CE0142960E94D24782E099
:109130000E94ED476AE67AE080E090E00E94DF4618
:10914000CE0101960E94D24760E17EEA88E290E07B
:109150000E94DF4680E00E94FF4760E17EEA88E2ED
:1091600090E00E94DF4681E00E94FF47A2960FB682
:10917000F894DEBF0FBECDBFDF91CF910895E6E436
:10918000F1E080812081908130818295869586955D
:10919000837022952F70822B832B92959F70892B41
:1091A0000895DF92EF92FF920F931F93CF93DF9377
:1091B00000D0CDB7DEB780E06CE046E00E946D4C99
:1091C00089E18093C4001092C50082E08093C000C2
:1091D00080E00E940F4D0E94994B84B784B784B7FA
:1091E00084B784B7E6E5FDE222E432E431832083EC
:1091F0003A968DB79EB70A97E817F907B8F300D0EB
:1092000000D08FE39EE0ADB7BEB712969C938E93CD
:1092100011978DE995E014969C938E9313970E9475
:10922000F6770F900F900F900F900E94945B0E9422
:10923000453B80E595E060E070E00E94F73B0E94CE
:10924000453FE091E805F091E90509950E94BF4886
:1092500090E00E94D15BCE0101960E94CB4A882308
:1092600059F000D08AE59EE0EDB7FEB79283818386
:109270000E94F6770F900F90CE0101960E94AE39B2
:109280000E94D54A8C010E94DA4ABC01C801AE0195
:109290004F5F5F4F0E9409500E94384A0E94EE4F74
:1092A0000E94DF4A0E948A5100D08AE79EE0ADB753
:1092B000BEB712969C938E9311970E94F67700D0BA
:1092C000EDB7FEB7319607E81EE0ADB7BEB7129610
:1092D0001C930E9311978A81828313820E94F677E2
:1092E000EDB7FEB73196ADB7BEB712961C930E938D
:1092F00011978981828313820E94F6770F900F90D5
:109300008BE89EE0EDB7FEB7928381830E94F677EB
:109310000F900F900E94D75BE0916B06F0916C0666
:109320000995E0915206F09153060995E0911406D3
:10933000F091150609950091500610915106E090A4
:109340006906F0906A060E94EB4FD82E0E94925157
:109350002DB73EB72A5030400FB6F8943EBF0FBE2F
:109360002DBFEDB7FEB731962DE83EE0ADB7BEB7E5
:1093700012963C932E93119713830283F582E48215
:10938000D6821782808711860E94F677E091750653
:10939000F09176062DB73EB7265F3F4F0FB6F89493
:1093A0003EBF0FBE2DBF3097D1F00995BC0100D054
:1093B00000D088EA9EE0ADB7BEB712969C938E931C
:1093C000119780E890E00E941274EDB7FEB77483A5
:1093D00063830E94F6770F900F900F900F9000D04C
:1093E0008BEB9EE0ADB7BEB712969C938E93119710
:1093F0000E94F6770F900F9084E996E060E070E0AD
:109400000E94F73B86E794E00E948D5A00D08DEBD6
:109410009EE0EDB7FEB7928381830E94F6770F90AE
:109420000F900F900F90DF91CF911F910F91FF90B0
:10943000EF90DF90089500D000D000D0EDB7FEB7D8
:10944000319625EC3EE0ADB7BEB712963C932E9315
:10945000119793838283758364830E94F6778DB717
:109460009EB706960FB6F8949EBF0FBE8DBF0895A7
:109470000F931F93CF93DF93CDB7DEB7A0970FB6AF
:10948000F894DEBF0FBECDBF83E290E00E94367934
:10949000082F282F2B50203108F0982F90958917EE
:1094A00009F46DC000D08BEE9EE0ADB7BEB712964A
:1094B0009C938E9311970E94F6778E010F5F1F4F3A
:1094C0000F900F90D80180E090E0FC01ED51F14F3A
:1094D000E491ED93019688309105B9F7F894CE01A7
:1094E00001966FE370E048E050E00E943C79D801BB
:1094F00080E090E0FC01EB52F14FE491ED93019696
:109500008E309105B9F7CE01019661E370E04EE02F
:1095100050E00E943C7980E090E0FC01E553F14F7F
:10952000E491D801ED938D0101968A309105A9F758
:10953000CE01019667E270E04AE050E00E943C797B
:1095400081E290E06DEC7BEA0E9454798FE190E03B
:1095500060E070E00E9454798EE190E060E00E944B
:10956000467985E290E060E070E00E9454790AE17B
:1095700083E290E06AE175EE0E9454797894802F3E
:10958000A0960FB6F894DEBF0FBECDBFDF91CF918E
:109590001F910F910895F8946FE370E042E050E05E
:1095A0000E941E79789480E0089581E290E00E9404
:1095B000367908958FE190E00E94367908958EE122
:1095C00090E00E942E7908954091E4245091E52482
:1095D0006091E6247091E72490E0A0E0B0E0480FAD
:1095E000591F6A1F7B1F4093E4245093E524609326
:1095F000E6247093E7244091E0245091E1246091A7
:10960000E2247091E324480F591F6A1F7B1F409387
:10961000E0245093E1246093E2247093E3242091AA
:1096200084262223A1F04091DC245091DD24609116
:10963000DE247091DF24480F591F6A1F7B1F40935F
:10964000DC245093DD246093DE247093DF2408959E
:109650001F920F920FB60F920BB60F9211242F93F9
:109660003F934F935F936F937F938F939F93AF93AA
:10967000BF93EF93FF938091D60F9091D70F0196F0
:109680009093D70F8093D60F8091D50F8F5F8093E3
:10969000D50F8038A9F41092D50F8091E4249091D1
:1096A000E524A091E624B091E7240196A11DB11D07
:1096B0008093E4249093E524A093E624B093E724D8
:1096C000809184268823E1F08091D40F8F5F80936E
:1096D000D40F8038A9F41092D40F8091DC2490919B
:1096E000DD24A091DE24B091DF240196A11DB11DDF
:1096F0008093DC249093DD24A093DE24B093DF24B8
:109700000E949C3E009711F00E94A33DFF91EF91B3
:10971000BF91AF919F918F917F916F915F914F9189
:109720003F912F910F900BBE0F900FBE0F901F9087
:109730001895F8941092B60016BC83EF87BD82E0AE
:1097400084BD94E095BD95B395BB80936E007894ED
:1097500008958091D60F9091D70F2091D60F309118
:10976000D70F82179307A9F7089507C022E330E0C7
:10977000000021503040E1F701970097B9F70895B4
:109780000F931F93CF93DF938C010E94A94BEC01A1
:109790000E94A94B8C1B9D0B80179107C8F3DF918A
:1097A000CF911F910F91089508950F931F930091EA
:1097B000E4241091E5242091E6243091E72480915F
:1097C000E4249091E524A091E624B091E7240817C1
:1097D00019072A073B0759F7B801C9011F910F91D3
:1097E00008951F920F920FB60F9211241092B30595
:1097F0000F900FBE0F901F9018951F920F920FB6EB
:109800000F920BB60F9211242F933F934F935F93B8
:109810006F937F938F939F93AF93BF93EF93FF9338
:10982000E091A905F091AA058081E091B405F0913D
:10983000B505309709F00995FF91EF91BF91AF9170
:109840009F918F917F916F915F914F913F912F9158
:109850000F900BBE0F900FBE0F901F9018951F9288
:109860000F920FB60F9211241092C0050F900FBEE9
:109870000F901F9018951F920F920FB60F920BB674
:109880000F9211242F933F934F935F936F937F9386
:109890008F939F93AF93BF93EF93FF93E091B605A0
:1098A000F091B7058081E091C105F091C205309734
:1098B00009F00995FF91EF91BF91AF919F918F9121
:1098C0007F916F915F914F913F912F910F900BBEC0
:1098D0000F900FBE0F901F90189590E02DE030E094
:1098E000829FF001839FF00D929FF00D1124E755A8
:1098F000FA4FA281B3811C92A481B5816C93A68199
:10990000B78188ED8C93A085B1854C93128614861F
:109910001386089590E02DE030E0829FF001839F50
:10992000F00D929FF00D1124E755FA4F81E08287E8
:10993000A081B1816C933A9680818823E9F70895DC
:10994000CF93C82F8A3031F4809118106DE00E94B7
:109950008A4C02C08D3029F0809118106C2F0E9423
:109960008A4C80E090E0CF9108951F93CF93DF93CE
:10997000182FEB010CC08A3021F4812F6DE00E947A
:109980008A4C69916D3019F0812F0E948A4C888130
:10999000882389F7DF91CF911F9108950F931F932B
:1099A000CF93DF93CDB7DEB79E01265F3F4F08ED23
:1099B0001FE0C80160E470E0488559850E948878FE
:1099C0008F81B8010E94B54CDF91CF911F910F910B
:1099D00008951F93CF93DF93182FEB0104C0812FBD
:1099E0000E948A4C2196FE0164916623C1F7DF91A3
:1099F000CF911F91089590E02DE030E0829FF0011B
:109A0000839FF00D929FF00D1124E755FA4F748754
:109A100063870895682F80E00E948A4C08958093A0
:109A2000181083EC95E09093512D8093502D08955C
:109A300084B7877F84BF88E10FB6F8948093600075
:109A4000109260000FBE08952FE088E190E00FB6FD
:109A5000F894A895809360000FBE2093600008954D
:109A6000A895089588E10FB6F8948093600010924D
:109A700060000FBE0895F89428E088E190E00FB6EA
:109A8000F894A895809360000FBE20936000FFCFEC
:109A90008091EF248091EF2490E008958091390126
:109AA00081FD10C081E491E06FE140E00E94295304
:109AB000813059F021E030E0813111F020E030E0D8
:109AC000C901089580E090E0089581E090E0089554
:109AD00081E491E06FE140E00E9429530895E9E3B9
:109AE000F1E0808180818D7F80838DE090E001971F
:109AF000F1F782E491E06FE140E023E00E9433530C
:109B000083E090E00197F1F708959091390191FD7C
:109B10000AC0282F803108F02FE085E491E06FE043
:109B200040E00E94335308958091390181FD13C0B4
:109B300081E491E06FE140E00E942953982F815128
:109B4000823038F09F3129F0913019F081E0923065
:109B500019F480E0089581E008950E94944D8823CF
:109B6000E1F30895CF93DF93C82F883049F0863012
:109B700039F0893029F0863119F0893109F045C072
:109B80008091390181FD44C00E94AD4D0E94684D15
:109B9000D82FC817B9F1C83019F40E946F4D2BC0E7
:109BA000C93141F48631A9F482E491E06FE140E0EB
:109BB00029E009C0C63169F4893159F482E491E0A1
:109BC0006FE140E026E00E943353E3E0F0E031979C
:109BD000F1F782E491E06FE140E02C2F0E943353D3
:109BE000D83029F489E691E00197F1F704C0E3E069
:109BF000F0E03197F1F70E94684D8C1719F083E47B
:109C000090E008C080E490E005C082E490E002C0EB
:109C100084E490E0DF91CF91089580919400909139
:109C2000950090931D2780931C2721E020930927FE
:109C30008091390181FF15C0209383268091940083
:109C400090919500909319278093182720930727C8
:109C5000809139018D7F80933901809183268823FB
:109C6000E1F786E10E94B24D81E080938426089559
:109C700080918426882351F480911A10882321F042
:109C800081E080939C1002C00E940D4E81E090E024
:109C900008950E94AD4D109284260E946F4D8091D0
:109CA0003901826080933901809107278823E9F187
:109CB0008091940090919500209118273091192758
:109CC00082179307A0F48091E4269091E526A09155
:109CD000E626B091E7268C57914EAF4FBF4F809349
:109CE000E4269093E526A093E626B093E72680919C
:109CF000940090919500821B930BA0E0B0E04091FE
:109D0000E4265091E5266091E6267091E726840FBF
:109D1000951FA61FB71F8093E4269093E526A09376
:109D2000E626B093E726109207278091092788231B
:109D3000E9F1809194009091950020911C27309139
:109D40001D2782179307A0F48091EC269091ED26B1
:109D5000A091EE26B091EF268C57914EAF4FBF4F9A
:109D60008093EC269093ED26A093EE26B093EF26F9
:109D70008091940090919500821B930BA0E0B0E03D
:109D80004091EC265091ED266091EE267091EF26E1
:109D9000840F951FA61FB71F8093EC269093ED2686
:109DA000A093EE26B093EF26109209270895809194
:109DB0009C10882321F00E940D4E10929C108091DF
:109DC0009D10882321F00E94494E10929D10109200
:109DD0001A1008950F931F93CF93DF93F82FE92F55
:109DE000AB0181E080931A100091C8261091C9261A
:109DF0002091CA263091CB260F5F1F4F2F4F3F4F28
:109E00000093C8261093C9262093CA263093CB26E8
:109E1000862F8E5F87FF0CC08091812690918226CD
:109E200001969093822680938126CFEFDFEF09C0C1
:109E30002BE130E1C9016F2F7E2F0E946577C0E0D2
:109E4000D0E00E94D74ECE01DF91CF911F910F91AC
:109E5000089580918426882399F080911A10882390
:109E600021F40E94944D882331F481E080939D1069
:109E700081E090E008950E94494E80E090E00895CE
:109E800080E090E008951F93CF93DF930F92CDB7BA
:109E9000DEB78FB7898380911A10882331F5F89443
:109EA00080918426882351F08091390181FD1BC067
:109EB0000E94944D8823B9F080E003C00E94384E80
:109EC00081E0909147019E3010F010E001C01FEF3B
:109ED000882311F00E94294F16FF05C089818FBF8A
:109EE00081E090E004C089818FBF80E090E00F9016
:109EF000DF91CF911F9108958093191008950E94CA
:109F0000684D8250813130F4E82FF0E0E450FA4F90
:109F10008081089581E0089508958FEF80934E0128
:109F20008CE691E060EF44E022E00E9433538CE243
:109F300090E06EE041E025E00E94335380E880939A
:109F40006F018091460180936D0184E491E060E2AD
:109F500045E021E00E9433530895CF93DF93CDEF86
:109F6000D3E0CE010197F1F70E941F531092F8241D
:109F700010927A251092FC251092F7241092F62464
:109F8000E9E3F1E080818E7F808380818D7F808313
:109F90008DE090E00197F1F780818160808382E419
:109FA00091E06FE140E023E00E9433532197F1F705
:109FB00080915D0180915E010E948D4F8EED95E054
:109FC00060E070E00E94F73B0E940D4E81E090E05F
:109FD000DF91CF91089580919E100895CF93DF93E4
:109FE0000F92CDB7DEB789830E94AD4D29812093B2
:109FF0009E1088E491E06FE140E00E9433530F909F
:10A00000DF91CF9108950E94EE4F86E00E94B24DFD
:10A010000895FA0180936201909363016093600157
:10A02000709361013097C1F0808180936B018181D1
:10A0300080936A01828180936901838180936801A2
:10A0400084818093670185818093660186818093F6
:10A05000650187818093640108958EED95E00E94EB
:10A06000193C81E08093EF248091F0249091F124B9
:10A0700001969093F1248093F02481E090E008957C
:10A08000CF93DF935091F724252F30E0F901EE0FA5
:10A09000FF1F3695322F222737952795E20FF31FA2
:10A0A000E850FB4D4081442309F4F4C0209139016C
:10A0B00021FDF0C020918426222309F4EBC047FF44
:10A0C00023C0852F90E0FC01EE0FFF1F9695982F7F
:10A0D000882797958795E80FF91FE850FB4D108268
:10A0E0008091B8269091B926A091BA26B091BB264E
:10A0F0000196A11DB11D8093B8269093B926A09317
:10A10000BA26B093BB26C6C0433018F5852F90E021
:10A11000FC01EE0FFF1F9695982F8827979587953E
:10A12000E80FF91FE850FB4D10828091B426909102
:10A13000B526A091B626B091B7260196A11DB11DF6
:10A140008093B4269093B526A093B626B093B726F5
:10A15000A1C0C42FD0E022976C177D0718F5852F7A
:10A1600090E0FC01EE0FFF1F9695982F882797959A
:10A170008795E80FF91FE850FB4D10828091B026BB
:10A180009091B126A091B226B091B3260196A11D5F
:10A19000B11D8093B0269093B126A093B226B093C0
:10A1A000B32678C0252F30E0B901660F771F3695AA
:10A1B000322F222737952795620F731F67507B4DEB
:10A1C00050E00E9465772091F724822F90E0FC01F7
:10A1D000EE0FFF1F9695982F882797958795E80F84
:10A1E000F91FE858FA4D80818093E824822F90E08F
:10A1F000FC01EE0FFF1F9695982F8827979587955E
:10A20000E80FF91FE850FB4D10822F5F2093F724D1
:10A21000233010F01092F7248091F72490E0FC0195
:10A22000EE0FFF1F9695982F882797958795E80F33
:10A23000F91FE850FB4D8081882311F00E942D50BA
:10A24000609147016093E9248091EE24882311F006
:10A25000681710F46093EE2484E070E00E946A4373
:10A260006091E82483E070E00E946A438091CC26EC
:10A270009091CD26A091CE26B091CF260196A11D1A
:10A28000B11D8093CC269093CD26A093CE26B0937B
:10A29000CF2602C0C0E0D0E0CE01DF91CF9108957B
:10A2A000CF93DF93EC0188819981009729F024E016
:10A2B0008B3F920739F505C08BEF94E09983888333
:10A2C00025C0623819F51092EF240E94F0420E94D6
:10A2D000514260E870E00E9440501816190644F49C
:10A2E0000E944C42E0916F06F09170060995E4CF10
:10A2F0008091EC249091ED2401969093ED2480932D
:10A30000EC24DACF1982188283E001C081E0DF916A
:10A31000CF91089591E090931A100E94854D0E946C
:10A32000D74E08958091390181FD07C085E491E001
:10A330006FE040E00E942953089580E108950F9353
:10A340001F93CF93DF93C82F21E020931A10D09151
:10A3500084268091390181FF16C0809194009091EC
:10A36000950090931927809318272093072720930F
:10A370008326809139018D7F8093390180918326D6
:10A380008823E1F7D0E00E94AD4D80918426882398
:10A3900009F441C0809109278823E9F18091940054
:10A3A0009091950020911C2730911D2782179307CB
:10A3B000A0F48091EC269091ED26A091EE26B0912C
:10A3C000EF268C57914EAF4FBF4F8093EC26909362
:10A3D000ED26A093EE26B093EF2680919400909105
:10A3E0009500821B930BA0E0B0E04091EC265091C9
:10A3F000ED266091EE267091EF26840F951FA61F23
:10A40000B71F8093EC269093ED26A093EE26B09391
:10A41000EF261092092789E10E94B24D86E00E9442
:10A420007543009751F00E949251082F86E00E94D8
:10A43000754381500E94854D02C000E010E080917C
:10A4400094009091950090931B2780931A2781E0A8
:10A4500080930827F89480913901826080933901B4
:10A46000809139018D7F809339016C2F6E5F8BE174
:10A4700090E10E946453789480917E2690917F268B
:10A48000019690937F2680937E260E94AD4D82E4B4
:10A4900091E060EE45E00E942953C82F86E00E94BB
:10A4A0007543009719F0802F0E94854DDD2319F028
:10A4B0000E940D4E02C00E94494E809108278823B9
:10A4C000E9F1809194009091950020911A273091A4
:10A4D0001B2782179307A0F48091E8269091E92624
:10A4E000A091EA26B091EB268C57914EAF4FBF4F0B
:10A4F0008093E8269093E926A093EA26B093EB2672
:10A500008091940090919500821B930BA0E0B0E0A5
:10A510004091E8265091E9266091EA267091EB2659
:10A52000840F951FA61FB71F8093E8269093E926F6
:10A53000A093EA26B093EB261092082780918426F8
:10A54000882361F0809194009091950090931D274D
:10A5500080931C2781E08093092707C082E491E063
:10A560006FE140E023E00E9433530E94D74EC13098
:10A57000E1F0C330A9F48091C0269091C126A0914A
:10A58000C226B091C3260196A11DB11D8093C0269D
:10A590009093C126A093C226B093C326C2E00AC0FE
:10A5A000C53029F0C73031F404C0C0E003C0C3E0B7
:10A5B00001C0C1E08C2F90E0DF91CF911F910F91EE
:10A5C0000895CF93DF93EB010E94EA4E009729F4A0
:10A5D000CE010E949F51009751F020918126309129
:10A5E00082262F5F3F4F3093822620938126DF9172
:10A5F000CF910895CF93DF9380918426882321F40F
:10A600000E94384EC1E001C0C0E00E94684D863112
:10A6100011F0813119F4D091470109C086E491E02D
:10A620006FE140E00E942953D82FDD0FD80FCC23D3
:10A6300011F00E94294F8D2FDF91CF910895109234
:10A64000A01010929F10EFE6F0E08081806280837E
:10A650000895FC018081862390E002C0959587953E
:10A660004A95E2F70895F894FC019081862F809531
:10A67000892330E002C0220F331F4A95E2F72623D8
:10A68000282B208378940895CF93DF93EC012196B3
:10A69000E0917B01DC01EC932E2FA0E8B1E03D912D
:10A6A00039932150E1F7E150F0E0E058FE4F21816D
:10A6B000FC01E058FF4F20838F579F4F21E0FC01A2
:10A6C0002083DF91CF910895FC0160938001A1E880
:10A6D000B1E0615881918D936A17E1F708951F9257
:10A6E0000F920FB60F920BB60F9211242F933F9338
:10A6F0004F935F936F937F938F939F93AF93BF938A
:10A70000EF93FF93809147018093E9242091F624F1
:10A7100030E0C901880F991F3695322F22273795CF
:10A720002795820F931F88509B4D0E944453809120
:10A73000F6248F5F8093F624833010F01092F62475
:10A740000E942D50FF91EF91BF91AF919F918F91FA
:10A750007F916F915F914F913F912F910F900BBE21
:10A760000F900FBE0F901F9018951F920F920FB66B
:10A770000F9211240F900FBE0F901F9018951F92EB
:10A780000F920FB60F9211240F900FBE0F901F90D3
:10A7900018951F920F920FB60F9211240F900FBEB3
:10A7A0000F901F9018951F920F920FB60F921124C1
:10A7B000109283260F900FBE0F901F9018951F9236
:10A7C0000F920FB60F921124109283260F900FBE96
:10A7D0000F901F9018951F920F920FB60F92112491
:10A7E0008F9381E08093EF248F910F900FBE0F9095
:10A7F0001F9018951F920F920FB60F92112410926E
:10A8000083260F900FBE0F901F9018951F920F92E6
:10A810000FB60F9211248F939F9380919F10909168
:10A82000A01001969093A01080939F109F918F91FC
:10A830000F900FBE0F901F9018950F931F93CF93FB
:10A84000DF9380918C2690918D26A0918E26B091D9
:10A850008F260196A11DB11D80938C2690938D2685
:10A86000A0938E26B0938F260E94B5568C0181EA64
:10A8700090E10E94C13C08C0EA81FB81309709F059
:10A880000995CE010E94673DEC010097A9F70115DB
:10A89000110519F0C8010E942F3ADF91CF911F9145
:10A8A0000F9108950E94D75B0E94F0420E94CE54FF
:10A8B00080E596E090938726809386260E94B25684
:10A8C00082E090E060E074E040E05EE12FEF31E094
:10A8D0000E9473560895CF92DF92EF92FF920F93EA
:10A8E0001F93CF93DF936C018B017A0181EA90E192
:10A8F0000E94C13C09C0EC81FD81309711F0C80174
:10A900000995CE010E94673DEC010097A1F7C601B1
:10A91000B801A7010E94393ADF91CF911F910F91A1
:10A92000FF90EF90DF90CF900895BC0181EA90E115
:10A930000E94303D0895BC0181EA90E10E94FB3CF9
:10A940000895CF93DF93EC0180918826909189261A
:10A95000A0918A26B0918B260196A11DB11D8093EE
:10A96000882690938926A0938A26B0938B26CE01C1
:10A970000E94C856009769F00E946B42E09154060D
:10A98000F09155068BE694E5BE01099581E090E0D3
:10A9900002C080E090E0DF91CF91089583EA90E1DA
:10A9A0000E94BD3C08950F93CF93DF93EC017B830E
:10A9B0006A8318865F834E8383EA90E1BE010E941A
:10A9C000303DE091A510F091A610309749F04C81F0
:10A9D0005D818A819B81688520E030E001E00995F6
:10A9E000DF91CF910F910895BC0183EA90E10E941D
:10A9F000FB3C08950F93DC0118961C921897E09188
:10AA0000A510F091A610309759F012968D919C9157
:10AA1000139760E040E050E020E030E000E009956E
:10AA20000F9108950F93DC01AB0114962D913C9189
:10AA3000159781E018968C93189715967C936E93D2
:10AA40001497E091A510F091A610309739F0129666
:10AA50008D919C91139761E000E009950F91089505
:10AA60000F93DC01E091A510F091A610309769F0EA
:10AA700014962D913C91159712968D919C91139758
:10AA800018966C91A90101E009950F910895E09144
:10AA9000A710F091A810309709F0099508959093A8
:10AAA000A8108093A71008959093A6108093A510E6
:10AAB000089583EA90E10E94C13C0895EF92FF92CD
:10AAC0000F931F93CF93DF938C01EB017A0183EAFD
:10AAD00090E10E94C13C15C0DC0112962D913C9181
:10AAE00013972C173D0759F41696ED91FC91179783
:10AAF000309749F0B801AE019701099504C00E9452
:10AB0000673D009749F7DF91CF911F910F91FF901B
:10AB1000EF9008950895AF92BF92CF92DF92EF9297
:10AB2000FF920F931F93CF93DF9300D0CDB7DEB783
:10AB30005B010E945142FC01E080F180FA82E982CF
:10AB4000FCE0EF16F10418F400E010E02DC000D096
:10AB500000D088E196E0EDB7FEB792838183F4825E
:10AB6000E3820E94E4770F900F900F900F901FC028
:10AB70000E945142F801EE0FFF1FEE0FFF1FE80F7A
:10AB8000F91FC280D3800E9451420F5F1F4FF8010E
:10AB9000EE0FFF1FEE0FFF1FE80FF91F40815181DD
:10ABA000C501B6010E945E550E151F0509F70F90ED
:10ABB0000F90DF91CF911F910F91FF90EF90DF9059
:10ABC000CF90BF90AF900895CF93DF93C4ECD0E1C6
:10ABD0006091DA107091DB10CE0147E056E520E07D
:10ABE00030E00E94523F0E94D45B6091DA10709175
:10ABF000DB100E941274BC01CE0140974BE256E577
:10AC000020E030E00E94523FDF91CF910895809183
:10AC1000DA109091DB102091D8103091D910880F64
:10AC2000991F2817390708F4C9019093DB10809306
:10AC3000DA100E94E45508950F93013051F4809189
:10AC4000D4109091D5109093DB108093DA100E946D
:10AC5000E4550F910895CF93DF930E94F0420E9434
:10AC60005142EC01198218820E94595520C0129657
:10AC70002D913C911397FC01EE0FFF1FEE0FFF1F6C
:10AC8000EC0FFD1F3383228314962D913C91159771
:10AC90000196FC01EE0FFF1FEE0FFF1FEC0FFD1FD3
:10ACA0003183208399838883CD010E94673DDC0135
:10ACB00088819981109729F018962C911897222352
:10ACC000B1F6880F991F880F991F02960E944C4277
:10ACD00088819981009721F089EA90E10E94023AE7
:10ACE000DF91CF910895EF92FF920F931F93CF932F
:10ACF000DF93FC018B017A01E90189EA90E1BF0150
:10AD000045E356E00E94E4391093D5100093D41027
:10AD1000F092D710E092D610D093D910C093D810EB
:10AD20008CE196E50E945455DF91CF911F910F91D0
:10AD3000FF90EF900895CF93DF93C4ECD0E1CE0164
:10AD40000E94D93FCE0140970E94D93FCE014B9738
:10AD50000E94FF39DF91CF9108958091DA10909190
:10AD6000DB1008950E94453A0895CF93DF93E09158
:10AD70003906F0913A060995EC01009729F06A81AD
:10AD80007B8181E00E946A43CE01DF91CF910895DB
:10AD90000F931F93CF93DF93EC01E0913B06F0916B
:10ADA0003C0609958C016A817B8181E00E946A439F
:10ADB00081E090E00115110511F480E090E0DF9151
:10ADC000CF911F910F910895E0913D06F0913E06BD
:10ADD000099508959C0180E090E005C0F901319744
:10ADE0004081840F911D2E5F3F4FF90132974081C2
:10ADF0004423A1F70895FC01308120E0818190E097
:10AE0000822B932B02C0880F991F6A95E2F7892F36
:10AE10009927FA01E15CF94F208130E082239323E6
:10AE200028E030E0241B350B02C0969587952A95C3
:10AE3000E2F708956F927F928F929F92AF92BF92A6
:10AE4000CF92DF92EF92FF920F931F93CF93DF93F6
:10AE50005C013B018A0169012830310544F4CB01D2
:10AE6000BA01A9010E94FB56F50180834EC0790109
:10AE700073E0F594E7947A95E1F74115510521F0D7
:10AE80004501C0E0D0E005C0F301D50180E090E0CD
:10AE900021C0C3018C0F9D1FB80148E050E00E9403
:10AEA000FB56F40181934F012196CE15DF058CF3FB
:10AEB000C701F7FE02C080E090E0A6014770507025
:10AEC0004115510511F1E501C80FD91F860D971DD8
:10AED000B80118C021912D9301968E159F05D4F3CA
:10AEE000C701F7FE02C080E090E0A60147705070F5
:10AEF0004115510551F0E501C80FD91F860D971D69
:10AF000060E070E00E94FB568883DF91CF911F9133
:10AF10000F91FF90EF90DF90CF90BF90AF909F90F8
:10AF20008F907F906F9008958F929F92AF92BF9273
:10AF3000CF92DF92EF92FF920F931F93CF93DF9305
:10AF400000D000D0CDB7DEB70E9451428C0182E024
:10AF500090E00E942E42009709F45FC0F8019181B1
:10AF600080E02081820F911D0E94593A7C01009758
:10AF700009F455C00E9451424C01F7018681482FC7
:10AF800046954695469550E090E08770907021E098
:10AF900030E0009711F420E030E0CA01820F931FE7
:10AFA0000E942E420097C9F1F70104811581CC243B
:10AFB000DD242EC0F801A180BB24B601A3E0759565
:10AFC0006795AA95E1F7680D791DA6014770507045
:10AFD000883168F0CE01039695010E941A57F80156
:10AFE0008081BE016D5F7F4F0E947E430DC01A823B
:10AFF0001982CE01019695010E941A5769817A81C2
:10B00000F80180810E946A43CA0CDB1C0E5F1F4F4F
:10B01000F8018081882371F602C0EE24FF24C70165
:10B020000F900F900F900F90DF91CF911F910F9184
:10B03000FF90EF90DF90CF90BF90AF909F908F9058
:10B040000895FC0150E080E190E0861B970B821B85
:10B05000930B02C0440F551F8A95E2F78081852B20
:10B0600080838181842B818308956F927F928F9258
:10B070009F92AF92BF92CF92DF92EF92FF920F9387
:10B080001F93CF93DF933C016B015A017901283064
:10B09000310524F4C301FA01408159C08901B3E0AC
:10B0A00015950795BA95E1F76115710521F04A01EB
:10B0B000C0E0D0E005C0FA01D30180E090E023C0F9
:10B0C000F40141914F01C3018C0F9D1FB60128E08F
:10B0D00030E00E9421582196C017D1078CF39801C7
:10B0E00017FF02C020E030E0D701A770B0701097C2
:10B0F00081F1F501E20FF31F408150E0C6018A1B88
:10B100009B0B089619C021912D93019680179107EA
:10B11000D4F3980117FF02C020E030E0D701A770F8
:10B12000B0701097B1F0F501E20FF31F408150E0CD
:10B1300088E090E08A1B9B0B02C0559547958A9545
:10B14000E2F7C301820F931F60E070E09D010E944F
:10B150002158DF91CF911F910F91FF90EF90DF90D9
:10B16000CF90BF90AF909F908F907F906F900895F9
:10B170006F927F928F929F92AF92BF92CF92DF9207
:10B18000EF92FF920F931F93CF93DF9300D0CDB731
:10B19000DEB77C01DC0116968C911697282F269538
:10B1A0002695269530E090E08770907001E010E0E1
:10B1B000009711F400E010E0020F131FC80102967F
:10B1C0000E94B642009709F451C00E945842FC0107
:10B1D000D70112968C911297808313968C9181835C
:10B1E0000E94584232E0632E712C680E791EC30112
:10B1F00060E070E0A8010E946E77F701E480F580BE
:10B20000CC24DD242CC0D7011196AC901197BB241F
:10B21000860193E0159507959A95E1F7060D171DA0
:10B2200027E0822E912C8C209D20883130F00E94C6
:10B230008843AC01C801B40109C00E9475439A83D8
:10B240008983C801B401AE014F5F5F4F95010E9431
:10B250003558CA0CDB1CE2E0F0E0EE0EFF1ED70111
:10B260008C91882381F681E090E002C080E090E03C
:10B270000F900F90DF91CF911F910F91FF90EF9062
:10B28000DF90CF90BF90AF909F908F907F906F9006
:10B290000895E0916D06F0916E0609950895E0918C
:10B2A0001606F091170609950895E0917106F09140
:10B2B000720609950895E0917306F0917406099558
:10B2C000089580E090E008950895E091F805F091E8
:10B2D000F9050995089580E090E008950F931F9374
:10B2E000CF93DF93CDB7DEB7E0970FB6F894DEBF0C
:10B2F0000FBECDBF0E94A1428C010E945142602F1F
:10B30000AE014F5F5F4F0E946461882309F446C01D
:10B3100088A99801281B3109C9010E942E42009773
:10B32000E9F12E81222379F18A859B853BEA8D3CC8
:10B33000930721F03FEF8F3F930781F5223069F0AB
:10B3400088E090E00197E1E0F0E0EC0FFD1FE80FEE
:10B35000F91F23852F3F21F007C082E090E0F2CF54
:10B36000181619067CF30FC089E1BE01645F7F4F98
:10B370000E947E4389E10E94884365E974E20E944D
:10B380009C39009759F088E1BE016A5E7F4F0E94A8
:10B390007E43E0915606F09157060995E0960FB668
:10B3A000F894DEBF0FBECDBFDF91CF911F910F91FB
:10B3B0000895AF92BF92CF92DF92EF92FF920F93D8
:10B3C0001F93CF93DF93CDB7DEB7E0970FB6F89416
:10B3D000DEBF0FBECDBF5C016B01FE01319680E385
:10B3E000DF011D928A95E9F781E089838CE00E9454
:10B3F00075438C831D821F828091DE1089878F5F49
:10B400008093DE1003E008878DEC9BEA9B878A8798
:10B4100089E10E94884368E375E00E949C390097A7
:10B4200031F082E08E838FEF8C878D8709C089E1B0
:10B430000E948843BC01CE010C960E9493390E8372
:10B440008DEC9BEA9D8B8C8BCE01469665E974E270
:10B450000E9493390E9451429FA78EA70E94A14249
:10B4600088ABCE0101960E947560082F90E00E9483
:10B47000B642009749F10E945842BC01CE010196A4
:10B48000402F0E9493600091EE051091EF050E94FD
:10B4900058427C010E94AB42BC01C701F8010995EA
:10B4A000A114B10489F0009721F08130910561F475
:10B4B00004C0C60160E070E003C0C60164E070E053
:10B4C00041E050E0F5010995E0960FB6F894DEBF33
:10B4D0000FBECDBFDF91CF911F910F91FF90EF90E5
:10B4E000DF90CF90BF90AF9008950E94D45B80937F
:10B4F000DE10E091F805F091F9050995089500979F
:10B5000031F0E091F805F091F90509950895E09181
:10B51000FA05F091FB0509950895CF93DF93EC01AF
:10B5200004C060E070E00E94F73B89919991009718
:10B53000C1F7DF91CF910895CF93DF93EC0102C063
:10B540000E943E3B899199910097D1F7DF91CF916D
:10B550000895CF93DF93EC017B836A830E94A94B0C
:10B5600099838883DF91CF910895FC018081918137
:10B5700022813381820F931F918380830895CF931B
:10B58000DF93EC010E94A94B99838883DF91CF91CF
:10B590000895CF93DF93EC010E94A94B2881398154
:10B5A000AC01421B530B9A012F5F3F4F81E090E0AB
:10B5B0004A815B814217530710F080E090E0DF91F1
:10B5C000CF910895CF93DF93FC01C281D381808115
:10B5D0009181C80FD91F0E94A94B9E01281B390BCE
:10B5E000C901DF91CF910895CF93DF93EEE0F7E2A9
:10B5F000C0EDD6E2A2E0B7E211921192199219922F
:10B60000199219921D9287E2E632F807A9F7DF91A5
:10B61000CF9108950F931F93CF93DF93FC01EE5FBB
:10B62000F84D20818C01000F111F000F111F2223E4
:10B6300011F12091940030919500E801C053D94D4B
:10B64000FC01EE0FFF1FE25FF84D80819181A9019F
:10B65000481B590BCA01A0E0B0E0488159816A81BA
:10B660007B81840F951FA61FB71F88839983AA83A8
:10B67000BB8331832083F801E053F94D60817181F0
:10B6800082819381DF91CF911F910F91089560E0A6
:10B6900070E080E090E00895FC01EE0FFF1FEE0FD8
:10B6A000FF1FE053F94D40835183628373830895F4
:10B6B000EF92FF920F931F93CF93DF93B2E0EB2EA5
:10B6C000B7E2FB2EE0EDF6E2CEE0D7E220E030E09C
:10B6D000D7018D917D018823C9F0009194001091CC
:10B6E000950088819981A801481B590B60E070E0A2
:10B6F00080819181A281B381840F951FA61FB71FFE
:10B7000080839183A283B383198308832F5F3F4F84
:10B71000349622962C303105D9F6DF91CF911F91C6
:10B720000F91FF90EF9008950E94F75F08950F9397
:10B730001F93FC018091DF109091E01033832283EE
:10B740001583048371836083F093E010E093DF102E
:10B75000009719F4CB010E94116080E090E01F91E6
:10B760000F9108958091DF109091E0100097C1F043
:10B770001092E0101092DF10DC0114966D917C9114
:10B7800015971296ED91FC9113970995E091DF10B2
:10B79000F091E010309721F0808191810E9411603A
:10B7A00008950E94077508950E940275089587E71D
:10B7B00096E00E942F3C8FE796E00E942F3C089570
:10B7C000CF93DF930E945E420097A9F08FE796E047
:10B7D0000E944E3CEC01009729F10E94A1429983FE
:10B7E00088830E949C429B838A83CE0104960E9498
:10B7F000D8418CAB17C087E796E00E944E3CEC0125
:10B80000009771F002960E94EA4199838883BE01F5
:10B810006E547F4FCE018E579F4F0E94484302C007
:10B82000C0E0D0E0CE01DF91CF910895BC016E540D
:10B830007F4F8E579F4F0E9448430895CF93DF93C9
:10B84000EC0187E796E0BE010E949F3C009719F04B
:10B8500087E796E009C08FE796E0BE010E949F3C13
:10B86000009729F08FE796E0BE010E94793CDF91B6
:10B87000CF910895CF93DF93EC0187E796E0BE0167
:10B880000E949F3C009779F068817981CE010296F1
:10B890000E941943BE016E547F4FCE018E579F4FB9
:10B8A0000E9459431CC08FE796E0BE010E949F3C56
:10B8B0000097A9F00E94F042688179818A819B817A
:10B8C0000E9419438CA990E00E94B6420E945842FF
:10B8D0004CA9BE016C5F7F4F50E00E946577DF91FD
:10B8E000CF910895CF93DF93EC0187E796E0BE01F7
:10B8F0000E949F3C009719F0CE0102960CC08FE782
:10B9000096E0BE010E949F3C009719F08A819B81BE
:10B9100002C080E090E0DF91CF910895FC0180812A
:10B920009181089570E06F5B7F4F660F771F680FFE
:10B93000791FCB010895E62FF0E0EF5BFF4FEE0F8C
:10B94000FF1FE80FF91F80819181089508958AE310
:10B9500097E10E94843E009721F08AE397E10E94DC
:10B960006F3E0895E0912517F0912617309711F05A
:10B970000995089580E00895EF92FF920F931F9329
:10B98000CF93DF937C018A01FC0180819181009734
:10B9900031F0F3E08C309F0709F0FFC02BC080E04E
:10B9A000E82FF0E0EE0FFF1FEE0FFF1FE85DF84EEF
:10B9B000118210828F5F843098F3809327178091D3
:10B9C000640E9091650EE8E2F7E1918B808B0E9406
:10B9D000373B809326278AE397E160E470E00E947A
:10B9E000593E0E94D9628CE093E0F70191838083F5
:10B9F00081E0D7C0623009F4B2C0633030F466230E
:10BA000009F482C0613079F795C0673819F0683859
:10BA100051F73AC010924217C8E2D7E113C08A81A9
:10BA20009B818017910741F4888199810E940F645E
:10BA3000198218821B821A822496809142178F5F86
:10BA40008093421780914217843048F3E6E3FCE28A
:10BA5000848D958D8017910719F4158E148E118E93
:10BA6000B0962CE2E63BF20798F3ECECFCE2818521
:10BA700092858017910711F4158214823D968DE20C
:10BA8000EE34F807A0F3AFCFE7E14A335E0709F0E1
:10BA9000AACFCA010E94843E009709F4A4CF109255
:10BAA00042172DC0F0E035E0EE0FFF1F3A95E1F7A9
:10BAB000EA5CF34D818D8823E9F08AE397E10E94E7
:10BAC0006F3E8091421790E025E0880F991F2A95DC
:10BAD000E1F78A5C934D9093352C8093342C82E06F
:10BAE0000E9443648091272790912827009711F0A6
:10BAF0000E94B25C809142178F5F80934217E09161
:10BB00004217E43078F26FCF4115510509F46BCF3D
:10BB10005093352C4093342C83E00E9443648091F1
:10BB2000272790912827009711F00E94B25C0E946D
:10BB3000A75C59CF4115510509F455CF5093312CCD
:10BB40004093302C85E00E94436480912727909198
:10BB50002827009709F447CF0E94B25C44CF809118
:10BB6000272790912827009709F43DCF8091382707
:10BB7000863031F48091502781FF02C00E94A75C7B
:10BB800081E00E94436480912727909128270097A5
:10BB900009F429CF0E94DF5E26CFF70111821082BF
:10BBA00083E0DF91CF911F910F91FF90EF90089567
:10BBB000909326178093251708959C014091640E59
:10BBC0005091650E60E0E8E2F7E114C08081918158
:10BBD0008217930769F4828193818417950741F452
:10BBE0006093431711821082C9010E940F64089567
:10BBF00034966F5F643050F360934317089540E0CC
:10BC0000E8E2F7E116C0542F5F5F208131812115F2
:10BC1000310569F440934417918380832091640E29
:10BC20003091650E338322830E94296408953496EF
:10BC3000452F443040F3409344170895FC01809110
:10BC4000640E9091650E958F848F778F668F08951F
:10BC5000FC018091640E9091650E928781877487B4
:10BC600063870895CF93DF93EA010E949B63009757
:10BC700049F02091640E3091650EFC0132872187D6
:10BC8000D487C387DF91CF9108950F931F93CF93EC
:10BC9000DF9300D000D0CDB7DEB78C01AB018FEFC2
:10BCA00089838A838B838C83CE010196B8010E949D
:10BCB000325E009719F0FC01158304830F900F90FA
:10BCC0000F900F90DF91CF911F910F91089584E90C
:10BCD00096E062E040E050E00E94E83B10922827A6
:10BCE000109227270895AC0184E996E061E00E9454
:10BCF000C53B0895AC0184E996E060E00E94C53B35
:10BD000008950F931F93CF93DF938A010E940F63CF
:10BD1000EC01009759F08091640E9091650E9D8F13
:10BD20008C8F1F8F0E8FCE010E947A5ECE01DF9125
:10BD3000CF911F910F910895CF93DF93A091342C51
:10BD4000B091352C109719F0ED016C9605C0C0919B
:10BD5000302CD091312C299680912F2C86FF22C037
:10BD60001092451740E0E8E2F7E116C0808191812A
:10BD700014962D913C9115978217930759F482815F
:10BD80009381009739F040934517998388831B82EC
:10BD90001A8206C034964F5F443040F340934517F3
:10BDA0000E94A75C88819981009731F04A815B816C
:10BDB000609126270E94E83BDF91CF9108950F9371
:10BDC0001F93CF93DF9380913827863009F074C09A
:10BDD000809127279091282725E08030920709F04D
:10BDE0006BC0C4E9D2E0D0932827C093272702E094
:10BDF0000093312714E910933227109254271092A0
:10BE000053270E94D16280959095909354278093F8
:10BE1000532710923A27109239270E94C0628095CA
:10BE2000909590933A27809339270E94B25CD093E3
:10BE30002827C0932727009331271093322790910A
:10BE4000322C8091332CE92FF82FDF01A459BD4FFC
:10BE50008CE692E00D9001920197E1F787E497E27A
:10BE60006CE672E00E947D6280912B2780934727C9
:10BE700080912C278093482780912D2780934927F4
:10BE800080912E2780934A2710925427109253278F
:10BE90000E94D16280959095909354278093532768
:10BEA00010923A27109239270E94C062809590958F
:10BEB00090933A27809339270E94B25CDF91CF910B
:10BEC0001F910F910895FC0120E030E080E0A8E18F
:10BED00011C0419198E0542F5827B52FB17050FDF3
:10BEE0008A278695B13009F480684695915099F774
:10BEF0002F5F3F4F2617370761F708951F920F9264
:10BF00000FB60F920BB60F9211242F933F934F93BE
:10BF10005F936F937F938F939F93AF93BF93EF93B1
:10BF2000FF938091940090919500909313278093B4
:10BF3000122781E08093042780917100807D809397
:10BF400071000E94B25B809104278823E9F18091FF
:10BF50009400909195002091122730911327821719
:10BF60009307A0F48091D8269091D926A091DA2643
:10BF7000B091DB268C57914EAF4FBF4F8093D826A0
:10BF80009093D926A093DA26B093DB268091940073
:10BF900090919500821B930BA0E0B0E04091D826D1
:10BFA0005091D9266091DA267091DB26840F951F77
:10BFB000A61FB71F8093D8269093D926A093DA2680
:10BFC000B093DB2610920427FF91EF91BF91AF91C0
:10BFD0009F918F917F916F915F914F913F912F91A1
:10BFE0000F900BBE0F900FBE0F901F9018959FB72C
:10BFF000F894E1E7F0E08081807D808388B38F62F0
:10C0000088BB10929000E1E9F0E01082109292005B
:10C0100010929500109294008081856080839FBF6C
:10C0200008952FB7F894909399008093980088B35F
:10C030008F6288BBE1E7F0E08081826080832FBF60
:10C040000895CF93DF93FC01DB0185E0EB011992AA
:10C050008A95E9F7858190E083709070009711F0E0
:10C0600082E08C93878190E083709070009721F03C
:10C0700082E012968C931297858190E08370907085
:10C08000009799F0878190E083709070009769F035
:10C0900023893489818592852817390731F481E015
:10C0A000848312961C92129701C01482C581C370BA
:10C0B000C250C23028F4D0E0C256D94F888101C0A6
:10C0C00080E011968C931197E781E370E250E230A3
:10C0D00028F4F0E0E256F94F808101C080E0139629
:10C0E0008C931397DF91CF910895CF93DF9300D076
:10C0F00000D00F92CDB7DEB7BE016F5F7F4F0E94B9
:10C10000216089819A81890F8D5F9B81890F9C8134
:10C11000890F9D81890F0F900F900F900F900F90B6
:10C12000DF91CF910895DF92EF92FF920F931F93CB
:10C13000CF93DF9300D000D000D0CDB7DEB78C0115
:10C140007B01BE016F5F7F4F4E830E94216079812A
:10C150006A81AB81BC81872F90E00396860F911D89
:10C160008A0F911D8B0F911D2D81820F911D4E8184
:10C1700050E0481759070CF498C0F801218130E0CD
:10C180002170307083E0220F331F8A95E1F782819E
:10C1900090E08170907034E0880F991F3A95E1F734
:10C1A000822B90819770892B438150E041705070B1
:10C1B00095E0440F551F9A95E1F7842B448150E098
:10C1C0004170507026E0440F551F2A95E1F7842BEB
:10C1D000F7018083F801258130E023703070220F51
:10C1E000331F220F331F868190E08370907054E0DC
:10C1F000880F991F5A95E1F7822B97819295990F95
:10C20000990F907C982BF7019183F8018085F701B5
:10C210008283723051F4F8018185F7018383F8013C
:10C220008285F701848355E001C053E040E080E05F
:10C2300090E09801260F311D09C0F901E80FF91FA0
:10C24000D384F701E70FF11DD0824F5F742F750F74
:10C250000197461791F7972FA23089F49701270F7E
:10C26000311DF8018389F9018083872F8F5F970142
:10C27000280F311DF8018489F90180839E5F40E019
:10C2800020E030E00B0F111D09C0F801E20FF31F91
:10C290005589F701E80FF11D50834F5F842F890FF7
:10C2A000215030404B1789F701C080E026960FB629
:10C2B000F894DEBF0FBECDBFDF91CF911F910F91DC
:10C2C000FF90EF90DF900895BF92CF92DF92EF92B0
:10C2D000FF920F931F93CF93DF937C01B62EEA0159
:10C2E00082E0861708F0AEC0F7018081D82ED29484
:10C2F000D694D69463E0D622F1E0DF22F701918153
:10C30000292F269526952370C92EC294C694C694CB
:10C3100073E0C722382F37703883382F369536951B
:10C32000369531703983382F329531703A83829542
:10C33000869581708B83DC822D83892F8295837013
:10C340008E83CF8282818887222369F13381948111
:10C3500080E0830F911D9A878987223079F4CA0182
:10C360000B9668E375E00E949339F70186818B870D
:10C3700085818C878701095F1F4F20C087010B5F74
:10C380001F4F2330D9F4F7013D96DA0180E09291F6
:10C390001B969C931B978F5F11968830C1F787017E
:10C3A000035F1F4F0BC087010D5F1F4FCA010B9624
:10C3B00068E375E00E9493391A861986CC2089F1CA
:10C3C000DD2059F4F8012081918180E0820F911DD8
:10C3D0009C8B8B8B0E5F1F4F04C089859A859C8B2D
:10C3E0008B8BF2E0CF1671F4CE01459668E375E0D1
:10C3F0000E949339F80181818D8B80818E8B0E5F35
:10C400001F4F17C0F3E0CF16A1F4085F1F4FD801EC
:10C41000FE0180E09E91958B8F5F31968830D1F739
:10C4200008C0CE01459668E375E00E9493391C8AE6
:10C430001B8A802F8E199B2D981B9FA71EA70DA7C7
:10C44000B81608F480E0DF91CF911F910F91FF9013
:10C45000EF90DF90CF90BF9008959C0141505040E5
:10C46000460F571FFB010EC0B081A0E08181BD01C6
:10C47000680F711D260F371F2617370710F42F5F1F
:10C480003F4F3296E417F50778F3E417F50749F4C0
:10C49000908180E0280F391F2817390710F42F5F8B
:10C4A0003F4FC9010895CF93DF93C0913227D0E069
:10C4B00064973091312720E0C20FD31F9E01280FCF
:10C4C000311DC9016BE377E248E050E00E942D6224
:10C4D00063E477E2AE010E942D62009721F0982775
:10C4E0008927982702C08FEF9FEFDF91CF910895A2
:10C4F00090934D1780934C170895FC014381460F8C
:10C5000040932E27872F99272281280F20932D27AC
:10C51000A181A0932C27508150932B2730E028171E
:10C52000390748F48A2F8F5F80932C27882319F4CA
:10C530005F5F50932B27842F90E0707086179707CA
:10C5400098F480912D278F5F80932D27882361F4A5
:10C5500080912C278F5F80932C27882329F480914A
:10C560002B278F5F80932B2708959C01AB0180E0E0
:10C5700090E0B9010E942D62982789279827089595
:10C5800080E090E06FE277E244E150E00E942D62AB
:10C59000009721F098278927982708958FEF9FEF1C
:10C5A000089586E00E945362089581E10E945362DB
:10C5B000089580E0E82FF0E0EE0FFF1FEA54F34DFE
:10C5C000118210828F5F8430A8F380E0E82FF0E0C2
:10C5D00035E0EE0FFF1F3A95E1F7EA5CF34D118E5F
:10C5E0008F5F843098F380E094E0909350178093AD
:10C5F0004F1740E08DE090E0242F30E0289FF001BD
:10C60000299FF00D389FF00D1124E453F34D15824E
:10C6100014824F5F4A3080F340934E170895CF93B2
:10C62000DF93EC0120914F17309150172F5F3F4F50
:10C630008DE72030380710F020E030E1522F432FF3
:10C64000A0E012C0EA2FF0E0B5E0EE0FFF1FBA95B0
:10C65000E1F7EA5CF34D818D882329F0848195818F
:10C660008417950719F3AF5FA43061F73093501723
:10C6700020934F1710924E1780E0E0E0F0E01EC0CC
:10C68000A82FB0E055E0AA0FBB1F5A95E1F7AA5CAE
:10C69000B34D59969C915997992321F480934E1745
:10C6A000FD0110C0973049F4309731F05A962C9123
:10C6B0005A97928D921708F4FD018F5F843000F332
:10C6C00080934E17309799F182E0818F80915117B6
:10C6D0008487809152178587809153178687809130
:10C6E0005417878788ED94E0938B828B958B848B8E
:10C6F00081E090E0918B808B138E81E0828F83E0CC
:10C70000808F168A80E1878B80914F179091501708
:10C7100098278927982795838483778366838881E0
:10C720009981AA81BB8180839183A283B383CF0146
:10C73000DF91CF9108950F931F93CF93DF93EC0177
:10C740008B0120914F17309150176DE070E02F5FF3
:10C750003F4F8DE72030380710F020E030E1522FB6
:10C76000432FA0E011C08A2F90E0869FF001879FA1
:10C77000F00D969FF00D1124E453F34D84819581C3
:10C78000AF5F8417950719F3AA3069F730935017F4
:10C7900020934F1740E02DE030E018C0542F5F5F2A
:10C7A000842F90E0829FF001839FF00D929FF00D07
:10C7B0001124E453F34D84819581009731F4409323
:10C7C0004E179F01309749F424C0452F4A3030F36B
:10C7D00040934E1720E030E01CC080914F1790919D
:10C7E0005017982789279827958384831783068372
:10C7F000209729F4108211821282138208C0888146
:10C800009981AA81BB8180839183A283B38380E4D1
:10C810008087C901DF91CF911F910F91089540E06A
:10C8200013C0E42FF0E0542F5F5FEE0FFF1FEA54B8
:10C83000F34D208131812817390729F440934E1791
:10C84000118210820895452F443058F340934E17BB
:10C85000089540E013C0E42FF0E0542F5F5FEE0F27
:10C86000FF1FEA54F34D208131812115310529F450
:10C8700040934E17918380830895452F443058F399
:10C8800040934E170895AF92BF92CF92DF92EF92EE
:10C89000FF920F931F93CF93DF93C091342CD091CD
:10C8A000352C843009F4F1C127E537E23093332C7D
:10C8B0002093322C30932A2720932927833071F438
:10C8C000898D90E08F7090708330910509F074C06D
:10C8D00088899989009709F031C78DC0823009F0A5
:10C8E0008EC0809154178F5F80935417882399F4DA
:10C8F000809153178F5F80935317882361F4809141
:10C9000052178F5F80935217882329F48091511713
:10C910008F5F80935117109228271092272710922B
:10C92000CB2C1092CA2C898D873011F0853041F4C0
:10C930008A8D8F5F8A8F843109F000C7198EFEC6F9
:10C94000882309F4FBC6288939892115310509F4A2
:10C950004EC09A8D292F21502A8F992309F0EEC6B7
:10C960009B8D983031F0282F2150223048F495309B
:10C9700039F4198E80E880932F2C0E949C5E94C518
:10C98000953048F423E030E0092E02C0220F331F17
:10C990000A94E2F701C020E32A8F9F5F9B8F90E00B
:10C9A0008F70907083309105E1F0843091054CF4E4
:10C9B0008130910509F469C38230910509F0BEC642
:10C9C0000DC08630910509F47EC58830910509F4C3
:10C9D0007AC58430910509F0B1C675C5109250270B
:10C9E00057C384E080932F2C0E949C5E92C58F7069
:10C9F000833009F0A3C688E080932F2C4AC5853088
:10CA000019F5E091302CF091312C848195810097BB
:10CA100009F494C61092352C1092342C2C503040CE
:10CA20003093332C2093322C30932A2720932927BC
:10CA30001092CB2C1092CA2C1092282710922727E4
:10CA400088E080932F2C1FC180912F27853409F017
:10CA500075C61091312700E080913227080F111D13
:10CA600080912727909128278017910708F466C6A0
:10CA700010932827009327278091352790E08F7304
:10CA80009070009709F05AC680913627882309F0E4
:10CA900055C64091C62C5091C72CA090A006B090CE
:10CAA000A1064A155B0559F48091C82C9091C92CB8
:10CAB0002091A2063091A30682179307A1F08091DE
:10CAC0003F27909140278417950709F037C620919A
:10CAD0004127309142278091C82C9091C92C28176A
:10CAE000390709F02BC60E94C0622FEF8F3F9207D3
:10CAF00009F024C680913827863009F42EC181318F
:10CB0000D1F1813009F01AC680914327883009F0AD
:10CB100015C61092432780914527909146272FEF05
:10CB2000873F920710F0099601C008969093462718
:10CB300080934527EFE2F7E280913B2790913C27D5
:10CB4000A0913D27B0913E2780933F2790934027A7
:10CB5000A0934127B09342278091C62C9091C72C77
:10CB6000A091C82CB091C92C84879587A687B787D8
:10CB700080E48087C0C50C51104010932827009393
:10CB800027278BE497E29093332C8093322C80916B
:10CB9000492790914A27009739F00E94D5622FEFDC
:10CBA0008F3F920709F0CAC540914527509146270B
:10CBB0004115510509F4C2C58CEC9CE29093312CCF
:10CBC0008093302C6091432770914427A091A20656
:10CBD000B091A306C091A406D091A5060091A60627
:10CBE0001091A706E0903B27F0903C27C0903D278E
:10CBF000D0903E272EC084819581009721F148175F
:10CC0000590709F586819781009719F06817790708
:10CC1000D1F4208131812A153B0529F48281938149
:10CC20008A179B07F9F02C173D0729F4828193811D
:10CC300080179107B9F0E216F30629F482819381F7
:10CC4000C816D90679F0CF010D969093312C8093B8
:10CC5000302CE091302CF091312C8DE2EE34F8073D
:10CC600050F26CC51092352C1092342C82E08093D7
:10CC70002F2C8BE497E290932A27809329271092F8
:10CC8000CB2C1092CA2C0E949C5E8091CA2C909151
:10CC9000CB2C009709F452C59C01245E3F4F309382
:10CCA0002827209327273093312720933227E0919C
:10CCB000302CF091312C20852093372721E12093CF
:10CCC0003827089698278927982790934827809394
:10CCD000472710924A271092492784819581909383
:10CCE000442780934327868197819093462780939A
:10CCF00045278091C62C9091C72CA091C82CB0914B
:10CD0000C92C80933B2790933C27A0933D27B09359
:10CD10003E2780819181A281B38180933F279093A8
:10CD20004027A0934127B093422787E597E290934D
:10CD3000332C8093322C0E94D562809590959093ED
:10CD40004A2780934927009709F0D5C48FEF9FEFBA
:10CD500090934A2780934927CEC40E94D1622FEF37
:10CD60008F3F920709F0EAC420914527309146276A
:10CD70002115310509F4E2C440914327509144271D
:10CD80004115510509F4DAC4E0913B27F0913C27A5
:10CD9000A0913D27B0913E27C6E3DCE2698D662372
:10CDA000A9F08C819D812817390781F48E819F819C
:10CDB0004817590759F488819981E817F90731F420
:10CDC0008A819B81A817B90709F47AC1A0968CE2E1
:10CDD000C639D80719F310F3809150278F7382302A
:10CDE000B9F4309356172093551740E00DC0E42F47
:10CDF000F0E0EE0FFF1FEA54F34D808191814F5F09
:10CE00002817390709F47DC0443088F340934E1742
:10CE10008091502782FD92C484E18093502788E25C
:10CE200090E0909328278093272780E580934F27D1
:10CE300080914A2790914E2790934A273091492715
:10CE400090914D279093492730934D272091482763
:10CE500090914C279093482720934C2790914727F7
:10CE600090934E1740914B274093472790934B2721
:10CE70008F5F80934E27882379F4832F8F5F809371
:10CE80004D27882349F4822F8F5F80934C27882376
:10CE900019F49F5F90934B278091432790914427EB
:10CEA0009093561780935517209145273091462728
:10CEB0003093442720934327909346278093452718
:10CEC00080913B2790913C27A0913D27B0913E2730
:10CED00080933F2790934027A0934127B093422708
:10CEE0008091C62C9091C72CA091C82CB091C92CD0
:10CEF00080933B2790933C27A0933D27B0933E27F8
:10CF0000DFC310924E1780E0C0E0D0E022C0E82FCF
:10CF1000F0E075E0EE0FFF1F7A95E1F7EA5CF34D64
:10CF2000918D992321F480934E17EF0116C097300D
:10CF300079F4209721F0228D9A8D921748F4C82F0A
:10CF4000D0E065E0CC0FDD1F6A95E1F7CA5CD34DF8
:10CF50008F5F8430E0F280934E17209709F4EEC380
:10CF6000D093352CC093342C83E08A8F888F1E8A0F
:10CF700084E08F8B1B8E80914527909146279D835F
:10CF80008C8380914327909144279F838E83809147
:10CF90003B2790913C27A0913D27B0913E27888365
:10CFA0009983AA83BB8381E0898F809151178C87F5
:10CFB000809152178D87809153178E8780915417D7
:10CFC0008F8781E090E0998B888B80914A278B87AF
:10CFD000809149278A8780914827898780914727B0
:10CFE000888781E090E00E94DA6C80914F27282F9B
:10CFF00030E0207F3070213531050CF446C0829539
:10D000008F7090E00597880F991F880F991F3091B6
:10D01000571720E031C0E15DF84D30A5332329F4E6
:10D0200020934E171092571730C0313011F42F5FF4
:10D0300023C03230E9F441A54430D1F420934E1797
:10D040003093571792A580E023A530E0282B392B89
:10D050003093561720935517C90124E0893D920754
:10D0600010F088ED94E09B8B8A8B9D8B8C8B0DC090
:10D0700041A5442331F0240FE22FF0E0E817F9072F
:10D0800054F220934E173093571780E18093502726
:10D090008091502782608093502782E080935727A9
:10D0A00084E0809358278093592788ED80935A27EE
:10D0B0008CE290E0909328278093272780E6ADC2EA
:10D0C000D093352CC093342C10922F2C40915027A4
:10D0D00050E042FF03C0198E80E248C280914F2782
:10D0E00082958F70880F880F80934E179801281BA8
:10D0F0003109245130403093282720932727862F49
:10D1000090E08F7090708230910539F4CA018F736E
:10D1100090708231910551F429C08130910531F42C
:10D12000CA018F7390708230910501F1211531058C
:10D1300029F4CA01837090700097C1F0909147273D
:10D140008885981709F05FC29091482789859817BC
:10D1500009F059C2909149278A85981709F053C25E
:10D1600090914A278B85981709F04DC244FF4AC019
:10D17000688979896115710509F444C0CE010C965E
:10D180000E947D6230914B2780912B273817D1F573
:10D1900020914C2780912C272817A1F590914D279D
:10D1A00080912D27981771F580914E2740912E2759
:10D1B000841741F53C872D879E878F878B8D882329
:10D1C000D1F42E89888D9A8D891B922F96959695EC
:10D1D0009695891B280F2E8B87FD81959F89392F66
:10D1E00036953695931B980F9F8B822F8695869543
:10D1F0008695890F888F81E080932F2C888D8A8F68
:10D20000198A188A498D50E0CA018F709070843055
:10D21000910509F4B0C18530910564F4823091051F
:10D22000C9F1833091050CF0B6C08130910509F049
:10D2300085C211C08630910509F4DDC186309105A3
:10D240000CF4B9C18730910509F4DDC1883091052E
:10D2500009F074C285C180912F2C80FF14C083E037
:10D26000898F80E480932F2C198A188A8091272730
:10D2700090912827009709F408C122E420932F2CCD
:10D280000E94DA6C02C1809150278F73823009F0BE
:10D2900055C2FBCE80912F2C80FF72C08091502709
:10D2A0008F73823109F06CC080914F27282F30E0B6
:10D2B000207F3070213531050CF446C082958F7087
:10D2C00090E00597880F991F880F991F3091571785
:10D2D00020E031C0E15DF84D30A5332329F42093DF
:10D2E0004E171092571730C0313011F42F5F23C002
:10D2F0003230E9F441A54430D1F420934E173093F5
:10D30000571792A580E023A530E0282B392B3093C6
:10D31000561720935517C90124E0893D920710F054
:10D3200088ED94E09B8B8A8B9D8B8C8B0DC041A5E7
:10D33000442331F0240FE22FF0E0E817F90754F20C
:10D3400020934E173093571783E0898F809147279A
:10D350008887809148278987809149278A8780918B
:10D360004A278B8781E090E00E94DA6C82E4809308
:10D370002F2C198A188A109228271092272785C0E7
:10D3800080E280932F2C0E949C5EE091342CF091DF
:10D39000352C118E3DCD8091502780FF25C044FD56
:10D3A00023C088899989009709F0C8C180912727EF
:10D3B0009091282701960E94DA6C20912F2C822FC1
:10D3C000806180932F2C80912727909128270097A8
:10D3D00019F0226120932F2C0E949C5E81E090E046
:10D3E000998B888B88E06DC085FF1CC09091552774
:10D3F00080E02091562730E0282B392B8091322C69
:10D400009091332C820F931F9093332C8093322C66
:10D410008091272790912827821B930B9093282790
:10D42000809327278091272790912827009749F0FC
:10D4300044FD07C020912F2C226020932F2C0E94A6
:10D44000DA6C9091512780E020915227820F911D34
:10D4500090935617809355172C893D8928173907C3
:10D4600010F0009721F430935617209355178091B0
:10D470005517909156179B8B8A8B80912F2C90E09B
:10D4800083709070009709F459C11092CB2C1092C0
:10D49000CA2C0E949C5E20912F2C25FF07C0109261
:10D4A000CB2C1092CA2C198E84E1AEC024FF0DC083
:10D4B0001092CB2C1092CA2C81E090E0998B888B33
:10D4C00084E0898F1B8E81E19FC08091CA2C90914E
:10D4D000CB2C0097E9F020FF02C0198A188A28890E
:10D4E00039892115310581F42A893B8928173907A3
:10D4F00020F43093CB2C2093CA2C8091CA2C90918D
:10D50000CB2C998B888B04C03093CB2C2093CA2CC6
:10D510001B8E8091292790912A279093332C8093FA
:10D52000322C8091CA2C9091CB2C009759F088898D
:10D530009989009739F08896909328278093272718
:10D5400088E10BC080912F2C81FFF8C088E290E029
:10D55000909328278093272780E1809350275CC0F1
:10D5600080912F2C80FFEAC0198E80E180932F2CB0
:10D570000E949C5EE3C08091272790912827009706
:10D5800011F00E94DA6C9091502780912F2C90FF1F
:10D590000BC080FF06C087E0898F1A8E198A188A0F
:10D5A00019C086E0898F16C080FF1EC085E0898F74
:10D5B000198A188AC3C0809127279091282700973D
:10D5C00011F00E94DA6C8091502780FF0DC087E037
:10D5D000898F1A8E81E090E00E94DA6C80E180935E
:10D5E0002F2C0E949C5E0FC08091272790912827A6
:10D5F000009749F4A3C080912F2C80FF9FC087E043
:10D60000898F1A8E9BC080E18093502788E290E03A
:10D61000909328278093272780E580934F2788853C
:10D6200080934B27898580934C278A8580934D274B
:10D630008B8580934E278C85809347278D8580939B
:10D6400048278E85809349278F8580934A2786E0D7
:10D65000809338278C819D81909344278093432722
:10D660008E819F8190934627809345278091C62C79
:10D670009091C72CA091C82CB091C92C80933B27C6
:10D6800090933C27A0933D27B0933E2788819981B2
:10D69000AA81BB8180933F2790934027A093412785
:10D6A000B0934227898D84FF05C0109252271092B3
:10D6B000512706C084E08093512788ED809352273C
:10D6C00080E4809337278091272790912827909393
:10D6D00031278093322710925627109255271092A7
:10D6E0005427109253270E94D16280959095909371
:10D6F00054278093532785E480932F271092302757
:10D70000109236271092352780914C1790914D1723
:10D71000019690934D1780934C17909333278093E5
:10D72000342710923A27109239270E94C0628095C0
:10D73000909590933A278093392704C01092282718
:10D740001092272710922F2CDF91CF911F910F91CC
:10D75000FF90EF90DF90CF90BF90AF900895982703
:10D760008927982708950F931F93DC01CB011A2F67
:10D770000B2F20E030E0982789279827A0E0B0E021
:10D78000DC0199278827082B192B2A2B3B2BB80162
:10D79000C9011F910F910895FC0120912927309113
:10D7A0002A278FE29CE2821B930BAB018617970717
:10D7B0000CF4AC01141615065CF44093CA2C50937B
:10D7C000CB2CE217F30721F0C901BF010E94657756
:10D7D0000895CF92DF92EF92FF920F93CF93DF9352
:10D7E000CDB7DEB760970FB6F894DEBF0FBECDBFE2
:10D7F000002309F45AC029873A874B875C876D87D5
:10D800007E878F87988B80E2801B49855A856B8540
:10D810007C851816B4F019821A821B821C82992703
:10D8200087FD9095909581959F4F04C0440F551F9B
:10D83000661F771F8A95D2F74D835E836F83788743
:10D840002CC06A017B01002E04C0CC0CDD1CEE1C38
:10D85000FF1C0A94D2F7C982DA82EB82FC826A0149
:10D860007B0104C0F694E794D794C7948A95D2F7C5
:10D87000D701C6014D855E856F85788904C0440F48
:10D88000551F661F771F0A95D2F7842B952BA62B61
:10D89000B72B8D839E83AF83B88729813A814B81D3
:10D8A0005C816D817E818F81988560960FB6F8943A
:10D8B000DEBF0FBECDBFDF91CF910F91FF90EF90F4
:10D8C000DF90CF900895A0E1B0E0E9E6FCE60C948B
:10D8D0007E7429873A874B875C876D877E878F8721
:10D8E000988BA982BA82CB82DC82ED82FE820F8382
:10D8F00018874D855E856F8578898D819E81AF8182
:10D90000B885481759076A077B07C8F08417950739
:10D91000A607B70790F049855A856B857C85898174
:10D920009A81AB81BC81481759076A077B0738F099
:10D9300084179507A607B70720F482E003C080E0AC
:10D9400001C081E06096EAE00C949A7480E88093CC
:10D950006100109261000E94D1480E94553B0E94D4
:10D96000304D8091D6249091D724009729F00197CB
:10D970009093D7248093D624C090D824D090D924D3
:10D98000E090DA24F090DB240E94D54BDC01CB013F
:10D99000C816D906EA06FB0601F30E94D54BDC0146
:10D9A000CB018093D8249093D924A093DA24B09308
:10D9B000DB24D3CFBC018091342C9091352C089678
:10D9C0000E947D62E091342CF091352C80912B27C0
:10D9D000808780912C27818780912D278287809155
:10D9E0002E27838708952F923F924F925F926F92D6
:10D9F0007F928F929F92AF92BF92CF92DF92EF92DF
:10DA0000FF920F931F93CF93DF93CDB7DEB7659748
:10DA10000FB6F894DEBF0FBECDBF4C017F876E8777
:10DA2000FC0117821682838181FD04C076C34C8578
:10DA30005D8504C01E010894211C311CF4019381F2
:10DA4000EE85FF8593FD859193FF8191FF87EE879A
:10DA5000882309F45EC3853241F493FD859193FFD9
:10DA60008191FF87EE87853259F490E0B4014C8BA9
:10DA70005D8B0E94B8774C895D895D874C87D7CFD5
:10DA8000FF24DD2410E01032B0F48B3269F08C32C8
:10DA900028F4803251F0833271F40BC08D3239F0AA
:10DAA000803349F411602CC01260146029C01860E2
:10DAB00027C0106125C017FD2EC0282F20532A3003
:10DAC00098F416FF08C08F2D880FF82EFF0CFF0C5E
:10DAD000F80EF20E15C08D2D880FD82EDD0CDD0C42
:10DAE000D80ED20E10620CC08E3221F416FD11C376
:10DAF000106406C08C3611F4106802C0883659F4E0
:10DB0000EE85FF8593FD859193FF8191FF87EE87D9
:10DB1000882309F0B8CF982F9554933018F41061EA
:10DB2000805E06C0982F9556933008F0A2C11F7EE4
:10DB300016FD02C0E6E0FE2E1F73853611F4106458
:10DB400006C0863611F4106802C0F110FA9417FF6F
:10DB500007C0FBE3FF1548F0EF2CE39427E00DC06E
:10DB600027E02F1530F02F2D07C027E07CE3E72EAC
:10DB700004C027E067E0F62EEE24CA0104969D87D4
:10DB80008C87FA016081718182819381A1010E2DC0
:10DB90000E9475765C01C9802C2D30E0398B288B72
:10DBA000C0FE03C0388933FF06C011FD06C012FF56
:10DBB00006C000E205C00DE203C00BE201C000E0B8
:10DBC000888999898C709070009709F43CC0002373
:10DBD00011F084E001C083E08D1558F4D81A13FDCC
:10DBE00009C080E290E0B4010E94B877DA94C9F7E6
:10DBF00001C0DD24002329F0802F90E0B4010E94B1
:10DC0000B877888983FD05C03CE1E32E3FE0F32E21
:10DC100011C028E1E22E2FE0F22E0CC001151105F3
:10DC200009F0805290E0B4010E94B8770894E11C9A
:10DC3000F11C04C0012F10E000711070F7018491F5
:10DC4000882361F763C217FF0EC0EA0CF889F4FF5E
:10DC500004C08A81813309F4EA941E144CF528E04B
:10DC60002E1548F12CC016FD2AC08F2D90E08A1584
:10DC70009B0544F03CEFA3163FEFB3061CF0106881
:10DC800001C0FA94FF2049F0E2E0F0E0EC0FFD1F44
:10DC9000EF0DF11D80818033A1F317FF10C0EF2C31
:10DCA000E3948F2D90E0A816B90644F4FA1807C043
:10DCB000EE24E39404C098E0E92E01C0FF2417FF8E
:10DCC00007C01A141B043CF495012F5F3F4F05C099
:10DCD00025E030E002C021E030E0002311F02F5FAA
:10DCE0003F4FFF2029F08F2D90E00196280F391F1C
:10DCF0008D2D90E02817390714F4D21A01C0DD24C5
:10DD0000612E7724C30189709070009749F406C092
:10DD100080E290E0B4010E94B877DA94DD20C1F788
:10DD2000002329F0802F90E0B4010E94B87763FCB3
:10DD300009C006C080E390E0B4010E94B877DA948D
:10DD4000DD20C1F717FF48C08501B7FE02C000E023
:10DD500010E04424552495012E1931093B8B2A8B60
:10DD60003501601A710A620C731C6F2D70E0EE248D
:10DD7000FF24E61AF70A3FEF0F3F130729F48EE25C
:10DD800090E0B4010E94B877A016B10654F02A8939
:10DD90003B89201731072CF4F301E40DF51D818137
:10DDA00001C080E3015010400894411C511C0E1525
:10DDB0001F052CF090E0B4010E94B877DCCF0A1563
:10DDC0001B0541F49A81963320F4953319F4388970
:10DDD00034FF81E390E049C08A81813311F09FEEE6
:10DDE000C92290E0B4010E94B877FF2089F08EE24A
:10DDF00090E0B4010E94B87712E0F101E10FF11D4B
:10DE00001F5F808190E0B4010E94B877FA94A9F76F
:10DE100064FE03C085E490E002C085E690E0B401B2
:10DE20000E94B877B7FC05C0A114B10441F4C4FE48
:10DE300006C0B094A194B108B3948DE201C08BE206
:10DE400090E0B4010E94B87780E305C08F5FE6EFF1
:10DE5000FFEFAE0EBF1EFAE0AF16B104BCF790E0C4
:10DE6000B4010E94B877C501C096B4010E94B8778A
:10DE70004DC1833631F0833789F0833509F059C0BD
:10DE800022C09A012E5F3F4F3D872C87FA01808187
:10DE9000898381E0E82EF12C510113C09A012E5F95
:10DEA0003F4F3D872C87FA01A080B18016FF03C049
:10DEB0006F2D70E002C06FEF7FEFC5010E947E778B
:10DEC0007C011F7714C09A012E5F3F4F3D872C873E
:10DED000FA01A080B18016FF03C06F2D70E002C070
:10DEE0006FEF7FEFC5010E9455777C01106813FD2D
:10DEF0001CC006C080E290E0B4010E94B877DA94BA
:10DF00008D2D90E0E816F906A8F30FC0F50117FD76
:10DF1000859117FF81915F0190E0B4010E94B8776D
:10DF2000D110DA940894E108F108E114F10471F7D2
:10DF3000EDC0843611F0893671F59A0117FF0AC0D9
:10DF40002C5F3F4F3D872C87FA0180819181A28110
:10DF5000B3810BC02E5F3F4F3D872C87FA01808134
:10DF60009181AA2797FDA095BA2F012F0F76B7FFB1
:10DF700008C0B095A095909581959F4FAF4FBF4F2A
:10DF80000068BC01CD01A1012AE030E00E94C07808
:10DF9000E82EE21841C0853721F41F7E2AE030E0E8
:10DFA00020C0197F8F36A9F0803720F4883509F01A
:10DFB000B0C00BC0803721F0883709F0AAC001C07B
:10DFC000106114FF09C0146007C014FF08C0166078
:10DFD00006C028E030E005C020E130E002C020E1CA
:10DFE00032E0CA0117FF09C004969D878C87FA01A9
:10DFF000608171818281938108C002969D878C87A0
:10E00000FA016081718180E090E0A1010E94C078F6
:10E01000E82EE218012F0F7706FF09C00E7FEF14DC
:10E0200030F404FF06C002FD04C00F7E02C01E2DA6
:10E0300001C01F2D802F90E004FF0CC0FE01EE0DEB
:10E04000F11D2081203311F4097E09C002FF06C0B2
:10E050001E5F05C086789070009709F01F5FA02EA4
:10E06000BB2403FD12C000FF0DC0FE2C1D1550F493
:10E07000FD0CF11A1D2D06C080E290E0B4010E9453
:10E08000B8771F5F1D15C0F304C01D1510F4D11A19
:10E0900001C0DD24A4FE0FC080E390E0B4010E9423
:10E0A000B877A2FE1FC0A1FE03C088E590E010C0B3
:10E0B00088E790E00DC0C50186789070009791F0D8
:10E0C000A1FC02C080E201C08BE207FD8DE290E07E
:10E0D000B4010E94B87706C080E390E0B4010E94CA
:10E0E000B877FA94EF14C0F3EA94F101EE0DF11D44
:10E0F000808190E0B4010E94B877EE20A9F706C0B5
:10E1000080E290E0B4010E94B877DA94DD20C1F794
:10E110008ECCF4018681978102C08FEF9FEF6596C8
:10E120000FB6F894DEBF0FBECDBFDF91CF911F9128
:10E130000F91FF90EF90DF90CF90BF90AF909F90A6
:10E140008F907F906F905F904F903F902F900895A9
:10E150005058BB27AA270ED044C135D130F03AD150
:10E1600020F031F49F3F11F41EF42AC10EF4E09523
:10E17000E7FB20C1E92F46D180F3BA176207730786
:10E180008407950718F071F49EF55EC10EF4E095D2
:10E190000B2EBA2FA02D0B01B90190010C01CA0161
:10E1A000A0011124FF27591B99F0593F50F4503E0C
:10E1B00068F11A16F040A22F232F342F4427585FFE
:10E1C000F3CF469537952795A795F0405395C9F716
:10E1D0007EF41F16BA0B620B730B840BBAF09150CE
:10E1E000A1F0FF0FBB1F661F771F881FC2F70EC06D
:10E1F000BA0F621F731F841F48F487957795679540
:10E20000B795F7959E3F08F0B3CF9395880F08F028
:10E210009927EE0F979587950895A8D008F481E087
:10E2200008950CD0DEC0D6D040F0CDD030F021F42F
:10E230005F3F19F0BFC0511108C1C2C0E3D098F3CD
:10E240009923C9F35523B1F3951B550BBB27AA2777
:10E2500062177307840738F09F5F5F4F220F331FE9
:10E26000441FAA1FA9F333D00E2E3AF0E0E830D0B5
:10E2700091505040E695001CCAF729D0FE2F27D0B8
:10E28000660F771F881FBB1F261737074807AB0786
:10E29000B0E809F0BB0B802DBF01FF2793585F4FFB
:10E2A0002AF09E3F510568F085C0CFC05F3FECF378
:10E2B000983EDCF3869577956795B795F7959F5FC0
:10E2C000C9F7880F911D9695879597F90895E1E014
:10E2D000660F771F881FBB1F621773078407BA0773
:10E2E00020F0621B730B840BBA0BEE1F88F7E095CE
:10E2F0000895E89409C097FB3EF490958095709539
:10E3000061957F4F8F4F9F4F9923A9F0F92F96E981
:10E31000BB279395F695879577956795B795F111F6
:10E32000F8CFFAF4BB0F11F460FF1BC06F5F7F4F93
:10E330008F4F9F4F16C0882311F096E911C07723A5
:10E3400021F09EE8872F762F05C0662371F096E8AE
:10E35000862F70E060E02AF09A95660F771F881F7D
:10E36000DAF7880F9695879597F90895990F000821
:10E37000550FAA0BE0E8FEEF16161706E807F90797
:10E38000C0F012161306E407F50798F0621B730B32
:10E39000840B950B39F40A2661F0232B242B252BB3
:10E3A00021F408950A2609F4A140A6958FEF811D56
:10E3B000811D089597F99F6780E870E060E00895F7
:10E3C0009FEF80EC089500240A941616170618068D
:10E3D0000906089500240A94121613061406050669
:10E3E0000895092E0394000C11F4882352F0BB0FFA
:10E3F00040F4BF2B11F460FF04C06F5F7F4F8F4F5D
:10E400009F4F089557FD9058440F551F59F05F3F97
:10E4100071F04795880F97FB991F61F09F3F79F046
:10E4200087950895121613061406551FF2CF4695C8
:10E43000F1DF08C0161617061806991FF1CF86954A
:10E440007105610508940895E894BB27662777272E
:10E45000CB0197F908950BD0C4CFB5DF28F0BADF10
:10E4600018F0952309F0A6CFABCF1124EECFCADF69
:10E47000A0F3959FD1F3950F50E0551F629FF001D7
:10E48000729FBB27F00DB11D639FAA27F00DB11D30
:10E49000AA1F649F6627B00DA11D661F829F2227B9
:10E4A000B00DA11D621F739FB00DA11D621F839F40
:10E4B000A00D611D221F749F3327A00D611D231F16
:10E4C000849F600D211D822F762F6A2F11249F5764
:10E4D00050408AF0E1F088234AF0EE0FFF1FBB1F87
:10E4E000661F771F881F91505040A9F79E3F510526
:10E4F00070F060CFAACF5F3FECF3983EDCF38695D7
:10E5000077956795B795F795E7959F5FC1F7FE2BD0
:10E51000880F911D9695879597F90895FA01EE0F4A
:10E52000FF1F30962105310599F16115710561F4E0
:10E530008038BFE39B0749F168949038810561F00A
:10E540008038BFEF9B0741F0992342F5FF3FE1057B
:10E550003105210511F1E8940894E795D901AA2322
:10E5600029F4AB2FBE2FF85FD0F310C0FF5F70F41B
:10E57000A695E0F7F73950F019F0FF3A38F49F7795
:10E580009F930CD00F9007FC905808953EF018CF41
:10E5900060E070E080E89FE308954FE79F775F9326
:10E5A0004F933F932F939ED02F913F914F915F9127
:10E5B00052DF05C019F40EF0FDCE46CF01CF2ADFA1
:10E5C000C8F39638C0F707F80F92E8942BE33AEABD
:10E5D00048EB5FE74EDF0F920F920F924DB75EB799
:10E5E0000F92C0D0E0E2F1E016D04F915F91EF9131
:10E5F000FF91E595EE1FFF1F49F0FE57E0684427A5
:10E60000EE0F441FFA95E1F74195550B32D00F906C
:10E6100007FE26C00895DF93CF931F930F93FF92B9
:10E62000EF92DF927B018C01689405C0DA2EEF0136
:10E630001EDFFE01E894A5912591359145915591F4
:10E64000AEF3EF0197DDFE019701A801DA9479F7A7
:10E65000DF90EF90FF900F911F91CF91DF91089580
:10E660009B01AC0160E070E080E89FE3DACDA2CED0
:10E67000ACC0D0DEE8F39923D9F3940F511DBBF35E
:10E680009150504094F059F0882332F0660F771F74
:10E69000881F91505040C1F79E3F510544F7880FA5
:10E6A000911D9695879597F908955F3FACF0983E38
:10E6B0009CF0BB27869577956795B79508F4B16070
:10E6C0009395C1F7BB0F58F711F460FFE8CF6F5F68
:10E6D0007F4F8F4F9F4FE3CFB8CE0EF076C070CEF6
:10E6E000689468CE97DEC8F39923D1F3C6F3DF931D
:10E6F000CF931F930F93FF92C92FDD2788232AF012
:10E700002197660F771F881FDAF720E030E040E896
:10E710005FEB9FE3883920F0803E30F021968F77C1
:10E7200018DDE8E4F1E003C014DDE5E7F1E073DFB4
:10E730008B01BE01EC01FB2E6F5771097595771F98
:10E74000880B990BD8DD28E132E741E35FE38FDEE8
:10E75000AF2D9801AE01FF900F911F91CF91DF91E6
:10E7600009DD3FCEFA01DC01AA0FBB1F9B01AC0102
:10E77000BF5728F422273327442750781FC0B751AA
:10E7800088F4AB2F0024469537952795011CA39557
:10E79000D2F3002069F0220F331F441FB395DAF340
:10E7A0000DD0D6CC61307105A0E88A07B94630F4A7
:10E7B0009B01AC016627772788279078309621F057
:10E7C000208331834283538308959F3F31F09150DA
:10E7D00020F4879577956795B795880F911D969545
:10E7E000879597F90895629FD001739FF001829FEA
:10E7F000E00DF11D649FE00DF11D929FF00D839FD0
:10E80000F00D749FF00D659FF00D9927729FB00D6C
:10E81000E11DF91F639FB00DE11DF91FBD01CF017F
:10E8200011240895AA1BBB1B51E107C0AA1FBB1FDF
:10E83000A617B70710F0A61BB70B881F991F5A958C
:10E84000A9F780959095BC01CD01089597FB092EFD
:10E8500007260AD077FD04D0E5DF06D000201AF4A1
:10E86000709561957F4F0895F6F7909581959F4F2C
:10E870000895A1E21A2EAA1BBB1BFD010DC0AA1F01
:10E88000BB1FEE1FFF1FA217B307E407F50720F019
:10E89000A21BB30BE40BF50B661F771F881F991F94
:10E8A0001A9469F760957095809590959B01AC01DD
:10E8B000BD01CF01089597FB092E05260ED057FD07
:10E8C00004D0D7DF0AD0001C38F45095409530951D
:10E8D00021953F4F4F4F5F4F0895F6F790958095E4
:10E8E000709561957F4F8F4F9F4F08952F923F9264
:10E8F0004F925F926F927F928F929F92AF92BF9250
:10E90000CF92DF92EF92FF920F931F93CF93DF93FB
:10E91000CDB7DEB7CA1BDB0B0FB6F894DEBF0FBE58
:10E92000CDBF09942A88398848885F846E847D84A5
:10E930008C849B84AA84B984C884DF80EE80FD80A7
:10E940000C811B81AA81B981CE0FD11D0FB6F8941D
:10E95000DEBF0FBECDBFED0108958F929F92AF92A3
:10E96000BF92CF92DF92EF92FF92CF93DF93EC01B1
:10E9700088819981AA81BB810097A105B10521F405
:10E9800084E299EDABE5B7E0BC01CD012DE133EFB9
:10E9900041E050E00E945B7449015A0127EA31E4EA
:10E9A00040E050E00E94F3736B017C01C501B401AB
:10E9B0002CEE34EF4FEF5FEF0E94F373DC01CB01DD
:10E9C000C80ED91EEA1EFB1EF7FE08C08FEF9FEF90
:10E9D000AFEFBFE7C80ED91EEA1EFB1EC882D98260
:10E9E000EA82FB82C6019F77DF91CF91FF90EF9083
:10E9F000DF90CF90BF90AF909F908F9008950E942E
:10EA0000AD74089588EA96E00E94AD740895A0E080
:10EA1000B0E08093A8069093A906A093AA06B093AD
:10EA2000AB0608953F924F925F926F927F928F92C2
:10EA30009F92AF92BF92CF92DF92EF92FF920F938D
:10EA40001F93CF93DF9300D000D0CDB7DEB72B015B
:10EA50007A016115710529F0DB018C9311969C9365
:10EA60001197E114F10439F097012250304023321C
:10EA7000310508F0FCC06C0186010894C11CD11C52
:10EA8000F80130803601832D90E00E944D77009789
:10EA900099F7FDE23F1661F4D80111963C90119769
:10EAA00092E0692E712C600E711ECC24C3940BC0B1
:10EAB000BBE23B1639F4F801318082E0682E712CFC
:10EAC000600E711ECC24E114F10421F0F0E1EF1688
:10EAD000F104F9F480E3381691F4D3018C9188376E
:10EAE00011F0883561F4F301318082E090E0680E26
:10EAF000791E92E0C92AB0E1EB2EF12C0AC0E11494
:10EB0000F10439F4A0E33A16D1F0AAE0EA2EF12C90
:10EB100030C0BAE0EB16F10461F1E0E1EE16F10469
:10EB200029F0F8E0EF16F104B1F409C0FFEF8F2EE1
:10EB3000FFEF9F2EFFEFAF2EFFE0BF2E22C078E049
:10EB4000E72EF12CEFEF8E2EEFEF9E2EEFEFAE2E95
:10EB5000EFE1BE2E16C09701442737FD4095542F94
:10EB60006FEF7FEF8FEF9FEF0E94397449015A01D9
:10EB700008C069E9862E69E9962E69E9A62E69E141
:10EB8000B62E40E000E010E020E030E0C701AA2708
:10EB900097FDA095BA2F89839A83AB83BC8350EDF0
:10EBA000D52ED30C99E09D1570F4832D81548A31B4
:10EBB00018F499ECD92E06C0832D81568A3168F558
:10EBC00089EAD82ED30C8D2D90E08E159F052CF55B
:10EBD0004F3FF9F080169106A206B306B8F0C901BE
:10EBE000B80129813A814B815C810E94F3738B01CA
:10EBF0009C018D2D90E0A0E0B0E0080F191F2A1FA6
:10EC00003B1F081719072A073B0710F44FEF01C0F5
:10EC100041E0D3013D903D01C2CF4114510489F040
:10EC2000442339F0089461087108F201718260820E
:10EC300008C0C1FE06C0C3010297D20111969C9381
:10EC40008E93C0FE07C030952095109501951F4FFB
:10EC50002F4F3F4F47FF0FC082E290E09093552D1A
:10EC60008093542D0FEF1FEF2FEF3FEF04C000E014
:10EC700010E020E030E0B801C9010F900F900F9034
:10EC80000F90DF91CF911F910F91FF90EF90DF9048
:10EC9000CF90BF90AF909F908F907F906F905F903C
:10ECA0004F903F900895662777270C945979FC017F
:10ECB00088279927E89421912032E9F3293010F030
:10ECC0002E30C8F32B3241F02D3239F4689404C051
:10ECD0000E94B077820F911D219120532A30C0F3FA
:10ECE0001EF4909581959F4F0895283008F027E0F5
:10ECF0003327DA01990F311D87FD91600096610578
:10ED0000710539F432602E5F3D9330E32A95E1F7C7
:10ED100008959F3F30F080387105610509F03C5F30
:10ED20003C5F3D93913008F08068911DDF93CF9355
:10ED30001F930F93FF92EF92192F987F9695E92FCB
:10ED400096959695E90FFF27E658F04F99273327B8
:10ED5000EE24FF24A701E70105900894079428F406
:10ED6000360FE71EF81E491F511D660F771F881FBB
:10ED7000991F0694A1F70590079428F4E70EF81E52
:10ED8000491F561FC11D770F881F991F661F0694C4
:10ED9000A1F70590079428F4F80E491F561FC71FC6
:10EDA000D11D880F991F661F771F0694A1F7059044
:10EDB000079420F4490F561FC71FD81F990F661FCD
:10EDC000771F881F0694A9F784911095177041F05A
:10EDD000D695C79557954795F794E7941A95C1F737
:10EDE000E0E2FFE068941590159135916591959159
:10EDF00005907FE27395E118F10A430B560BC90B9E
:10EE0000D009C0F7E10CF11E431F561FC91FD01DCA
:10EE10007EF4703311F48A95E6CFE894015030F017
:10EE2000080F0AF40027021708F4202F2395022F59
:10EE30007A3328F079E37D932A95E9F710C07D9322
:10EE40002A9589F60694979567953795179517949F
:10EE5000E118F10A430B560BC90BD00998F0239522
:10EE60007E9173957A3308F070E37C932013B8F7A2
:10EE70007E9170617D9330F0839571E37D9370E3B3
:10EE80002A95E1F71124EF90FF900F911F91CF91F8
:10EE9000DF91992787FD90950895911189C380325C
:10EEA00019F089508550D0F70895FC010590615004
:10EEB00070400110D8F7809590958E0F9F1F089590
:10EEC00048E557E10E9489770895FB01DC0102C003
:10EED00001900D9241505040D8F70895DC0101C0D7
:10EEE0006D9341505040E0F70895FB01DC018D9196
:10EEF000019080190110D9F3990B0895FC0161501C
:10EF0000704001900110D8F7809590958E0F9F1F4B
:10EF10000895FA01A191B081009719F41097E1F0DA
:10EF2000CD01DC01CD010D90002011F4C00113C012
:10EF3000FB012191222319F02015D9F7F3CFFB0112
:10EF40002191201519F41E92119606C02223C1F7B3
:10EF50000D900020A1F7D001FA01A193B08308958C
:10EF60007AE0979F902D879F802D910D1124089511
:10EF70000F931F93CF93DF938C01EB018B8181FF64
:10EF80001BC082FF0DC02E813F818C819D8128177F
:10EF9000390764F4E881F9810193F983E88306C0B5
:10EFA000E885F985802F0995009731F48E819F813E
:10EFB00001969F838E8302C00FEF1FEFC801DF9180
:10EFC000CF911F910F910895CF93DF93CDB7DEB707
:10EFD000FE013596619171918091502D9091512D46
:10EFE000AF010E94F36CDF91CF910895CF93DF932F
:10EFF000CDB7DEB7FE013596619171918091502DAC
:10F000009091512DDC0113962C9113972860139643
:10F010002C93AF010E94F36CE091502DF091512D93
:10F020002381277F2383DF91CF9108956091502D15
:10F030007091512D0E94B87708950F931F93CF932D
:10F04000DF938C01E091502DF091512D838181FF50
:10F050001AC0C0E0D0E005C00995009711F0CFEFCD
:10F06000DFEFF80181918F016091502D7091512D4A
:10F07000DB011896ED91FC911997882369F78AE0D6
:10F080000995009711F0CFEFDFEFCE01DF91CF911F
:10F090001F910F9108950F931F93CF93DF93CDB7D7
:10F0A000DEB72E970FB6F894DEBF0FBECDBF0D8929
:10F0B0001E898F89988D26E02C831A83098397FFF8
:10F0C00002C080E090E801979E838D83AE01455E8B
:10F0D0005F4FCE010196698D7A8D0E94F36C4D8150
:10F0E0005E8157FD0AC02F813885421753070CF403
:10F0F0009A01020F131FF80110822E960FB6F89492
:10F10000DEBF0FBECDBFDF91CF911F910F9108954C
:10F110000F931F93CF93DF93CDB7DEB72E970FB624
:10F12000F894DEBF0FBECDBF8C0186E08C831A83BE
:10F13000098377FF02C060E070E8615070407E8311
:10F140006D83CE010196BA01A9010E94F36C4D8135
:10F150005E8157FD0AC02F813885421753070CF492
:10F160009A01020F131FF80110822E960FB6F89421
:10F17000DEBF0FBECDBFDF91CF911F910F910895DC
:10F18000FA01AA27283051F1203181F1E8946F93D8
:10F190006E7F6E5F7F4F8F4F9F4FAF4FB1E03ED07E
:10F1A000B4E03CD0670F781F891F9A1FA11D680F1C
:10F1B000791F8A1F911DA11D6A0F711D811D911D4F
:10F1C000A11D20D009F468943F912AE0269F1124C4
:10F1D0003019305D3193DEF6CF010895462F477028
:10F1E000405D4193B3E00FD0C9F7F6CF462F4F7083
:10F1F000405D4A3318F0495D31FD4052419302D0E1
:10F20000A9F7EACFB4E0A695979587957795679586
:10F21000BA95C9F700976105710508959B01AC0186
:10F220000A2E06945795479537952795BA95C9F7AD
:10F23000620F731F841F951FA01D0895DC01CB0171
:10F24000FC01F999FECF06C0F2BDE1BDF89A3196F6
:10F2500000B40D9241505040B8F70895F999FECF8F
:10F2600092BD81BDF89A992780B50895A8E1B0E0D4
:10F2700042E050E00C942079DC01CB0103C02D91D9
:10F280000E94477941505040D0F70895262FF999B0
:10F29000FECF1FBA92BD81BD20BD0FB6F894FA9A79
:10F2A000F99A0FBE019608950E944679272F0C9473
:10F2B00047796F927F928F929F92AF92BF92CF9237
:10F2C000DF92EF92FF920F931F93CF93DF935B0137
:10F2D0006115710521F0DB018C9311969C937C01E3
:10F2E000E7010894E11CF11C08816701802F90E080
:10F2F0000E944D770097A1F70D3241F4098142E059
:10F30000C42ED12CCC0EDD1E11E009C00B3231F41D
:10F31000098132E0C32ED12CCC0EDD1E10E0E601B7
:10F320002197CE016AE170E143E050E00E94DB7A70
:10F330000097D1F4E6012296CE016DE170E145E03F
:10F3400050E00E94DB7A009711F4E6012796A114A1
:10F35000B10419F0F501D183C08330E020E090E8DA
:10F36000112309F40DC107C1CE0162E270E143E04F
:10F3700050E00E94DB7A009759F4A114B10409F41B
:10F38000FCC0C6010296D50111969C938E93F5C0E0
:10F3900040E050E060E070E08824992400530A3097
:10F3A00090F51260212F30E0C9018870907012FF33
:10F3B00006C0009769F50894811C911C29C000972C
:10F3C00019F0089481089108DB01CA01D2E0880F86
:10F3D000991FAA1FBB1FDA95D1F7480F591F6A1F43
:10F3E0007B1F440F551F661F771F400F511D611D66
:10F3F000711D4839B9E95B07B9E96B07B9E17B07CA
:10F4000038F0146005C00E3F39F413FD43C0186096
:10F41000F60101916F01C2CF053311F00531D1F52D
:10F42000D601EC91ED3211F4106108C0EB3229F0F5
:10F43000C601019621E030E008C0D6011196EC919A
:10F440001197C601029622E030E0E053EA3020F046
:10F450006C01C21AD30A1EC0DC0120E030E0FCE0DF
:10F4600020383F075CF4C901880F991F880F991F46
:10F47000280F391F220F331F2E0F311DED91E0533E
:10F480006D01EA3060F314FF03C0309521953F4FC2
:10F49000820E931EC12FD0E011FF08C0A114B10449
:10F4A00029F0C6010197D5018D939C93CB01BA0138
:10F4B0000E9479716B017C01CE0183709070833062
:10F4C000910521F4F7FAF094F7F8F094C701B6012A
:10F4D00020E030E040E050E00E940D71882309F404
:10F4E00045C097FE07C09094819491089394C1E51C
:10F4F000D0E102C0C9E3D0E198EE692E9FEF792EEA
:10F500006C0E7D1E20E2A22EB12C0FC0FE010591D3
:10F51000159125913491C701B601A90198010E9466
:10F520002B726B017C018A189B088A149B0474F768
:10F530002497B594A794C615D705B9F7C601D70186
:10F540002A2F220F2B2F221F2F3F51F0BC01CD015C
:10F5500020E030E040E050E00E940D71882331F45B
:10F5600082E290E09093552D8093542D3C2D2D2DCB
:10F570009E2D8F2D06C08FEF04C030E020E090EC70
:10F580008FE7B901AC01872F922FA52FB42FBC01B3
:10F59000CD01DF91CF911F910F91FF90EF90DF9000
:10F5A000CF90BF90AF909F908F907F906F90089575
:10F5B000992788270895FB01DC014150504088F0CD
:10F5C0008D9181341CF08B350CF4805E6591613433
:10F5D0001CF06B350CF4605E861B611171F3990BA6
:0AF5E0000895881BFCCFF894FFCFBC
:10F5EA00263A202573205B414444523D252D642E42
:10F5FA00252D64205345513D252D642052535349EE
:10F60A003D252D75204C51493D252D7520445250DC
:10F61A003D252D642E253032645D0A00523D252D8C
:10F62A0075204C3D252D7520533D252D6420005411
:10F63A00696D656F757420414444523D252D642ED1
:10F64A00252D64205345513D252D6420525353499D
:10F65A003D252D75204C51493D252D750A0028451B
:10F66A00787450777229000045554936343D002593
:10F67A003032582D00253032580A00534E3D004191
:10F68A003A202564202564202564200A00433A2074
:10F69A002564202564202564200A0073746174752A
:10F6AA00733D3078253032780A2000312E302046DA
:10F6BA0069726D77617265205665722E20332E3914
:10F6CA0020323031332D30332D303400656570727D
:10F6DA006F6D006F6E006F666600666F7263655FBE
:10F6EA0069646C650064656570004F6E0061310085
:10F6FA007265736574006E6F6E6500613200765FC5
:10F70A00696E0031003200330034006175746F0095
:10F71A00666C75736800414444523D252D642E255C
:10F72A002D64205345513D252D6420525353493DA4
:10F73A00252D75204C51493D252D750A007077728B
:10F74A00733D25730A007472696D007465737400E1
:10F75A0043683D252D642054785077723D252D64E9
:10F76A000A004572726F72205458204C656E677495
:10F77A00683D25640A0049443D002530327800205E
:10F78A0050533D25640020543D252D362E32660007
:10F79A002054313D252D362E32660020545F4D43CC
:10F7AA00553D252D352E31660020565F4D43553D7A
:10F7BA00252D342E3266002050303D252D6C580000
:10F7CA002050305F543D252D372E336600205031AE
:10F7DA003D252D6C58002050315F543D252D372E84
:10F7EA003366002055503D252D6C58002052483D67
:10F7FA00252D342E31660020565F494E3D252D3584
:10F80A002E32660020565F41313D252D352E326657
:10F81A000020565F41323D252D352E32660020509C
:10F82A003D252D6C64002050413D252D372E326632
:10F83A0000263A2025730A00545820706B74206CF5
:10F84A00656E203D2025640A0025303258006C651B
:10F85A006E3D25640A00F504DF04C7049304AB0473
:10F86A000000506572696F6469632070726F636526
:10F87A00737300000082047E1600000000536C655A
:10F88A0065702070726F636573730000009D04BF1A
:10F89A000F0000000062726F61646361737420700C
:10F8AA00726F63657373000000B504A5320000002F
:10F8BA0000737464696E2070726F636573730000FD
:10F8CA0000D104D10E00000000636D642070726FD5
:10F8DA0063657373000000E904D331000000000A75
:10F8EA00003C00130A6162636465666768696A6B53
:10F8FA006C6D6E6F7020090D0015051A22FFCC3B46
:10F90A0022FFCC3BED478A3C010010001D0040005D
:10F91A00E2062207670800000000C039B43918104F
:10F92A00000000004576656E742074696D6572008A
:10F93A0000004405A83D000000004374696D65722B
:10F94A002070726F636573730000005A05DE3E0013
:10F95A00000000020306070A0B0E0F284329203273
:10F96A00303132204865726A756C66005574766566
:10F97A00636B6C696E6720202020202000436F6E25
:10F98A0074696B6920322E3500C600C500C400C1F7
:10F99A0000C200000000CE00CD00CC00C900CA00A1
:10F9AA000000000000000200000000A04C0000005F
:10F9BA000052463233302064726976657200000064
:10F9CA00D105505100000000AD4FEA4E9F51E1525F
:10F9DA004050434F4E4D484D384E294F00010101CA
:10F9EA000101010101010101010101010052696DD9
:10F9FA0065000D0652541D5461646174612E6E7562
:10FA0A006D20776179206F75742074686572653A24
:10FA1A002025640A008B558A559457B858EA56002F
:10FA2A0080C0E0F0F8FCFEFF6E756C6C6D616300DF
:10FA3A004806645949594F5955595B59615973696F
:10FA4A0063736C6F776D6163005E06755AD9596E80
:10FA5A005965597F5A6B59BA000800E110E9103507
:10FA6A00000200B916BB165443502F495020737434
:10FA7A0061636B0000008706BC5C0000000002089E
:0CFA8A0000000000FFFFFFFF0100000073
:00000001FF
